:100000000C94E8080C9437090C9437090C943709C0
:100010000C9437090C9437090C9437090C94370960
:100020000C9437090C94DE1B0C9437090C94370997
:100030000C94EE350C9437090C9437090C9437095D
:100040000C9437090C9437090C9448180C94370910
:100050000C94760E0C9437090C94400E0C943709CE
:100060000C94CE1E0C9437090C9474310C943709FF
:100070000C94348B0C9437090C9412840C9437092B
:100080000C9437090C9437090C943709F51EFA1EA5
:10009000FF1E081F1F1F361F461F561F911F7A2164
:1000A000361F3C204D207C209A20B72011216C2146
:1000B00087235424E32463259B253E264528AF2827
:1000C00029297229BC29EA29172A7A2AC42A0E2B3F
:1000D000072C9331C7310A327A329232D3328A33C3
:1000E00051345134513451345134513451345134E8
:1000F000513451345134063408340D342534273406
:10010000B6755076D67638778C77F577B17F767876
:10011000A878A878A878A878A878A878A878A878DF
:10012000A878D6785179E6790B7A4E7AA67A317B1F
:100130001A7C817C817C817C817C817C817C817C3E
:10014000817C817CB77CD57CFA7C567D8E7DFD7D63
:100150002A7ECA7EB17F1F7F1F7F1F7F1F7F1F7F69
:100160001F7F1F7F1F7F87898A898A898A89938950
:1001700096899989AB89A8890A0D3D3D3D3D3D3D54
:100180003D3D3D3D3D3D3D3D3D3D3D3D3D3D3D3D9F
:100190003D3D3D3D3D3D3D3D3D3D3D3D3D000A0D2F
:1001A000426174743A002025642043656C6C7320AE
:1001B00000204C6F77207761726E696E673A202558
:1001C000642E2564000A0D466F756E6420424C2D26
:1001D0004374726C3A20002564000A0D0A0D212137
:1001E000204D495353494E4720424C2D4354524CC5
:1001F0003A202564202121000A0D43616C69627256
:100200006174696E672070726573737572652073AF
:10021000656E736F722E2E004F4B0A0D000A0D464D
:100220006C696768742D74696D65202575206D692A
:100230006E20546F74616C3A2575206D696E0041B3
:100240006E676C654E69636B202020202020204162
:100250006E676C65526F6C6C20202020202020413E
:1002600063634E69636B20202020202020202041E2
:100270006363526F6C6C20202020202020202059A6
:1002800061774779726F202020202020202020488D
:1002900065696768742056616C756520202020416F
:1002A00063635A2020202020202020202020204767
:1002B0006173202020202020202020202020204387
:1002C0006F6D706173732056616C756520202056C8
:1002D0006F6C74616765205B302E31565D20205253
:1002E00065636569766572204C6576656C2020478C
:1002F00079726F20436F6D70617373202020204DE1
:100300006F746F7220312020202020202020204D6B
:100310006F746F7220322020202020202020204D5A
:100320006F746F7220332020202020202020204D49
:100330006F746F7220342020202020202020203154
:100340003620202020202020202020202020203186
:100350003720202020202020202020202020203175
:100360003820202020202020202020202020203164
:100370003920202020202020202020202020205331
:100380006572766F20202020202020202020204809
:100390006F76657267617320202020202020204323
:1003A000757272656E74205B302E31415D20204382
:1003B00061706163697479205B6D41685D202048DC
:1003C000656967687420536574706F696E74203254
:1003D00035202020202020202020202020202032F6
:1003E00036202020202020202020202020202043D4
:1003F0006F6D7061737320536574706F696E7449AB
:1004000032432D4572726F7220202020202020421E
:100410004C204C696D69742020202020202020472A
:1004200050535F4E69636B202020202020202047FE
:1004300050535F526F6C6C20202020202020202100
:10044000212120494E434F4D50415449424C4520B3
:10045000212121002A002E000A0D20444143206F53
:100460007220493243204552524F52212043686541
:10047000636B204932432C2033567265662C20442E
:10048000414320616E6420424C2D4374726C005BCA
:1004900025695D005B25695D002B204D696B726FDE
:1004A0004B6F70746572202B0048573A5625642EA6
:1004B00025642053573A25642E256425632056343D
:1004C0000053657474696E673A2564202573004D86
:1004D00069786572204572726F722100455252250B
:1004E00032643A00486172647761726520457272C5
:1004F0006F7220313A2564202121004D69737369A0
:100500006E6720424C2D4374726C3A2564212100A1
:10051000493243204552524F5221212100486569FA
:100520006768743A202025356900536574706F69D7
:100530006E743A2535690050726573737572653A49
:10054000253569004F66667365743A202025356944
:100550000048656967687420636F6E74726F6C0021
:1005600044495341424C4544006163742E20626506
:100570006172696E67004E69636B3A20202020200B
:100580002025356900526F6C6C3A202020202020F5
:1005900025356900436F6D706173733A2020202503
:1005A0003569004B25693A25346920204B25693A85
:1005B00025346920004E693A2534692020526F3A6B
:1005C000253469200047733A253469202047693A69
:1005D000253469200050313A253469202050323AC0
:1005E000253469200050333A253469202050343AAC
:1005F00025346920004779726F202D2053656E7372
:100600006F72004E69636B25346920282533692E8B
:1006100025692900526F6C6C2534692028253369BF
:100620002E256929004769657225346920282533FC
:100630006929004E69636B202534692028253369B8
:100640002E25782900526F6C6C20253469202825CE
:1006500033692E25782900596177202025346920B7
:100660002825336929004E69636B202534692028C9
:1006700025336929282533692900526F6C6C2025A0
:1006800034692028253369292825336929005961CF
:1006900077202025346920282533692928253369C6
:1006A0002900414343202D2053656E736F72004E25
:1006B00069636B2025346920282533692900526F2E
:1006C0006C6C20253469202825336929005A2020A4
:1006D000202025346920282533692900566F6C7441
:1006E0006167653A2020202533692E25316956003F
:1006F00043757272656E743A2020202533692E2569
:1007000031694100506F7765723A20202020202502
:10071000346957004469736368617267653A2025DC
:1007200035696D416800526563656976657200528E
:10073000432D525353493A2020202025346900523A
:10074000432D5175616C6974793A202534690052E2
:10075000432D4368616E6E656C733A2534690043BE
:100760006F6D70617373004D61676E65743A202020
:1007700020253569004779726F3A202020202025F6
:10078000356900536574706F696E743A2025356958
:1007900000506F746925693A202025336900506F35
:1007A000746925693A202025336900536572766F94
:1007B000202000536574706F696E742020253369A2
:1007C00000506F736974696F6E3A20253369005267
:1007D000616E67653A2533692D25336900424C2DDA
:1007E0004374726C204572726F72732000253364FB
:1007F0002025336420253364202533642000424CB7
:100800002054656D7065726174757265002533647E
:100810002025336420253364202533642000424C96
:100820002D4374726C20666F756E64200020256302
:1008300020202025632020202563202020256320E0
:1008400000202563202020256320202025632020F0
:1008500020256320002025632020202D2020202D0E
:100860002020202D2000313000313100313200466F
:100870006C696768742D54696D65202000546F742D
:10088000616C3A2535756D696E004163743A2020BC
:100890002535756D696E0028726573657429000AC7
:1008A0000D47656E65726174696E67206465666187
:1008B000756C7420506172616D657465722053654A
:1008C00074202564000A0D5573696E6720506172AB
:1008D000616D6574657220536574202564000A0D8E
:1008E00047656E65726174696E67206465666175DF
:1008F0006C74204D69786572205461626C65000AE1
:100900000D4D697865722D436F6E6669673A2027D1
:1009100025732720282575204D6F746F7273290069
:100920000A0D414343206E6F742063616C696272EB
:1009300061746564210D0A0000008F001E01AD0185
:100940003B02CA025803E603740402058F051B0626
:10095000A7063307BE074808D2085B09E3096B0AFC
:10096000F20A780BFD0B810C040D860D070E870E25
:10097000060F840F00107B10F5106E11E5115B124D
:10098000CF124213B31323149214FE146A15D31515
:100990003B16A11605176717C81727188318DE1806
:1009A00037198E19E319361A871AD61A231B6E1BAC
:1009B000B61BFD1B411C831CC31C001D3C1D751D6B
:1009C000AB1DE01D121E421E6F1E9A1EC31EE91EA5
:1009D0000D1F2E1F4D1F691F841F9B1FB01FC31F9C
:1009E000D31FE11FEC1FF51FFB1FFF1F002000009E
:1009F00005000500040106010800060102000400CC
:100A000004000700070007000700070007000700B1
:100A100003010301050017010F01060009010A0186
:100A200019010501050119011A010F014E6F204539
:100A300072726F722020202020202020004E6F74C0
:100A400020636F6D70617469626C652020004D4B8E
:100A5000334D6167206E6F7420636F6D7061004E5F
:100A60006F20464320636F6D6D756E69636174001E
:100A70004D4B334D616720636F6D6D756E696361BA
:100A80000047505320636F6D6D756E6963617469C3
:100A90006F00636F6D706173732076616C75652094
:100AA0002020005243205369676E616C206C6F7385
:100AB000742020004643207370692072782065728C
:100AC000726F7220004E6F204E4320636F6D6D7504
:100AD0006E69636174004643204E69636B204779F9
:100AE000726F2020202000464320526F6C6C2047FC
:100AF00079726F20202020004643205961772047DB
:100B000079726F2020202020004643204E69636BBD
:100B100020414343202020202000464320526F6C78
:100B20006C204143432020202020004643205A2DA2
:100B30004143432020202020202020005072657354
:100B4000737572652073656E736F7220004932434E
:100B50002046432D3E424C2D4374726C2000426C63
:100B6000204D697373696E67202020202020004D7E
:100B700069786572204572726F72202020202000F3
:100B80004361726566726565204572726F722020DE
:100B90000047505320466978206C6F7374202020E2
:100BA00020004D61676E6574204572726F7220205F
:100BB0002020004D6F746F722072657374617274BF
:100BC00020202000424C204C696D69746174696F6B
:100BD0006E202020004750532052616E6765202010
:100BE0002020202020004E6F2053442D436172644A
:100BF0002020202020200053442D4C6F6767696E11
:100C000067206572726F7200466C79696E67207238
:100C1000616E676521202020004D617820416C7451
:100C2000697475646521202020004E6F2047505361
:100C30002066697820202020202000202121204CBF
:100C400069506F20766F6C746167652021212020C8
:100C50000020202020204D696B726F4B6F707465EF
:100C60007220202020200020202020202020202052
:100C7000202020202020202020202020002020258F
:100C800032692E2531695620200020202532692E18
:100C900025316956202000414C543A2534696D2095
:100CA000256300414C543A2534696D202000414CA5
:100CB000543A2D2D2D2D200020202532693A253043
:100CC000326920200020202532693A2530326920FF
:100CD00020004449523A2025336425630043002014
:100CE000002020253569202000202025356920207E
:100CF00000493A2532692E2531694120003A003AEF
:100D0000003A002D2D2D2D2D2D2D2D2D2B2D2D2D62
:100D10002D2D2D2D2D2D2D2D002D2D2D2D2D2D2D30
:100D20002D2D2D2D2D2D2D2D2D2D2D2D2D2D003A13
:100D3000005341543A2532642000444953543A2523
:100D400033646D004420003344002121004D4147AD
:100D50003A25337525252000484D3A25336425630F
:100D600020256300696E636C3A253264256328256B
:100D700032692900202020202532756D2F733A20FA
:100D800020484D3A2533642563202563004552529F
:100D90003A202532642021004552523A2000212178
:100DA000204C69506F20766F6C746167652021213B
:100DB00000207777772E4D696B726F4B6F7074657B
:100DC000722E6465202000202532693A2530326970
:100DD00020202532692E25316956202534696D4140
:100DE0006800202532693A25303269202025326991
:100DF0002E25316956202534696D416800444952D9
:100E00003A253364256300414C543A2534696D001A
:100E1000414C543A2534696D00414C543A2D2D2DE6
:100E20002D2000256300484D3A253364256320209A
:100E3000444953543A2533646D202563005057527A
:100E40003A2532692E253169412028256957292004
:100E5000004346002020004750533A2532756D2F3D
:100E600073205341543A256420002020334420004D
:100E70004E4F464958004447505320002020204EF2
:100E80006F204E6176694374726C202020202020F0
:100E900020002532692E2569202532692E256920FA
:100EA0002532692E2569202532692E2569410025C4
:100EB000336920253369202533692025336925636B
:100EC00043002532692E2569202532692E25694186
:100ED000002532692E2569202532692E25692025B5
:100EE00032692E2569202532692E25694100253376
:100EF00069202533692563432020202020202020DD
:100F0000002533692025336920253369202533697D
:100F1000256343004552523A202532642021004582
:100F200052523A20002121204C69506F20766F6C7C
:100F30007461676520212100207777772E4D696BDA
:100F4000726F4B6F707465722E646520200053655C
:100F50007474696E673A257520257320004D696E9B
:100F60003A2532692E253169562025732000414CDF
:100F7000543A00504F54493A2533752000284F4EBB
:100F800029202000284F46462920004C494D49542D
:100F900000564152494F0044495341424C45440098
:100FA00043463A0044495341424C45440020284FAF
:100FB0004E29200020284F46462900205445414311
:100FC00048004750533A0044495341424C4544007D
:100FD0002846524545290028484F4D4529002841BB
:100FE000494429200028484F4C4429002046533AC0
:100FF000257573656B2000484F4D4520414C543A90
:101000000025756D00484F4C4420004E693A253448
:101010006920526F3A25346920433A2533690047E5
:10102000733A2534692059613A25346920005031DA
:101030003A2534692050323A25346920333A253331
:10104000690050343A2534692050353A25346920F6
:10105000363A25336900434F55504C494E47204F8F
:1010600046462120004C4F4F50494E472120004812
:1010700048212000434F4D50415353204F464621B5
:101080002000537065616B3A00416C6C204D6573B4
:10109000736167657320005761726E696E677320B4
:1010A0006F6E6C7900557365202873657429207400
:1010B0006F2073656C656374000A0D7777772E4D2A
:1010C000696B726F4B6F707465722E646520286354
:1010D0002920486953797374656D7320476D6248A0
:1010E000000A0D74686520757365206F662074684A
:1010F000697320736F667477617265206973206FFE
:101100006E6C79207065726D6974746564200A0D67
:101110006F6E206F726967696E616C204D696B72CA
:101120006F4B6F707465722D486172647761726580
:10113000005573657200486F545420563400414383
:10114000542044534C004A657469005370656B74B5
:1011500072756D0050504D000A0D526563656976D9
:1011600065723A2000532E42757300756E6B6E6F78
:10117000776E2E205573696E672050504D2E2E2E9F
:10118000006E6F7420737570706F72746564206286
:101190007920686172647761726521000A0D466C7E
:1011A00069676874436F6E74726F6C0A0D48617280
:1011B00064776172653A25642E25640A0D536F6663
:1011C00074776172653A5625642E25642563200084
:1011D00011241FBECFEFD0E4DEBFCDBF11E0A0E0F1
:1011E000B1E0E6E2FCE101E00BBF02C007900D9226
:1011F000A83AB107D9F71AE0A8EAB1E001C01D92F8
:10120000A038B107E1F77AEAE2E0F0E081E280930A
:101210005700D4907E010894E11CF11C20EF37EFB9
:1012200041E050E087016FE0DA01C9012F5F3F4FD5
:101230004F4F5F4FABBFFC018791F80181938F0146
:10124000615067FFF1CFF7016EE0819178277095CB
:10125000615067FFFACF8889781729F0F7E9DF1620
:1012600011F40000FECF0E940A0A0C94128E0C9416
:10127000000088E791E09F938F938CE295E19F9324
:101280008F93E0910204F091030409950F900F9061
:101290000F900F90089580914906E82FFF27EE0FD9
:1012A000FF1FE558F84F808191818D5E9F4F14F0AC
:1012B00010920201808191818A5B9F4FCCF48091D2
:1012C00002018823A9F481E0809302018091360411
:1012D0008F5F80933604853038F088EE93E09093EA
:1012E000DD018093DC0104C066E970E00E9488396A
:1012F0008091360499279093CE058093CD0508956B
:101300001F93CF93DF93182F882389F08EE991E004
:101310009F938F938CE295E19F938F93E0910204CA
:10132000F091030409950F900F900F900F9080910A
:101330006C06823308F044C084EF91E00E943B19B0
:10134000EC01112329F0CE010E9444198823D9F31E
:10135000C2E0D0E026E530E080911D0190911E01B1
:101360008217930730F02196255D3F4FC730D10596
:1013700098F380916C069927C89F9001C99F300D02
:10138000D89F300D1124209300011123D9F068EC6F
:1013900070E08C2F0E948839DF93CF9386EA91E02A
:1013A0009F938F938CE295E19F938F93E09102043A
:1013B000F091030409958DB79EB706968DBF02C0C4
:1013C00080930001112311F1809100016AE00E94D5
:1013D000658D892F99279F938F93809100010E949B
:1013E000658D99279F938F9381EB91E09F938F93C6
:1013F0008CE295E19F938F93E0910204F0910304B6
:1014000009952DB73EB7285F3F4F2DBFDF91CF9194
:101410001F910895CFEFD0E4DEBFCDBF882499247B
:1014200014B815B8B7EEEB2EB3E0FB2E2EEC3FEF61
:10143000E20EF31EF7FEFACF85E18093010181E809
:1014400087B93E9A8FEF88B98BE184B911E015B95D
:101450008EE38AB987E48BB9469A84B7877F84BFC5
:10146000809160008861809360001092600084EC3D
:1014700099E09093DD018093DC011092E8021092D4
:10148000E7021092800710927F071092EA021092F2
:10149000E9021092EC021092EB0284EC94E0A0E0DE
:1014A000B0E08093420190934301A0934401B09334
:1014B000450128980E94A4190E9475190E943415AC
:1014C0000E94C5350E945F1D812F0E9428310E9415
:1014D000C0670E94FD700E94FF89809101018C30DD
:1014E00010F4299A01C0299878940E94473080917D
:1014F0002302826080932302109226020E94B74446
:1015000084EF91E00E943B197C018091230280FDD1
:1015100005C0C7010E9444198823B9F385EC91E006
:101520009F938F93ACE2AA2EA5E1BA2EBF92AF9201
:10153000E0910204F0910304099580EA9FE00E9483
:101540003B197C0100E010E00F900F900F900F907E
:10155000CDE1D7E0F1EDCF2EF6E0DF2E0E94B744CB
:101560008091230280FD05C0C7010E944419882391
:10157000B9F3F60180811816A4F40BC00E94B74499
:101580008091230280FD05C0C7010E944419882371
:10159000B9F3C7010E944419882319F4888188236C
:1015A0006CF7888187FF1BC00F5F1F4F1F930F933E
:1015B0000150104087ED91E09F938F93BF92AF92BF
:1015C000E0910204F091030409958091A9018F5FD5
:1015D0008093A9012DB73EB72A5F3F4F2DBF0F5F04
:1015E0001F4F84E090E0C80ED91E28960C301105DC
:1015F00008F4B4CF00E010E0CAE1D7E0E1EDEE2E50
:10160000E6E0FE2E8B8187FD1FC0F7018081181652
:10161000DCF40F5F1F4F1F930F93015010408AEDB2
:1016200091E09F938F938CE295E19F938F93E0914C
:101630000204F0910304099582E08093DA012DB74A
:101640003EB72A5F3F4F2DBF8B8180788B830F5F22
:101650001F4F84E090E0E80EF91E28960C3011052B
:1016600088F20E943909909147068091A901981744
:1016700028F480911C04806180931C0488EF91E021
:101680009F938F93CCE2D5E1DF93CF93E091020457
:10169000F0910304099588EE93E00E943B197C01C8
:1016A0000E94651D0F900F900F900F90C7010E9430
:1016B00044198823D9F388E192E09F938F93DF93B5
:1016C000CF93E0910204F0910304099580E00E9419
:1016D000573A809101010F900F900F900F908A3030
:1016E00011F0843110F0289801C0289A80ED97E01D
:1016F0009093DD018093DC0185E5809338048EE0D2
:1017000090E00E946B2E9927182F00278FE090E021
:101710000E946B2E080F111D1093AF010093AE01B4
:101720008AE090E00E946B2E9927182F00278BE00B
:1017300090E00E946B2E080F111D1093AD010093D5
:10174000AC010F5F1F4F39F08091AE019091AF0156
:101750008F5F9F4F41F41092AF011092AE01109233
:10176000AD011092AC018091AC019091AD019F93BD
:101770008F938091AE019091AF019F938F938DE1F4
:1017800092E09F938F93DF93CF93E0910204F091C7
:10179000030409950E94F92288E893E190933D01A2
:1017A00080933C01C1E0C09337048C2F0E948009D4
:1017B00080916F060E944B890E94390980ED97E065
:1017C0000E943B197C018AEF90E00E943B1983E064
:1017D0008093A5051092A8018091B5062DB73EB75C
:1017E000285F3F4F2DBF84FF02C0C093B00180919E
:1017F000B201882311F04798FECF8091E001882341
:1018000009F436C280910F01882309F431C2109285
:10181000E00180913604882319F00E944B0902C030
:101820000E94F6470E94B744209101012A3011F02E
:10183000243110F0289801C0289A8091DB02882377
:1018400031F08091DB0281508093DB020EC08091E9
:101850006F00806280936F0010927C0710927B076C
:1018600080911C04886080931C0480913C019091BD
:101870003D01019790933D0180933C0180913C0193
:1018800090913D01892B21F0809124028823C9F198
:1018900080913C0190913D01892BD9F40E945231F5
:1018A00085E090E090933D0180933C018091DF05BD
:1018B0009091E00501969093E0058093DF0580917B
:1018C0001C04816080931C048091A6058260809333
:1018D000A60580910701909108018F5F9F4FC1F489
:1018E0008091DA028823A1F088EA91E69093DD01E5
:1018F0008093DC0180E890E09093080180930701D9
:1019000007C02A3011F0243110F0289801C0289A1D
:101910000E94B78A8091E001882309F0A9C18091D3
:10192000E903882319F00E943580A2C180910D013E
:10193000882311F00E94BB190E9478150E94C610DE
:10194000C7010E944419882309F48EC184E190E004
:10195000E80EF91E80916F06863011F40E947A75A8
:1019600080912402882349F080911C048260809336
:101970001C048091A60582600FC08091DC019091CB
:10198000DD01892B59F480913C0190913D0107972D
:1019900028F08091A6058D7F8093A6058091B001E7
:1019A000882361F08091DB02873940F01092B0010A
:1019B00088E893E19093DD018093DC01809104013C
:1019C000882321F08150809304012EC0809342042B
:1019D0001092AF021092AE021092AD021092AC02C1
:1019E0001092AB021092AA028091DB028823E1F4EC
:1019F00080910701909108018F5F9F4FA9F420917A
:101A0000B001223089F088E99AE39093DD01809358
:101A1000DC0180E09CE09093080180930701222381
:101A200019F082E08093B00180919B01893C48F0DD
:101A3000815080939B0180911C048B7F80931C04B8
:101A40003FC080915C088823F9F080911C04846079
:101A500080931C0489E08093B603809107019091E4
:101A600008018F5F9F4F81F48091DA02882361F033
:101A700088E99AE39093DD018093DC0180E098EAA5
:101A800090930801809307011092A8031092A70376
:101A90001092A6031092A5031092A40310924F086F
:101AA00010928E0810928D081092900810928F0854
:101AB0008FEF9FEF90938C0880938B0810929B017F
:101AC00080910001282F332780911D0190911E01E4
:101AD00082179307CCF48091A30280628093A302C3
:101AE00080910701909108018F5F9F4FC1F480E7BB
:101AF00097E19093DD018093DC0180E093E0909387
:101B00000801809307010BC08091DC019091DD01F9
:101B1000892B29F48091A3028F7D8093A3020E94D8
:101B2000966C84E08093DB018091B1018F5F80939C
:101B3000B101813309F04FC01092B1018091A3022D
:101B400081FF0AC08091AA019091AB010196909308
:101B5000AB018093AA013FC05AEA852E55E0952E2D
:101B60008091EC059091ED059C01442737FD40954F
:101B7000542F8091150190911601A0911701B091F9
:101B80001801281739074A075B0734F48091EC05E0
:101B90009091ED0501961BC08091EC059091ED05AB
:101BA0009C01442737FD4095542F80911501909159
:101BB0001601A0911701B091180182179307A4078D
:101BC000B5074CF48091EC059091ED050197909349
:101BD000ED058093EC050894811C911C32E7831677
:101BE0003BE0930609F040C0882499242091AE017F
:101BF0003091AF012F5F3F4F3093AF012093AE0183
:101C00008091AC019091AD0101969093AD018093CC
:101C1000AC01832F9927682F8EE090E00E94732EED
:101C20008091AE019091AF019070682F8FE090E0AD
:101C30000E94732E8091AC019091AD01892F99275C
:101C4000682F8AE090E00E94732E8091AC01909101
:101C5000AD019070682F8BE090E00E94732E84E1BC
:101C600090E00E943B197C010E94E66C0E94147176
:101C70008091DB01882309F0BACD0E94E167B7CDDE
:101C80001F920F920FB60F9211248F939F93EF9391
:101C9000FF93809106018823E1F48091CC0190911B
:101CA000CD0101969093CD018093CC01FC01EA50C7
:101CB000FB4FE081ED3019F08F3A910539F4109225
:101CC000CD011092CC0181E080930601E093C60023
:101CD00004C01092CD011092CC01FF91EF919F9121
:101CE0008F910F900FBE0F901F9018951F920F921B
:101CF0000FB60F9211242F933F934F935F936F93DF
:101D00007F938F939F93AF93BF93CF93EF93FF9363
:101D100090E08091B201813029F48091C6008093D7
:101D2000CE00CCC08091B201823029F48091C600EF
:101D300080934504C3C08091C6008093C401509134
:101D4000D2015F3A10F09093D3018091C4018D309D
:101D500009F065C08091D301823009F060C0909392
:101D6000D301852F99278B5B9B4FFC0132974081D4
:101D70002091CE013091CF01241B3109DC01119754
:101D80008C91281B3109C9019F709093CF018093DA
:101D9000CE0146E0969587954A95E1F7982F935C9A
:101DA0009093D0012F733070235C2093D1018081F8
:101DB000981729F48C91281711F491E006C090E04F
:101DC0008091C1018F5F8093C101C091C301CC2379
:101DD00009F074C0992309F471C081E08093C301B4
:101DE000580F5093C0015150E52FFF27EB5BFB4F7D
:101DF0008DE0808380914704823509F05FC00E94A6
:101E0000F92288E190E02CE00FB6F894A895809331
:101E100060000FBE20936000C093DA014FC0209194
:101E2000D301822F992781309105F9F082309105F5
:101E30001CF4892B21F040C0029711F13DC0809124
:101E4000C401833239F48091C301882319F481E0FD
:101E50008093D3018091C4018093450481E08093F5
:101E6000D2018091C401992722C02F5F2093D30112
:101E7000E52FFF27EB5BFB4F8091C401808309C0F6
:101E8000E52FFF27EB5BFB4F8091C40180835F3A16
:101E900020F45F5F5093D20102C01092D3012091D1
:101EA000C4018091CE019091CF01820F911D90933A
:101EB000CF018093CE0102C01092D301FF91EF9128
:101EC000CF91BF91AF919F918F917F916F915F91D2
:101ED0004F913F912F910F900FBE0F901F9018952B
:101EE000AC01A0E0B0E09D01A817B90748F4E6EF07
:101EF000F4E08191280F311D1196A417B507C8F39E
:101F00003F70FD01EA50FB4FC90156E09695879559
:101F10005A95E1F7835C80831196FD01EA50FB4FEF
:101F20002F733070822F835C8083A950BB4F8DE06C
:101F30008C93109206018091F6048093C600089558
:101F4000A0E0B0E0E6EAFFE00C94DE8D2C859D85F4
:101F50000E85BB2483E28093F6049F599093F70487
:101F60002093F80433E0E32EF12C002309F49EC003
:101F7000CF84D888BE016D5E7F4FA989BA89015090
:101F8000109709F493C01097B9F0F601EB0DF11D0D
:101F9000B3949081119791F4002349F1FB016E5F96
:101FA0007F4FDB01C080D1806E5F7F4F0D90BC9171
:101FB000A02DBB24015002C090E019C01097B9F0C9
:101FC000F601EB0DF11DB3944081119791F40023BC
:101FD00041F1FB016E5F7F4FDB01C080D1806E5FFE
:101FE0007F4F0D90BC91A02DBB24015002C040E05A
:101FF00018C01097B1F0F601EB0DF11DB3941081EC
:10200000119781F4002371F0FB013296DB01CD9032
:10201000DC90BF016E5F7F4FA081B181BB24015076
:1020200001C010E0F701EA50FB4F892F8695869595
:10203000835C80830894E11CF11CF701EA50FB4F9C
:10204000892F99278370907024E0880F991F2A9513
:10205000E1F755279A0194E0369527959A95E1F78F
:10206000822B835C80830894E11CF11CF701EA5009
:10207000FB4F4F705070440F551F440F551F812F59
:10208000992726E0969587952A95E1F7842B835C1E
:1020900080830894E11CF11CF701EA50FB4F1F7389
:1020A000135C10830894E11CF11C6ACFC7010E94E5
:1020B000700FE9E00C94FA8DA3E07A2F4091C001F3
:1020C0004650442309F458C0E72FFF27EB5BFB4F32
:1020D00080818D537F5FE72FFF27EB5BFB4F2081D4
:1020E0002D537F5FE72FFF27EB5BFB4F30813D5385
:1020F0007F5FE72FFF27EB5BFB4F60816D537F5FB7
:102100009927880F991F880F991F522F52955F703A
:10211000582B822F99278F709070F4E0880F991FA9
:10212000FA95E1F7232F26952695282B832F9927BB
:1021300083709070E6E0880F991FEA95E1F7682BAD
:1021400041504F3FC9F0EA2FFF27EB5BFB4F508315
:10215000AF5F41504F3F81F0EA2FFF27EB5BFB4F12
:102160002083AF5F41504F3F39F0EA2FFF27EB5BF1
:10217000FB4F6083AF5FA5CF88E494E09093BF01ED
:102180008093BE01A350A093BD010895A2E0B0E0EA
:10219000ECECF0E10C94E48D8091C301882309F408
:1021A00057C40E945C1080914604823609F023C314
:1021B0008091470499278037910509F4AFC0813792
:1021C0009105C4F48A36910509F480C28B369105D5
:1021D00044F48B34910571F18636910509F45FC1A1
:1021E0000AC38D36910509F469C08E36910509F44C
:1021F0004DC001C38437910541F1853791054CF4F9
:102200008137910509F491C08337910509F4DFC046
:10221000F2C28737910509F41BC2883791052CF467
:102220008537910509F4D7C1E6C28937910509F4CC
:102230006DC1E1C2E091BE01F091BF018081918149
:1022400090938F0180938E01D6C28091C001A0919E
:10225000BE01B091BF01853140F080E1E0E2F4E0E1
:102260000D9001928A95E1F70DC08D919D910D9091
:10227000BC91A02D8093200490932104A09322046C
:10228000B093230480EF8093BB014BC08091060183
:102290008823E1F38DE490E09F938F9384EC96E0A4
:1022A0009F938F9381E08F938F938EE48F930E94FF
:1022B000A00F8DB79EB707968DBF9DC2A091BE019E
:1022C000B091BF011C91113081F48DE4E4ECF6E093
:1022D0000D9001928A95E1F70E94842F19838091D5
:1022E0001C048F7E80931C0401C01982809106011A
:1022F0008823E1F381E090E09F938F93CE010196D4
:102300009F938F9381E08F938F938DE48F930E949F
:10231000A00FADB7BEB71796ADBF6DC281E0809379
:10232000C6018FEF8093040166C2E091BE01F09177
:10233000BF01E0818E2F8A508A3058F48983882328
:1023400011F481E003C0863010F085E0898361E0FC
:102350000EC08E2F84518A3070F48983882311F443
:1023600081E003C0863010F085E0898360E08981D8
:102370000E94043012C0E983EF3F19F40E94E72F56
:1023800089838981882311F481E003C0863010F0AD
:1023900085E0898389810E94892E809106018823A6
:1023A000E1F38BE790E09F938F9388E496E09F930F
:1023B0008F9381E090E09F938F93CE0101969F933E
:1023C0008F9382E08F9381E08F9381E577C1209195
:1023D000BE013091BF01D9018C918150853008F048
:1023E00045C0F90181818B3509F040C08091DA0246
:1023F0008823E1F52F5F3F4F8BE7E8E4F6E0D90152
:102400000D9001928A95E1F7F90182910E94F42ED4
:10241000809189069927AA27BB27BC01CD0124EC0E
:1024200039E040E050E00E94468DDC01CB01809312
:10243000860190938701A0938801B09389018091D0
:102440008A069927AA27BB27BC01CD010E94468D89
:10245000DC01CB018093820190938301A0938401DE
:10246000B09385010E94E72F898301C01982809172
:1024700006018823E1F381E090E09F938F93CE01E2
:1024800001969F938F9381E08F938F9383E58F9332
:102490000E94A00F8DB79EB707968DBF26C0E09112
:1024A000BE01F091BF01E0818E2F8150853018F47C
:1024B0008E2F0E94892E0E94E72F8983809106012A
:1024C0008823E1F381E090E09F938F93CE01019602
:1024D0009F938F9381E08F938F9386E48F930E94D5
:1024E000A00FADB7BEB71796ADBF8091DA028823B3
:1024F00029F46EE670E089810E94883980E00E94AC
:10250000800980916F060E944B8975C1E091BE01E0
:10251000F091BF018081992787FD90959093960750
:10252000809395078181992787FD909590939807CF
:10253000809397078281992787FD909590939A07BA
:10254000809399078381992787FD909590939C07A5
:1025500080939B078481992787FD909590939E0790
:1025600080939D078581992787FD90959093A0077B
:1025700080939F078681992787FD90959093A20766
:102580008093A1078781992787FD90959093A40751
:102590008093A3078085992787FD90959093A60740
:1025A0008093A5078185992787FD90959093A8072B
:1025B0008093A7078285992787FD90959093AA0716
:1025C0008093A9078385992787FD90959093AC0701
:1025D0008093AB0710C1E091BE01F091BF018081F3
:1025E0000E941E358A83882319F481E0898301C003
:1025F0001982809106018823E1F388E090E09F939F
:102600008F9382E197E09F938F9321E030E03F9397
:102610002F938091BE019091BF019F938F933F9321
:102620002F93CE0102969F938F933F932F93CE01CA
:10263000820F931F9F938F9384E08F9381E08F93FA
:1026400085E58F930E94A00FEDB7FEB773963CC04F
:102650008091BD01893008F4CEC02091BE01309137
:10266000BF012F5F3F4F88E0A2E1B7E0F901019081
:102670000D928A95E1F7D9018E910E9474348A8374
:10268000882319F481E0898301C0198280910601B1
:102690008823E1F321E030E03F932F93CE010296AF
:1026A0009F938F933F932F93CE01820F931F9F93FE
:1026B0008F9382E08F9381E08F9387E58F930E94C1
:1026C000A00FEDB7FEB73B96EDBF95C08091DA0243
:1026D000882309F090C00E94FE888983823019F017
:1026E000843009F088C020E430E0F8948091C10083
:1026F0008F738093C1008091C9008F738093C9004C
:102700008091C100877E8093C1008091C900877E3F
:102710008093C9008091C80087FF03C08091CE00DC
:10272000F9CF8091C00087FF03C08091C600F9CF28
:10273000E091BE01F091BF01E081E13021F482E03F
:102740008093B2012EC0E43611F421E830E081E03C
:102750008093B201832F99278093CD002093CC00E2
:102760008091CD008093C5008091CC008093C400FF
:102770008091CA008F7D8093CA008091CA008F7EAD
:102780008093CA008091C9008B7F8093C90080919B
:10279000CA0084608093CA008091CA0082608093DE
:1027A000CA008091CA00877F8093CA008091C200CE
:1027B000877F8093C2008091C9008E7F8093C9007B
:1027C0008091C10088618093C1008091C9008861B7
:1027D0008093C9008091C10080688093C10080917E
:1027E000C90080688093C90010926E0010926F003B
:1027F000109270007894809147049927843691054F
:1028000009F4BBC085369105ACF48136910509F415
:102810006FC0823691052CF48B34910509F45DC0AC
:102820000FC18236910509F470C08336910509F411
:102830007FC006C18C36910509F4EDC08D36910537
:102840004CF48736910509F4F8C08836910509F4EF
:10285000B2C0F6C08437910529F08637910509F496
:10286000E8C0EEC08091C001A091BE01B091BF014F
:10287000803140F080E1E0E2F4E00D9001928A9531
:10288000E1F70DC08D919D910D90BC91A02D80938D
:10289000200490932104A0932204B09323048091F8
:1028A00006018823E1F31F92809103018F9384E551
:1028B0008F930E94A00F8AEF8093BB018FEF8093CC
:1028C000040180EA9FE00E943B199093B401809339
:1028D000B3010F900F900F90B3C0E091BE01F09143
:1028E000BF018081918190938F0180938E01A8C058
:1028F000E091BE01F091BF0180818093050180329B
:1029000098F08FE1809305010FC0A091BE01B091B6
:10291000BF018BE0E8E3F4E00D9001928A95E1F7C6
:10292000809141048093E7058FEF8093040188C074
:102930008091B7019091B801892B89F4E091BE0193
:10294000F091BF01E081EE2351F08AE0E89FC001E1
:1029500011240E943B199093130480931204E09178
:10296000BE01F091BF0190818AE0989FC0011124BF
:102970009093B8018093B70115C08FEF8093040145
:10298000E091BE01F091BF0190818AE0989FC00163
:1029900011249093BA018093B901892B19F081E039
:1029A0008093C80180EA9FE00E943B199093B40194
:1029B0008093B30145C08FEF80930401E091BE0185
:1029C000F091BF01908197FD08C082E08093C5011E
:1029D0001092B6011092B5011AC0909580911C0218
:1029E000892B80931C0291818AE0989FC001112459
:1029F0009093B6018093B50184E08093C50180EA8D
:102A00009FE00E943B199093B4018093B30181E051
:102A10008093C90115C08FEF80930401E091BE013E
:102A2000F091BF01808180931D0281E08093CA01F3
:102A300007C081E08093C70103C081E08093CB0190
:102A40001092C3011092BF011092BE011092BD01FD
:102A5000E3E0CE5F0C94008E982F8091C00085FF3C
:102A6000FCCF9093C60008950F931F9388E1809345
:102A7000C1008091C00082608093C0008091C1003D
:102A800080688093C1008091C10080648093C10000
:102A900000E010E00093C5008AE290E08093C4005B
:102AA0008091B9019091BA010E943B19909315044D
:102AB000809314048CED90E00E943B1990934404A1
:102AC000809343041092160488E5809317048DE0E8
:102AD00080931A048BE080931804109219041093C9
:102AE000BF010093BE011092BD011F910F91089587
:102AF000A0E1B0E0EEE7F5E10C94E18D80910601F4
:102B0000882309F4C1C28091B3019091B4010E945D
:102B10004419882361F01092B6011092B501109209
:102B2000BA011092B9011092B8011092B7018091C8
:102B3000B5019091B601892B41F08091F4049091F8
:102B4000F5040E944419882329F48091C90188233F
:102B500009F460C080910601882309F45BC080916C
:102B6000C50107EF15E08430A8F00E940F2380E52F
:102B700090E09F938F931F930F9381E08F938F9398
:102B800088E48F930E94A00F2DB73EB7295F3F4F77
:102B90002DBF34C010921E028FE394E09F938F9359
:102BA00082E093E29F938F93E0910204F0910304FB
:102BB000099584E190E09F938F931F930F9381E099
:102BC00090E09F938F9385EC91E09F938F9382E0A9
:102BD0008F9381E08F9388E48F930E94A00F809160
:102BE000C501982F8F5F8093C5012DB73EB7215F38
:102BF0003F4F2DBF943010F01092C5018091B50168
:102C00009091B6010E943B199093F5048093F404CF
:102C10001092C9018091CA01882351F18091060167
:102C2000882331F10E940F2380E590E09F938F93DA
:102C300087EF95E09F938F9321E030E03F932F93B0
:102C40008FE191E09F938F933F932F938DE192E0DB
:102C50009F938F9383E08F9381E08F938CE48F9386
:102C60000E94A00F1092CA018DB79EB70F968DBF1C
:102C70008091C7018823D1F0809106018823B1F0AB
:102C80008AE090E09F938F9386E194E09F938F93E7
:102C900081E08F938F9386E58F930E94A00F10920F
:102CA000C7012DB73EB7295F3F4F2DBF8091CB01A4
:102CB0008823D9F0809106018823B9F08BE090E059
:102CC0009F938F9388E394E09F938F9381E08F93FA
:102CD000809103018F9387E48F930E94A00F10923D
:102CE000CB018DB79EB707968DBF8091430490911D
:102CF00044040E944419882309F461C080910601AC
:102D0000882309F45CC0809164069927880F991F75
:102D1000880F991F7C010027F7FC0095102F8091E8
:102D2000350390913603A0913703B0913803BC016D
:102D3000CD01A80197010E94BA8D309331042093F0
:102D4000300480912D0390912E03A0912F03B09118
:102D50003003BC01CD01A80197010E94BA8D3093C8
:102D60003304209332048091B8028093340480911C
:102D7000B7028093350488E090E09F938F9380E3BF
:102D800094E09F938F9381E08F9383E08F938BE602
:102D90008F930E94A00F809136042DB73EB7295F14
:102DA0003F4F2DBF853018F086E08093360483E6D0
:102DB00090E00E943B1990934404809343048091D7
:102DC000B9019091BA01892B41F08091140490913E
:102DD00015040E944419882321F48091C801882396
:102DE00039F180910601882319F10E94723882E43A
:102DF00090E09F938F9385EA95E09F938F9381E076
:102E00008F938F9384E48F930E94A00F1092C80138
:102E10008DB79EB707968DBF8091B9019091BA0189
:102E2000009731F00E943B1990931504809314048D
:102E30008091B7019091B801892B09F4B8C08091B5
:102E40001204909113040E944419882309F4AFC01E
:102E500080910601882309F4AAC08091640699270D
:102E6000880F991F880F991F7C010027F7FC009598
:102E7000102F8091350390913603A0913703B091C4
:102E80003803BC01CD01A80197010E94BA8D30938F
:102E900005042093040480912D0390912E03A091AA
:102EA0002F03B0913003BC01CD01A80197010E940E
:102EB000BA8D309307042093060420914408309182
:102EC00045084091460850914708DA01C90163E07E
:102ED000880F991FAA1FBB1F6A95D1F7820F931FF6
:102EE000A41FB51F820F931FA41FB51F209142017D
:102EF000309143014091440150914501BC01CD0105
:102F00000E94BA8D30930904209308048091FD0239
:102F10009091FE02A091FF02B091000349E0B595A7
:102F2000A795979587954A95D1F780930A04809144
:102F3000F9029091FA02A091FB02B091FC0239E0F3
:102F4000B595A795979587953A95D1F780930B04FA
:102F50008091050390910603A0910703B0910803A7
:102F600029E0B595A795979587952A95D1F78093F0
:102F70000C048EE090E09F938F9384E094E09F9305
:102F80008F9381E08F938F9383E48F930E94A00FA0
:102F90008091B7019091B8010E943B19909313045E
:102FA000809312042DB73EB7295F3F4F2DBF80910C
:102FB00005018F3F71F1992704E0880F991F0A9549
:102FC000E1F7815C9D4F40E150E0BC01CE010196EC
:102FD0000E94998B80E190E09F938F93CE010196A0
:102FE0009F938F9381E090E09F938F9385E091E092
:102FF0009F938F9382E08F9381E08F9381E48F93EF
:103000000E94A00F8FEF809305018DB79EB70B969E
:103010008DBF8091E7058823D1F080910601882338
:10302000B1F081E090E09F938F9387EE95E09F93BE
:103030008F9381E08F938F9382E48F930E94A00FF0
:103040001092E7052DB73EB7295F3F4F2DBF809106
:10305000C6018823C9F0809106018823A9F084E382
:1030600090E09F938F938BE797E09F938F9381E0FE
:103070008F938F9380E58F930E94A00F1092C601CB
:103080008DB79EB707968DBFE6E0C05F0C94FD8DAF
:103090001F920F920FB60F9211242F933F935F93BD
:1030A0006F937F938F939F93AF93BF93EF93FF9310
:1030B00020E08091DB01882329F08091DB018150A1
:1030C0008093DB018091C903882319F0815080939C
:1030D000C9038091E30181508093E3018F3F09F0A0
:1030E0005BC089E08093E3018091E1019091E2016E
:1030F00001969093E2018093E10180910E018F5F30
:10310000817080930E01882319F481E08093E0019F
:10311000349903C081E08093E4018091DC019091B7
:10312000DD01892B21F18091DC019091DD010B976C
:1031300050F08091DC019091DD010A979093DD01C0
:103140008093DC0104C01092DD011092DC018091BB
:10315000DC019091DD01209107013091080182236B
:103160009323892B11F021E008C020E006C08FEFE7
:103170009FEF909308018093070180910101222322
:1031800031F08A3011F45A9A07C0479A05C08A3044
:1031900011F45A9801C047988091E401882309F4FA
:1031A0005AC020919B01222309F055C08091340818
:1031B00083FF51C086B19927FC01E071F07084FF54
:1031C00013C08091DE019091DF0101969093DF01A1
:1031D0008093DE018091DE019091DF01895E934052
:1031E000D0F12093E40137C08091DE019091DF019E
:1031F000892B69F18091DE019091DF018A5691401F
:1032000030F58091DE019091DF0169E270E00E946B
:10321000718D8091DE019091DF01860F971F909351
:10322000DF018093DE018091DE019091DF010B9739
:1032300050F08091DE019091DF010A9790938F0109
:1032400080938E0104C0F0938F01E0938E01109261
:10325000DF011092DE01FF91EF91BF91AF919F913D
:103260008F917F916F915F913F912F910F900FBE42
:103270000F901F9018952091E1013091E201280FE5
:10328000391FC901019608952091E1013091E201B1
:10329000821B930B892F99278695807490700895CF
:1032A000CF93DF930E943B19EC01CE010E94441999
:1032B0008823D9F3DF91CF910895CF93DF930E94B4
:1032C0003B19EC0109C080910F01882329F09093EC
:1032D0000F018FEC80937A00CE010E944419982F41
:1032E000882389F3DF91CF9108959FB7F8945F9871
:1032F0003E9A469A8091B0008F708093B000809182
:10330000B00083608093B0008091B1008B73809394
:10331000B1008091B1008B608093B1001092B20037
:103320008FEF8093B3008091B00080688093B000ED
:10333000809170008A7F809370008091700082601D
:10334000809370009FBF08958AE090E00E943B192F
:103350009093EA018093E90182E085BD83EA84BD10
:1033600017BC84EB88BD86E086BD80916E008160CD
:1033700080936E000895A0E0B0E0E1ECF9E10C94D8
:10338000E08D80917F06E82FFF27E85BFE4F968156
:10339000D08080910D01A92FBB27A7FDB095CB2F21
:1033A000DB2F813009F012C12091350330913603B3
:1033B0004091370350913803BD01CE010E94468DE4
:1033C00097FF04C061587F4F8F4F9F4F7B018C0147
:1033D00087E015950795F794E7948A95D1F78D2D99
:1033E000992787FD9095A92FB92F20912D03309112
:1033F0002E0340912F0350913003BC01CD010E9458
:10340000468D97FF04C061587F4F8F4F9F4FC7E095
:103410009595879577956795CA95D1F7F801E70156
:10342000C61BD70BE80BF90B2091AF033091B0030B
:10343000C901B3E0880F991FBA95E1F7821B930B7E
:10344000AA2797FDA095BA2FC81BD90BEA0BFB0B37
:10345000809176069927AA27BB27BC01CD019E0142
:10346000AF010E94468D97FF04C061507E4F8F4F81
:103470009F4FFC01EB01A9E0F595E795D795C7951E
:10348000AA95D1F780916D01992776E0880F991F51
:103490007A95E1F740910B0150910C0120917E0645
:1034A0003327841B950BB9010E94858D80910B01F8
:1034B00090910C01860F971F90930C0180930B0144
:1034C0008091B40680FF14C080910B0190910C0193
:1034D00097FD0F9664E0959587956A95E1F7AA2781
:1034E00097FDA095BA2FC80FD91FEA1FFB1F15C063
:1034F00080910B0190910C0197FD0F9654E09595EA
:1035000087955A95E1F7AA2797FDA095BA2F8C1BAE
:103510009D0BAE0BBF0BFD01EC012091B1062223E8
:1035200021F133278091D6019091D701829FA0018C
:10353000839F500D929F500D1124CA01AA2797FD19
:10354000A095BA2F8C0F9D1FAE1FBF1F2F5F3F4F3F
:10355000442737FD4095542FBC01CD010E94BA8D00
:103560003093D7012093D60104C0D093D701C093E4
:10357000D60180917706282F3327220F331F220F81
:10358000331F8091D6019091D701821793077CF069
:1035900080917806282F3327220F331F220F331FE5
:1035A0008091D6019091D7012817390724F43093E0
:1035B000D7012093D60180910101843108F4F7C02E
:1035C00080910D018F5F80930D01F3C020912D0339
:1035D00030912E0340912F0350913003BD01CE0155
:1035E0000E94468D97FF04C061587F4F8F4F9F4FB9
:1035F0007B018C0187E015950795F794E7948A95F0
:10360000D1F78D2D992787FD9095A92FB92F20915E
:103610003503309136034091370350913803BC0194
:10362000CD010E94468D9B01AC0197FF04C021583B
:103630003F4F4F4F5F4FC7E05595479537952795BB
:10364000CA95D1F72E0D3F1D401F511F80917A065C
:103650009927AA27BB27BC01CD010E94468D97FF61
:1036600004C061507E4F8F4F9F4FFC01EB01B9E0CA
:10367000F595E795D795C795BA95D1F780916C01E7
:103680009927A6E0880F991FAA95E1F740910901B3
:1036900050910A0120917E063327841B950BB901B6
:1036A0000E94858D8091090190910A01860F971FD4
:1036B00090930A01809309018091B40681FF14C0A0
:1036C0008091090190910A0197FD0F9674E09595FC
:1036D00087957A95E1F7AA2797FDA095BA2FC80F8D
:1036E000D91FEA1FFB1F15C08091090190910A01A3
:1036F00097FD0F9664E0959587956A95E1F7AA275F
:1037000097FDA095BA2F8C1B9D0BAE0BBF0BFD0137
:10371000EC012091B206222321F133278091D401BC
:103720009091D501829FA001839F500D929F500DD3
:103730001124CA01AA2797FDA095BA2F8C0F9D1FAF
:10374000AE1FBF1F2F5F3F4F442737FD4095542FBB
:10375000BC01CD010E94BA8D3093D5012093D401D4
:1037600004C0D093D501C093D40180917B06282F4B
:103770003327220F331F220F331F8091D4019091E2
:10378000D501821793077CF080917C06282F332780
:10379000220F331F220F331F8091D4019091D50146
:1037A0002817390724F43093D5012093D4011092BF
:1037B0000D01E7E0CDB7DEB70C94FC8D1F920F92A0
:1037C0000FB60F9211242F933F934F935F938F93D4
:1037D0009F93EF93FF93809101019091E5018431D4
:1037E00008F04CC0992309F029C18091B00086FFF0
:1037F00024C08091B0008F7B8093B0008091D6016F
:103800009091D70187559E4F9093D9018093D8010D
:1038100025E08D3D920718F08CED95E005C08757A7
:10382000914030F487E791E09093D9018093D801DB
:103830008091D8019091D901C2C08091B00080647C
:103840008093B00080917D06282F33278DED96E080
:10385000289FA001299F500D389F500D1124CA01A7
:103860002091E6013091E701821B930B9093D901DF
:103870008093D80181E080930D01DDC0992309F088
:10388000DDC08091B00086FF9FC08091B0008F7B2B
:103890008093B000E091E80120917D06EE23D9F4F9
:1038A00033278DED96E0289FA001299F500D389F6A
:1038B000500D1124CA012091E6013091E701821BCD
:1038C000930B9093D9018093D8011092E701109245
:1038D000E601469AB0C02E1738F48AE090E0909343
:1038E000D9018093D801A7C089EA93E09093D901C8
:1038F0008093D8018E2F992783309105D9F0843099
:10390000910534F48130910549F0029761F020C0AF
:103910008430910591F0059799F01AC08091D601F5
:103920009091D70104C08091D4019091D501875521
:103930009E4F1DC08091100805C08091E90702C00C
:10394000809119089927880F991F880F991FEFCF29
:10395000FF27EE0FFF1FE558F84F20813181220F1E
:10396000331F8091D8019091D901820F931F9093BA
:10397000D9018093D8018091D8019091D90155E067
:103980008D3D950718F08CED95E005C08757914067
:1039900030F487E791E09093D9018093D80120918A
:1039A000D8013091D9012C5B30403093D90120935C
:1039B000D8018091E6019091E701820F931F9093C7
:1039C000E7018093E60137C08091B0008064809366
:1039D000B0008CEB90E09093D9018093D801809156
:1039E000E6019091E70184549F4F9093E701809303
:1039F000E6018091DA01882321F08091DB0288239F
:103A000021F48091DA01823011F4469801C0469A7F
:103A10008091E8018F5F8093E801282F3327809100
:103A20007D0699270196821793072CF481E08093F5
:103A30000D011092E80181E08093E5012091D80109
:103A40003091D90141E02F37340730F08FEF809368
:103A5000B3002F5F30400FC02F3F3105C9F0C0F0D9
:103A6000A9014F5F50404F37510550F480E88093D3
:103A7000B300205830403093D9012093D80112C0B0
:103A80008FEF8093B3005093D9014093D8010AC0BF
:103A90008091D8018093B3001092D9011092D8017F
:103AA0001092E501FF91EF919F918F915F914F915E
:103AB0003F912F910F900FBE0F901F90189510926D
:103AC0007C008FEC80937A000895CF93DF9310925F
:103AD000EF0186E987BD83E090E00E946B2EC82F3E
:103AE000863E08F4C65FC8BD84E690E00E945D197A
:103AF00080911301909114018152934010F0C0EF16
:103B000002C0C530F8F0C8BD82E390E00E945D19A4
:103B100084E594E09F938F938CE295E19F938F933C
:103B2000E0910204F09103040995809113019091B2
:103B300014010F900F900F900F908152934010F44A
:103B4000C550DFCF6C2F83E090E00E94732ECF3002
:103B500018F0CCE8D0E002C0C0E0D0E0CA3FD10508
:103B6000F8F4C7BD82E390E00E945D1986E594E019
:103B70009F938F938CE295E19F938F93E091020442
:103B8000F0910304099580911301909114010F9015
:103B90000F900F900F908052934010F02196DECF3F
:103BA000C093F4058091550680FF09C08C2F8A5080
:103BB0008B3E28F080911B04806480931B04C7BD5A
:103BC0008CE291E00E945D19DF91CF910895EF9210
:103BD000FF921F93CF9310E080ED97E00E943B1976
:103BE0007C01CCE8133019F4CB3008F0C9E010E0C8
:103BF0008091FE019091FF018C5F934024F48091AD
:103C0000120181500AC08091FE019091FF018750FE
:103C1000944034F0809112018F5F8093120101C0B3
:103C200011E08091FC019091FD018C5F934024F4A0
:103C30008091110181500AC08091FC019091FD0199
:103C40008750944034F0809111018F5F809311016F
:103C500001C01F5F8091FA019091FB018C5F93403E
:103C600024F48091100181500AC08091FA01909152
:103C7000FB0187509440C4F0809110018F5F8093C6
:103C8000100113C088E594E09F938F938CE295E137
:103C90009F938F93E0910204F091030409950F9094
:103CA0000F900F900F905FC01F5F82E180932902F9
:103CB000809123028E7F8093230285EA8093BC004B
:103CC000809112018A3040F480911B0481608093BE
:103CD0001B048AE08093120180911201863F40F01C
:103CE00080911B04816080931B0485EF80931201F7
:103CF000809111018A3040F480911B04826080938E
:103D00001B048AE08093110180911101863F40F0ED
:103D100080911B04826080931B0485EF80931101C6
:103D2000809110018A3040F480911B04846080935C
:103D30001B048AE08093100180911001863F40F0BF
:103D400080911B04846080931B0485EF8093100195
:103D500080912902882339F0C7010E9444198823E1
:103D600009F090CFF5CF10920F018FEC80937A007D
:103D700080910F018823E1F3CA3020F48AE090E0BB
:103D80000E945D19C15009F02DCF86E490E00E9499
:103D90005D19CF911F91FF90EF9008951F920F92A0
:103DA0000FB60F921124EF92FF920F931F932F9350
:103DB0003F934F935F936F937F938F939F93AF93B3
:103DC000BF93EF93FF9380910702282F3327442757
:103DD00055278F5F80930702F9012231310508F0E2
:103DE000E3C3EA5BFF4F0C940C8E809178009091B6
:103DF000790046C0809178009091790047C1809108
:103E000078009091790090930A028093090272C120
:103E100080913E0390913F0320917800309179008A
:103E2000821B930B9093E9058093E8058091E80548
:103E30009091E905909314028093130279C18091C7
:103E40007800909179002091400330914103821BCA
:103E5000930B9093F3058093F2058091F205909176
:103E6000F3059093160280931502A0C380910D0272
:103E700090910E022091780030917900820F931F6B
:103E800090930E0280930D0281E091C380910B020A
:103E900090910C022091780030917900820F931F4D
:103EA00090930C0280930B0284E081C38091B5064D
:103EB00083FF1AC080911D0190911E019C01220F69
:103EC000331F280F391F40917800509179008BE003
:103ED00090E0489FB001499F700D589F700D1124CC
:103EE000CB016EE170E00FC080911D0190911E0129
:103EF0009C01220F331F280F391F80917800909169
:103F0000790063E070E00E94718D260F371F3695AF
:103F100027953695279530931E0120931D0185E046
:103F200046C3809178009091790040913A03509176
:103F30003B03841B950B9093F5018093F4018091D2
:103F4000F4019091F501029704F172E04E3E57079B
:103F500084F4209108022B5F209308022550809161
:103F6000A4029091A502845F914018F4215F2093F0
:103F7000080280910802853684F14F5F5F4F5093AD
:103F80003B0340933A03845626C08091F4019091FC
:103F9000F5018F5F9F4F0CF572E047325707ECF049
:103FA000209108022550209308022B5F8091A402E3
:103FB0009091A502845F914018F42F50209308023D
:103FC000809108028C394CF44150504050933B038F
:103FD00040933A038C598093080280917800909125
:103FE00079009093EB058093EA058091F40190911C
:103FF000F5019C01442737FD4095542F8091F5022F
:104000009091F602A091F702B091F802820F931FEF
:10401000A41FB51F8093F5029093F602A093F702B8
:10402000B093F8022091F5023091F6024091F70228
:104030005091F80257FF04C021503C4F4F4F5F4F43
:104040006AE055954795379527956A95D1F7809100
:10405000F5029091F602A091F702B091F802821B4E
:10406000930BA40BB50B8093F5029093F602A093EB
:10407000F702B093F8022EC180910B0290910C02CE
:104080002091780030917900820F931F90930C0259
:1040900080930B02109206028CC2809101018A303B
:1040A00071F480917800909179002091090230910B
:1040B0000A02820F931F01969695879517C040912B
:1040C000090250910A02843158F020917800309111
:1040D0007900240F351F8FEF97E0821B930B06C0EA
:1040E0008091780090917900840F951F9093FB0147
:1040F0008093FA0186E05BC280913E0390913F037A
:104100002091780030917900821B930B9093E90500
:104110008093E8058091E8059091E90520911302CC
:1041200030911402820F931F9093F9018093F8014C
:1041300087E03DC280917800909179002091400302
:1041400030914103821B930B9093F3058093F2050A
:104150008091F2059091F30520911502309116029D
:10416000820F931F9093F7018093F6011FC2209155
:104170000D0230910E028091780090917900280F05
:10418000391F30930E0220930D02809101018A3075
:1041900019F4220F331F04C0220F331F220F331FC5
:1041A00030930E0220930D0220910D0230910E02E9
:1041B000C90137FD079603E0959587950A95E1F7C4
:1041C0009093FF018093FE0180910F029091100265
:1041D000820F931F97FD01969595879590931002F6
:1041E00080930F0220914A0330914B03821B930B63
:1041F00090931C0180931B012091040230910502D1
:1042000080911B0190911C01280F391F37FF02C0BC
:104210002F5F3F4F35952795309305022093040279
:1042200033CE20910B0230910C0280917800909156
:104230007900280F391F30930C0220930B028091D4
:1042400001018A3019F4220F331F04C0220F331FDB
:10425000220F331F30930C0220930B0220910B028C
:1042600030910C02C90137FD0796F3E095958795CB
:10427000FA95E1F79093FD018093FC018091110282
:1042800090911202820F931F97FD01969595879545
:1042900090931202809311022091480330914903B8
:1042A000821B930B90931A018093190120910202B3
:1042B000309103028091190190911A01280F391F42
:1042C00037FF02C02F5F3F4F35952795309303028C
:1042D0002093020283E06BC11092070281E0809379
:1042E0000F018091EB019091EC0101969093EC010C
:1042F0008093EB0180917800909179009093140164
:10430000809313018091130190911401AA27BB2778
:1043100020911702309118024091190250911A020F
:10432000280F391F4A1F5B1F209317023093180272
:104330004093190250931A0280911B028F5F809361
:104340001B02803108F432C1809115019091160151
:10435000A0911701B09118017C018D0163E0EE0C72
:10436000FF1C001F111F6A95D1F7E81AF90A0A0B02
:104370001B0BE20EF31E041F151F8091EF019927FE
:1043800087FD9095A92FB92FBC01CD0120EB30E21C
:1043900040E050E00E94468DDC01CB01E81AF90AAA
:1043A0000A0B1B0BD801C7010496A11DB11DB7FF55
:1043B00005C0D801C7010B96A11DB11D23E0B5951D
:1043C000A795979587952A95D1F780931501909396
:1043D0001601A0931701B09318018091EC059091FC
:1043E000ED057C010027F7FC0095102F8091150149
:1043F00090911601A0911701B0911801E81AF90ADD
:104400000A0B1B0BE092D502F092D6020093D70262
:104410001093D8022091F0013091F1014091F20106
:104420005091F30157FF04C0215F3F4F4F4F5F4F43
:1044300084E055954795379527958A95D1F78091D2
:10444000F0019091F101A091F201B091F301821B72
:10445000930BA40BB50B8093F0019093F101A09303
:10446000F201B093F3018091F0019091F101A091DC
:10447000F201B091F3018E0D9F1DA01FB11F80931B
:10448000F0019093F101A093F201B093F3018091B8
:10449000F0019091F101A091F201B091F301B7FF09
:1044A00003C00F96A11DB11D14E0B595A795979572
:1044B00087951A95D1F72091D5023091D602281B05
:1044C000390B64E0213036071CF020E034E006C0F0
:1044D0007CEF2030370714F420E03CEF8091ED01B1
:1044E0009091EE018091ED019091EE0197FF03C054
:1044F000909581959F4FA901F3E0440F551FFA95C0
:10450000E1F78D5B9240C4F08091ED019091EE0156
:104510009C01E4E0220F331FEA95E1F7281B390BD9
:10452000240F351F37FF02C0215F3F4F74E03595E0
:1045300027957A95E1F717C08091ED019091EE01F2
:104540009C0165E0220F331F6A95E1F7281B390BA8
:10455000240F351F37FF02C0215E3F4F45E03595E0
:1045600027954A95E1F73093EE012093ED01809174
:10457000170290911802A0911902B0911A02B7FF88
:1045800003C00196A11DB11DB595A7959795879577
:104590008093170290931802A0931902B0931A0205
:1045A00088E080931B0202C01092070282E0809391
:1045B00006028091060280937C0080910702882386
:1045C00019F08FEC80937A00FF91EF91BF91AF913A
:1045D0009F918F917F916F915F914F913F912F911B
:1045E0001F910F91FF90EF900F900FBE0F901F90B3
:1045F000189590E2E7EFF5E08FE49193815087FF03
:10460000FCCF089590911E02903540F4E92FFF27CA
:10461000E950FA4F80839F5F90931E020895AF92F6
:10462000BF92CF92DF92FF920F931F93CF93DF93AE
:1046300020911C0220FF0AC080911D02882311F0E6
:10464000815002C080911F0180931D0221FF0CC088
:1046500090911D0280911F01981719F410921D026C
:1046600003C09F5F90931D02822F992780FF04C093
:1046700081FF02C010921D020E94F92280911D024A
:10468000282F332792E0C92E93E2D92EC09102043D
:10469000D09103048A3098F481E180931E023F9305
:1046A0002F938FE894E09F938F93DF92CF92FE0138
:1046B00009952DB73EB72A5F3F4F2DBF11C080E14E
:1046C00080931E023F932F9384E994E09F938F93EE
:1046D000DF92CF92FE0109958DB79EB706968DBFEA
:1046E00020911D02822F9927AA27BB27FC01419701
:1046F00010F00C94672CE85AFF4F02E0C02E03E242
:10470000D02EC0910204D09103040C940C8E109210
:104710001E0289E994E09F938F9302E013E2DF92F7
:10472000CF92FE01099584E180931E020F900F90B5
:104730000F900F908EE690E09F938F9388E590E026
:104740009F938F931F921F92809101016AE00E94B4
:10475000658D892F99279F938F93809101010E94E6
:10476000658D99279F938F9389EA94E09F938F9308
:10477000DF92CF92E0910204F0910304099588E260
:1047800080931E02EDB7FEB73E96EDBF85EC96E036
:104790009F938F930E94E72F99279F938F9381EC8C
:1047A00094E09F938F93DF92CF92E0910204F09177
:1047B0000304099580911C0499272DB73EB7285F03
:1047C0003F4F2DBFEC01C071D07084FF06C08CE359
:1047D00080931E028FEC94E0F1C09091B603992370
:1047E00049F18CE380931E02892F99279F938F9321
:1047F0008CED94E09F938F931F930F93E0910204AD
:10480000F09103040995DF93CF939091B60381E172
:10481000989FC0011124845D954F9F938F931F93A0
:104820000F93E0910204F091030409958DB79EB7B0
:104830000C9647C190911B049923B1F08CE38093AF
:104840001E02892F99279F938F9384EE94E09F9364
:104850008F931F930F93E0910204F0910304099545
:10486000EDB7FEB7369679C490912402992371F082
:104870008CE380931E02892F99279F938F938BEF50
:1048800094E09F938F931F930F93D9C480913C0121
:1048900090913D01069710F00C94702C8CE380935E
:1048A0001E0280E195E0A5C78091340812E0C12E78
:1048B00013E2D12EC0910204D091030480FF6BC09B
:1048C00010921E028091D5029091D602A091D7023B
:1048D000B091D802BC01CD0125E030E040E050E0CD
:1048E0000E94BA8D3F932F938DE195E09F938F9314
:1048F000DF92CF92FE01099584E180931E028DB76D
:104900009EB706968DBF8091D1029091D202A09160
:10491000D302B091D402BC01CD0125E030E040E0EB
:1049200050E00E94BA8D3F932F938AE295E09F93C7
:104930008F93DF92CF92E0910204F09103040995E6
:1049400088E280931E02EDB7FEB73696EDBF8091E8
:104950001301909114019F938F9387E395E09F93A8
:104960008F93DF92CF92E0910204F09103040995B6
:104970008CE380931E022DB73EB72A5F3F4F2DBFB9
:1049800087B599279F938F9384E495E09F938F93A6
:10499000DF92CF928EC010921E0281E595E09F9328
:1049A0008F93DF92CF92FE01099584E180931E02DE
:1049B0000F900F900F900F9080E695E09F938F934C
:1049C000DF92CF921AC710921E0289E695E09F935C
:1049D0008F9302E013E2DF92CF92FE01099584E10A
:1049E00080931E020F900F900F900F9080913503CF
:1049F00090913603A0913703B0913803B7FF04C0FC
:104A000081509C4FAF4FBF4FCAE0B595A795979582
:104A10008795CA95D1F7BF93AF939F938F9386E7FE
:104A200095E09F938F931F930F93E0910204F09171
:104A30000304099588E280931E02EDB7FEB738960D
:104A4000EDBF80912D0390912E03A0912F03B09183
:104A50003003B7FF04C081509C4FAF4FBF4FFAE007
:104A6000B595A79597958795FA95D1F7BF93AF938D
:104A70009F938F9385E895E09F938F931F930F9358
:104A8000E0910204F091030409958CE380931E02E7
:104A90002DB73EB7285F3F4F2DBF8091F107909112
:104AA000F2079F938F9384E995E09F938F931F93D1
:104AB0000F93E0910204F091030409958DB79EB71E
:104AC00006968DBF0DC7E1E0FE2EC1E0D0E00DE7F8
:104AD00017E09F2D969584E1989FC0011124809343
:104AE0001E02F801828193819F938F932196DF9319
:104AF000CF932197808191819F938F93DF93CF9361
:104B000083EA95E09F938F9382E093E29F938F9344
:104B1000E0910204F091030409952DB73EB7245F9C
:104B20003F4F2DBF32E0F30E22960C5F1F4F88E0FF
:104B30008F1578F6D5C610921E0280914A06E82F8E
:104B4000FF27EE0FFF1FE558F84F808191819F935B
:104B50008F9380914906E82FFF27EE0FFF1FE5583E
:104B6000F84F808191819F938F9385EB95E09F9380
:104B70008F93DF92CF92FE01099584E180931E020C
:104B8000EDB7FEB73896EDBF80914C06E82FFF27B2
:104B9000EE0FFF1FE558F84F808191819F938F930F
:104BA00080914B06E82FFF27EE0FFF1FE558F84FC7
:104BB0008081918181589F4F9F938F9385EC95E0E1
:104BC0009F938F93DF92CF92E0910204F0910304C0
:104BD000099588E280931E022DB73EB7285F3F4FAC
:104BE0002DBF80914E06E82FFF27EE0FFF1FE558DF
:104BF000F84F8081918181589F4F9F938F9380912F
:104C00004D06E82FFF27EE0FFF1FE558F84F808174
:104C1000918181589F4F9F938F9385ED95E09F934E
:104C20008F93DF92CF92E0910204F09103040995F3
:104C30008CE380931E028DB79EB708968DBF80913E
:104C40005006E82FFF27EE0FFF1FE558F84F808131
:104C5000918181589F4F9F938F9380914F06E82FAA
:104C6000FF27EE0FFF1FE558F84F80819181815893
:104C70009F4F9F938F9385EE95E063C210921E0223
:104C800085EF95E09F938F9302E013E2DF92CF923E
:104C9000FE010995809101010F900F900F900F90E8
:104CA0008A3009F09DC084E180931E0280914A03FE
:104CB00090914B039C0197FF02C0295F3F4F287FD3
:104CC000821B930B9F938F9380914A0390914B0388
:104CD00097FD079673E0959587957A95E1F79F93F1
:104CE0008F9320914A0330914B0337FF02C0295F15
:104CF0003F4F63E0359527956A95E1F78091FE0176
:104D00009091FF01821B930B9F938F9383E096E01A
:104D10009F938F931F930F93E0910204F0910304EC
:104D2000099588E280931E022DB73EB7265F3F4F5C
:104D30002DBF80914803909149039C0197FF02C0C9
:104D4000295F3F4F287F821B930B9F938F93809106
:104D500048039091490397FD079653E095958795F1
:104D60005A95E1F79F938F9320914803309149031F
:104D700037FF02C0295F3F4F43E0359527954A959D
:104D8000E1F78091FC019091FD01821B930B9F93B1
:104D90008F9384E196E09F938F931F930F93E091FD
:104DA0000204F091030409958CE380931E028DB7F1
:104DB0009EB70A968DBF80914603909147039F93BB
:104DC0008F9380914603909147032091FA0130918F
:104DD000FB01821B930B9F938F9385E296E0ADC0FE
:104DE0008B3019F0843108F4ADC084E180931E0249
:104DF00080914A0390914B039C0197FF02C0215F71
:104E00003F4F207F821B930B97FD019695958795C9
:104E10009F938F9380914A0390914B0397FD0F9638
:104E200024E0959587952A95E1F79F938F9320919C
:104E30004A0330914B0337FF02C0295F3F4FC3E065
:104E400035952795CA95E1F78091FE019091FF0174
:104E5000821B930B9F938F9383E396E09F938F9393
:104E60001F930F93E0910204F0910304099588E2E7
:104E700080931E022DB73EB7265F3F4F2DBF809116
:104E80004803909149039C0197FF02C0215F3F4F67
:104E9000207F821B930B97FD0196959587959F9395
:104EA0008F93809148039091490397FD0F96A4E05A
:104EB00095958795AA95E1F79F938F932091480345
:104EC0003091490337FF02C0295F3F4FF3E035952A
:104ED0002795FA95E1F78091FC019091FD01821BE5
:104EE000930B9F938F9385E496E09F938F931F93EB
:104EF0000F93E0910204F091030409958CE38093F1
:104F00001E028DB79EB70A968DBF80914603909181
:104F1000470397FD0196959587959F938F93809171
:104F20004603909147032091FA013091FB01821BC7
:104F3000930B9F938F9387E596E09F938F931F9397
:104F40000F9303C18D3009F0CBC484E180931E021E
:104F50008091120199279F938F9380914A0390919A
:104F60004B0397FD0F9674E0959587957A95E1F739
:104F70009F938F9320914A0330914B0337FF02C0D8
:104F8000295F3F4F63E0359527956A95E1F780915A
:104F9000FE019091FF01821B930B9F938F9386E6F6
:104FA00096E09F938F931F930F93E0910204F091EB
:104FB0000304099588E280931E022DB73EB7265F51
:104FC0003F4F2DBF8091110199279F938F9380911F
:104FD00048039091490397FD0F9654E09595879566
:104FE0005A95E1F79F938F9320914803309149039D
:104FF00037FF02C0295F3F4F43E0359527954A951B
:10500000E1F78091FC019091FD01821B930B9F932E
:105010008F938AE796E09F938F931F930F93E0916E
:105020000204F091030409958CE380931E028DB76E
:105030009EB70A968DBF8091100199279F938F93F9
:10504000809146039091470397FD0196959587952A
:105050009F938F9380914603909147032091FA018B
:105060003091FB01821B930B9F938F938EE896E008
:105070009F938F931F930F93E0910204F091030489
:105080000995EDB7FEB73A9668C010921E0282EA03
:1050900096E09F938F93DF92CF92FE01099584E172
:1050A00080931E020F900F900F900F9080914003FD
:1050B000909141039F938F938091F6019091F70116
:1050C0009F938F938FEA96E09F938F93DF92CF9277
:1050D000E0910204F0910304099588E280931E0296
:1050E0002DB73EB7285F3F4F2DBF80913E03909173
:1050F0003F039F938F938091F8019091F9019F93C3
:105100008F938EEB96E09F938F93DF92CF92E091F7
:105110000204F091030409958CE380931E028DB77D
:105120009EB708968DBF80913A0390913B039F9361
:105130008F938091F4019091F5019F938F938DEC63
:1051400096E09F938F93DF92CF92E0910204F091CB
:1051500003040995EDB7FEB73896EDBFC1C31092B1
:105160001E0280911D0190911E016AE070E00E9474
:10517000858D9F938F9380911D0190911E016AE010
:1051800070E00E94858D7F936F938CED96E09F93E6
:105190008F93DF92CF92FE01099584E180931E02E6
:1051A0002DB73EB7285F3F4F2DBF8091D408909117
:1051B000D5086AE070E00E94718D9F938F93809173
:1051C000D4089091D5086AE070E00E94718D7F93B9
:1051D0006F9380EF96E09F938F93DF92CF92E09151
:1051E0000204F0910304099588E280931E028DB7B2
:1051F0009EB708968DBF8091D6089091D7089F934F
:105200008F9384E097E09F938F93DF92CF92E0910A
:105210000204F091030409958CE380931E02EDB71C
:10522000FEB73696EDBF8091D8089091D9089F932C
:105230008F9384E197E09F938F93DF92CF92E091D9
:105240000204F091030409952DB73EB72A5F3F4F42
:105250004FC110921E0286E297E09F938F93DF92D8
:10526000CF92FE01099584E180931E020F900F906A
:105270000F900F9080917B0790917C079F938F9365
:105280008FE297E09F938F93DF92CF92E091020499
:10529000F0910304099588E280931E028DB79EB7B2
:1052A00006968DBF8091DB0299279F938F938FE3A2
:1052B00097E09F938F93DF92CF92E0910204F09159
:1052C000030409958CE380931E02EDB7FEB7369672
:1052D000EDBF80917A07992701979F938F938FE471
:1052E00097E0A9CF10921E028FE597E09F938F93CE
:1052F000DF92CF92FE01099584E180931E020F9008
:105300000F900F900F9080918E0190918F019F933D
:105310008F9387E697E09F938F93DF92CF92E091F0
:105320000204F0910304099588E280931E028DB770
:105330009EB706968DBF8091F1079091F2079F93DB
:105340008F9385E797E09F938F93DF92CF92E091C1
:105350000204F091030409958CE380931E02EDB7DB
:10536000FEB73696EDBF8091F3029091F4029F93C1
:105370008F9383E897E05FCFCCEDCC2EC2E0DC2E9C
:1053800020E030E0E901B3E0FB2EC0931E02F601FD
:1053900081916F0199279F938F9389010F5F1F4F11
:1053A0001F930F9381E997E09F938F9382E093E29D
:1053B0009F938F93E0910204F091030409952DB718
:1053C0003EB7285F3F4F2DBFFA9464969801F7FED1
:1053D000DCCF86C2A0EECA2EA2E0DA2EC0E0D0E07A
:1053E0008E01F3E0FF2E00931E02F60181916F0102
:1053F00099279F938F932596DF93CF938EE997E01C
:105400009F938F9382E093E29F938F93E0910204A6
:10541000F091030409952DB73EB7285F3F4F2DBF8C
:10542000FA940C5E1F4F2497F7FEDDCF59C21092FD
:105430001E028BEA97E09F938F9302E013E2DF92C4
:10544000CF92FE01099584E180931E020F900F9088
:105450000F900F9080916D0199279F938F9383EB0D
:1054600097E09F938F93DF92CF92E0910204F091A7
:105470000304099588E280931E028DB79EB70696B5
:105480008DBF8091D6019091D70197FD0396959598
:105490008795959587959F938F9381EC97E09F9340
:1054A0008F931F930F93E0910204F09103040995E9
:1054B0008CE380931E02EDB7FEB73696EDBF809168
:1054C000780699279F938F938091770699279F93CA
:1054D0008F938FEC97E09F938F931F930F93E0919F
:1054E0000204F091030409952DB73EB7285F3F4FA2
:1054F0002DBFF6C110921E028DED97E09F938F9302
:1055000072E0A72E73E2B72EDF92CF92FE010995CB
:105510000F900F900F900F90CAE1D7E000E010E0DD
:1055200062E0F62E802F8C5E80931E028B8D992771
:105530008F7790709F938F938B8999278F77907037
:105540009F938F938B8599278F7790709F938F93DD
:105550008B8199278F7790709F938F938DEE97E033
:105560009F938F93BF92AF92E0910204F091030456
:1055700009958DB79EB70C968DBFFA940C5E1F4FA0
:10558000A096F7FECFCFACC110921E028EEF97E02F
:105590009F938F9352E0A52E53E2B52EDF92CF92C8
:1055A000FE0109950F900F900F900F90CAE1D7E080
:1055B00000E010E042E0F42E802F8C5E80931E020B
:1055C0008F8D992787FD90959F938F938F8999272A
:1055D00087FD90959F938F938F85992787FD909551
:1055E0009F938F938F81992787FD90959F938F939A
:1055F0008DE098E09F938F93BF92AF92E091020469
:10560000F09103040995EDB7FEB73C96EDBFFA940F
:105610000C5E1F4FA096F7FECFCF62C110921E0204
:105620008EE198E09F938F9302E013E2DF92CF9296
:10563000FE01099584E180931E020F900F900F9058
:105640000F9080913507881F8827881F97E0899FD2
:10565000C00111248D969F938F9380912D07881FF1
:105660008827881F96E0899FC00111248D969F93FB
:105670008F9380912507881F8827881F95E0899F31
:10568000C00111248D969F938F9380911D07881FD1
:105690008827881F9927880F991F880F991F8D9633
:1056A0009F938F938DE298E09F938F93DF92CF9299
:1056B000E0910204F0910304099588E280931E02B0
:1056C0002DB73EB7245F3F4F2DBF80915507881FF0
:1056D0008827881F9BE0899FC00111248D969F9386
:1056E0008F9380914D07881F8827881F9AE0899F94
:1056F000C00111248D969F938F9380914507881F39
:105700008827881F99E0899FC00111248D969F9357
:105710008F9380913D07881F8827881F992723E052
:10572000880F991F2A95E1F78D969F938F9381E4B7
:1057300098E09F938F93DF92CF92E0910204F091D3
:10574000030409958CE380931E028DB79EB70C96D7
:105750008DBF80915D07881F8827881F9CE0899FE7
:10576000C00111248D969F938F9385E598E09F93B8
:105770008F93DF92CF92E0910204F0910304099598
:1057800080916507EDB7FEB73696EDBF87FF12C073
:1057900080E480931E0286E698E09F938F93DF92C9
:1057A000CF92E0910204F091030409950F900F90BD
:1057B0000F900F9080916D0787FF12C084E4809353
:1057C0001E0289E698E09F938F931F930F93E091B9
:1057D0000204F091030409950F900F900F900F9021
:1057E0008091750787FF7CC088E480931E028CE659
:1057F00098E09F938F931F930F93E0910204F09191
:10580000030409950F900F900F900F9069C01092AC
:105810001E028FE698E09F938F93DF92CF92FE0156
:10582000099584E180931E020F900F900F900F90C6
:105830008091AC019091AD019F938F938DE798E09B
:105840009F938F93DF92CF92E0910204F091030433
:10585000099588E280931E022DB73EB72A5F3F4F1D
:105860002DBF8091AE019091AF019F938F938AE8F5
:1058700098E09F938F93DF92CF92E0910204F09192
:105880000304099589E480931E028DB79EB706969E
:105890008DBF87E998E09F938F93DF92CF92E0913D
:1058A0000204F0910304099580911C020F900F905F
:1058B0000F900F9083FF14C01092AF011092AE01B1
:1058C00060E070E08EE090E00E94842E09C080913C
:1058D0001F01281719F4215020931F0110921D0257
:1058E00010921C02DF91CF911F910F91FF90DF90DA
:1058F000CF90BF90AF900895F999FECF92BD81BD32
:10590000F89A80B599270895F999FECF1FBA92BDEC
:1059100081BD60BD0FB6F894FA9AF99A0FBE08954A
:105920004AEA20E030E02617370740F4FC01819175
:10593000480F2F5F3F4F26173707C8F3842F99274B
:105940000895EAEA40E050E04617570778F49C01D2
:10595000F999FECF32BD21BDF89A80B5E80F4F5FAF
:105960005F4F2F5F3F4F4617570790F38E2F9927B2
:10597000089581E080934B0682E080934A0683E09D
:105980008093490684E080934C0685E080934D0621
:1059900086E080934E0687E080934F0688E08093F0
:1059A000500689E0809351068AE0809352068BE08E
:1059B000809353068CE08093540608958BE5809382
:1059C000480680910101843150F08AE08093680696
:1059D00010928C068BE1809364068EE40AC083E00B
:1059E0008093680680E280938C068EE18093640643
:1059F00085E58093890680938A0680E280938B06F2
:105A00001092B3068AE68093550682E28093B5062B
:105A10001092B60664E060936F061092AB06109287
:105A2000A80648E04093620656EE5093630680E471
:105A3000809365069EE1909356068FEF80935806FB
:105A40002FE0209359069093570610925B064093DF
:105A50005C0684E180935D0610925E0620935A06F0
:105A600010927106109272061092730610927406CC
:105A700010928E0610928F06109290061092910648
:105A800090E89093750632E33093760682E0809337
:105A9000B406209377065093780660937D068DE7D1
:105AA0008093800680938106809382069093790686
:105AB00025E520937A0686E480937B068CED80931F
:105AC0007C068CE380937E0610927F068FE58093A0
:105AD000920683EF809394068AEA809396068093D9
:105AE000970688E280939306809395063093830609
:105AF0009AE590938406309385068EEF80939806FE
:105B000084E68093990690939A0690939B069093CF
:105B10009C068BE480939D0620939E0680939F06AF
:105B20001092A00686E08093A1064093A20690936F
:105B3000A3068AE28093A40685EF8093A5068CE8ED
:105B40008093A60685E08093A7061092A90610927E
:105B5000AA0681E280936C0681E480936D0690939F
:105B60006E061092AC061092AD061092AE0686E953
:105B70008093AF069093860687E380938706109202
:105B8000B0061092B1061092B2060895CF93DF933B
:105B90000E94DE2C8AE080935F0680E1809360069D
:105BA00026E0209361069AE59093660688E7809345
:105BB00067069093690680936A0620936B0680E2DD
:105BC000809370068CE3809388068BE480938D0627
:105BD000A7EBB6E08CE0E0E2F1E0ED010190099284
:105BE0008A95E1F76BE770E0CD018F5690400E94F7
:105BF000902C8093C306DF91CF910895CF93DF93CC
:105C00000E94DE2C88E080935F0630E130936006CE
:105C100026E02093610694E69093660688E78093D9
:105C200067069093690680936A0620936B0630930B
:105C3000700686E48093880680938D06A7EBB6E015
:105C40008CE0E6E2F1E0ED01019009928A95E1F73E
:105C50006BE770E0CD018F5690400E94902C8093AE
:105C6000C306DF91CF910895CF93DF930E94DE2C7E
:105C700026E020935F068AE08093600684E08093AC
:105C8000610694E69093660688E780936706909392
:105C9000690680936A0620936B0680E18093700604
:105CA00086E48093880680938D06A7EBB6E08CE0AF
:105CB000EEE2F1E0ED01019009928A95E1F76BE7E0
:105CC00070E0CD018F5690400E94902C8093C306C7
:105CD000DF91CF910895F999FECF92BD81BDF89AD9
:105CE00080B599270895F999FECF1FBA92BD81BD5D
:105CF00060BD0FB6F894FA9AF99A0FBE08956CE752
:105D00007CE20E94D48B089544E85CE20E940E8CF1
:105D10000895EF92FF920F931F93CF93C82F815056
:105D2000853008F0C3E08CE7C89F8001112488EE1D
:105D3000E82E8FEFF82EE00EF11E6BE770E0C70142
:105D40000E94A12C682F98012D593F4F8FB399279E
:105D5000AC014270507081FDF9CF32BD21BDF89A7F
:105D600080B5861711F0CA0123C08FB399279C0113
:105D70002270307081FDF9CFF2BCE1BCF89A80B599
:105D80008B3511F0C90114C08CE7C89FC0011124E4
:105D900048972CE73CE24CE750E0BC0188E496E0F1
:105DA0000E94AF8B0E94D76C0E94958781E090E0A3
:105DB000CF911F910F91FF90EF900895282F86307B
:105DC00010F025E003C0882309F421E0F999FECF03
:105DD0001FBA82E090E092BD81BD20BD0FB6F8945D
:105DE000FA9AF99A0FBE0895CF93C82F809148066A
:105DF0008B3509F051C0C63010F0C5E003C0CC238C
:105E000009F44AC00E94A18A8091B60682FF07C0A9
:105E100080916D06843618F080E580936D066BE7FF
:105E200070E088E496E00E94902C8093C3068CE793
:105E3000C89FC001112424E83CE24CE750E068E42C
:105E400076E048970E94EC8B24E83CE24CE050E07E
:105E500069E476E080E590E00E94EC8B6CE070E015
:105E600089E496E00E94902C282FF999FECF1FBA62
:105E70008CE590E092BD81BD20BD0FB6F894FA9AF2
:105E8000F99A0FBE8C2F0E94DE2E0E94D76C0E94C2
:105E9000958781E090E002C080E090E0CF91089586
:105EA0006DE470E088EE93E00E94A12C482F8FB340
:105EB00099279C012270307081FDF9CF85E394E031
:105EC00092BD81BDF89A80B5841779F48FB3992774
:105ED0009C012270307081FDF9CF88EE93E092BD75
:105EE00081BDF89A80B5813011F0C90108952CE781
:105EF0003CE24EE450E068EE73E084EC96E00E94F1
:105F0000AF8B81E090E008958091C4068130A9F4C0
:105F10006DE470E084EC96E00E94902C8093110771
:105F200024E83CE24EE450E064EC76E088EE93E056
:105F30000E94EC8B81E090E0089580E090E008956D
:105F4000CF93DF9381E08093C406E4ECF6E08FE02A
:105F5000158616861786108A8150349687FFF8CFEB
:105F600080E48093D1068093D2061092D30680936A
:105F7000D4068093D50690EC9093D6061092D7065F
:105F80008093D8068093D9061092DA069093DB06A8
:105F90009093DC068093DD061092DE068093DF0688
:105FA0009093E006A5ECB6E087E0E4E3F1E0ED01D4
:105FB000019009928A95E1F76DE470E0CD010197B7
:105FC0000E94902C80931107DF91CF910895F99949
:105FD000FECF82E090E092BD81BDF89A80B5282F77
:105FE000863078F023E0322FF999FECF1FBA82E095
:105FF00090E092BD81BD30BD0FB6F894FA9AF99A3F
:106000000FBE822F992708951F93CF93C82F162F65
:10601000863010F0C5E003C0882309F4C1E08C2F5E
:1060200099278230910541F08330910544F401971E
:1060300031F40E94C62D05C00E94FE2D02C00E94B0
:10604000342E1123E1F06CE070E080E590E00E94D6
:10605000A12C282FF999FECF8CE590E092BD81BD4F
:10606000F89A80B5821759F42CE73CE24CE050E0F6
:1060700060E570E089E496E00E94AF8B02C00E9468
:10608000B92C8C2F0E94F42ECF911F910895DF928E
:10609000EF92FF920F931F93CF93FF24DF2CEF2CEF
:1060A00081E090E00E946B2E8B3511F031E0E32E01
:1060B0006CE070E080E590E00E94A12CC82FF99977
:1060C000FECF8CE590E092BD81BDF89A80B58C172B
:1060D00011F421E0D22EC1E001E010E0EE2029F41D
:1060E0008C2F0E94892E8823C9F591E0F92E1F93E9
:1060F0000F938FE998E09F938F938CE295E19F93A4
:106100008F93E0910204F091030409952DB73EB7F7
:106110002A5F3F4F2DBF0230110549F003301105B2
:106120004CF40130110531F40E94C62D05C00E94C7
:10613000FE2D02C00E94342EDD2059F02CE73CE2F7
:106140004CE050E060E570E089E496E00E94AF8B9F
:1061500002C00E94B92C8C2F0E94F42ECF5F0F5FDB
:106160001F4FC63008F4BACFFF2019F083E00E9419
:10617000DE2E0E94E72FC82F0E94892E8C2F992790
:106180009F938F9385EC98E09F938F930CE215E19A
:106190001F930F93E0910204F0910304099581E0AD
:1061A00090E00E946B2E2DB73EB72A5F3F4F2DBF68
:1061B0008F3F21F00E94502F882399F48EED98E0B4
:1061C0009F938F931F930F93E0910204F091030428
:1061D00009950E94A02F0E94842F0F900F900F907E
:1061E0000F90EE2029F06BE581E090E00E94732E85
:1061F0001092470690E0E1EDF6E0CFE08081349622
:1062000018160CF49F5FC150C7FFF8CF9093470654
:10621000892F99279F938F9385EC96E09F938F9377
:106220008FEF98E09F938F931F930F93E091020459
:10623000F091030409950E9439098DB79EB708961D
:106240008DBFCF911F910F91FF90EF90DF90089538
:10625000982F2FB7F8943998389A88B1836088B905
:106260008091B9008C7F8093B9008AE28093B80056
:10627000109229021092270210922602992379F097
:10628000EAE1F7E08BE0108211821282138214821D
:106290001582168217828150389687FFF4CF789442
:1062A0002FBF08951092290284E98093BC0080E8F2
:1062B0008093BC001092BD001092BA001092BB00F7
:1062C0001092B9001092B8001092250280E00E944E
:1062D00028311092BB0085E88093BC008091230296
:1062E00082608093230208951F920F920FB60F923F
:1062F00011242F933F934F935F938F939F93EF932B
:10630000FF9380912902282F3327442755278F5F39
:1063100080932902F9012731310508F0C2C2E759FB
:10632000FF4F0C940C8E81E08093250209C0809170
:1063300027028C3090F4809127028F5F8093270290
:1063400080912702E82FFF27EE0FFF1FEE0FFF1FA0
:10635000EC53F94F8585181654F7809127028C303D
:1063600070F010922202109221021092270285E012
:106370008093290280912602880F8D5A04C0809153
:106380002702880F8E5A8093BB0085E87FC28091D8
:106390002702E82FFF2783E0EE0FFF1F8A95E1F722
:1063A000E65EF84F81818093BB0085E88093BC0056
:1063B00080912702E82FFF27EE0FFF1FEE0FFF1F30
:1063C000EE0FFF1FE65EF84F808180FF91C0809145
:1063D0002702E82FFF27EE0FFF1FEE0FFF1FEE0F24
:1063E000FF1FE65EF84F8281882329F080914706DF
:1063F000873008F46CC28091210290912202892B8F
:1064000009F065C280911F0290912002892B09F04A
:106410005EC26EC08091270221E030E002C0220FF0
:10642000331F8A95E2F780911F0290912002282362
:106430003923232B79F080912702E82FFF27EE0FD5
:10644000FF1FEE0FFF1FEE0FFF1FE65EF84F80E10C
:1064500084830DC080912702E82FFF27EE0FFF1FD6
:10646000EE0FFF1FEE0FFF1FE65EF84F14828091C4
:106470002702E82FFF2753E0EE0FFF1F5A95E1F7A1
:10648000E65EF84F8481282F332743E0220F331F25
:106490004A95E1F780912702E82FFF2793E0EE0F5E
:1064A000FF1F9A95E1F7E65EF84F82818770822B95
:1064B0008093BB0085E88093BC002091270281E097
:1064C00090E002C0880F991F2A95E2F720912102DF
:1064D0003091220282239323892B51F082E197E0AD
:1064E00090932D0280932C0288E080932E02EFC1BE
:1064F00084E089C1E0912C02F0912D02819180937A
:10650000BB0085E88093BC00F0932D02E0932C0241
:1065100080912E02815080932E02882309F4D7C1E6
:1065200083E071C18091B900803351F580912A02D6
:10653000882329F4809127028F5F80932A0280911B
:106540002702E82FFF2783E0EE0FFF1F8A95E1F770
:10655000E65EF84F838199278F7790708F3791058A
:106560007CF480912702E82FFF27EE0FFF1FEE0F2C
:10657000FF1FEE0FFF1FE65EF84F83818F5F83835F
:106580001092290284E98093BC008AE090E0909305
:106590003D0180933C01809127028F5F8093270209
:1065A000109229026DC18091B9008034C9F18091A7
:1065B0002602E82FFF27EE0FFF1FEE0FFF1FEE0F43
:1065C000FF1FE65EF84F83818F77838380912602D9
:1065D0008F5F80932602809126028C30A0F010926B
:1065E00026021092200210921F0280912B028F5FD0
:1065F00080932B028C3038F010922B028091230272
:106600008D7F8093230280912302816080932302F7
:106610001092290284E98093BC001092250273C075
:1066200080912602E82FFF27EE0FFF1FEE0FFF1FBE
:10663000EE0FFF1FE65EF84F8381806883838091B1
:106640002602E82FFF27EE0FFF1FEE0FFF1FEE0FB2
:10665000FF1FE65EF84F808180FF2FC080912602E9
:10666000E82FFF2753E0EE0FFF1F5A95E1F7E65E94
:10667000F84F84819927009751F04097D9F582E12E
:1066800097E090932D0280932C0288E031C0809196
:106690002602992743E0880F991F4A95E1F7815E0A
:1066A000984F90932D0280932C0290912602809116
:1066B0002B029817E1F483E01BC0809126029927F2
:1066C00033E0880F991F3A95E1F7815E984F9093D8
:1066D0002D0280932C028091230281FD06C09091AF
:1066E000260280912B02981711F482E001C081E00C
:1066F00080932E0280912E02813011F485E801C032
:1067000085EC8093BC0080912A0280932402109231
:106710002A02DDC0E0912C02F0912D028091BB0095
:10672000808380912C0290912D02019690932D02EE
:1067300080932C0280912E02815080932E02823011
:1067400010F085EC5DC0813011F485E859C080916E
:10675000230281FF2DC08091A30280FD1DC0809186
:106760002602E82FFF2723E0EE0FFF1F2A95E1F70F
:10677000E65EF84F86818A3F79F480912602E82F01
:10678000FF2793E0EE0FFF1F9A95E1F7E65EF84FC3
:106790008081816080830CC080912602E82FFF27D2
:1067A00083E0EE0FFF1F8A95E1F7E65EF84F108257
:1067B000809126028F5F80932602809126028C3082
:1067C000A0F0109226021092200210921F028091D7
:1067D0002B028F5F80932B028C3038F010922B02AB
:1067E000809123028D7F809323021092290284E9F5
:1067F0008093BC008091230281608093230265C056
:106800008093BC0086E08093290261C088E9BBCDFB
:1068100080912802880F805FB6CD80912802992749
:106820008130910561F0823091051CF4892B21F0B3
:106830004EC0029739F04BC080911201A4CD8091D7
:106840001101A1CD809110019ECD80E89CCD1092C8
:10685000290284E98093BC00109225028AE090E02E
:1068600090933D0180933C0180912802823088F40E
:10687000809128028F5F8093280282E18093290211
:10688000809123028E7F8093230285EA8093BC004F
:106890001EC01092280280912302816080932302FF
:1068A00016C01092290284E98093BC0080912302D3
:1068B0008160809323028AE090E090933D01809371
:1068C0003C01109227021092260210922502FF919D
:1068D000EF919F918F915F914F913F912F910F90E9
:1068E0000FBE0F901F9018951F93CF93DF93182F13
:1068F0008091DA02882321F48091BB01882319F06A
:1069000081E090E097C01D3008F092C01123B1F0F3
:10691000E12FFF2723E0EE0FFF1F2A95E1F7E65E48
:10692000F84F35978081359688230CF081C03897D1
:10693000808180FD03C083E090E07CC080911207DD
:10694000823019F084E090E075C067E070E082E189
:1069500097E00E94902C90911907891719F085E013
:1069600090E068C080ED97E00E943B19EC018091B7
:10697000230280FD05C0CE010E9444198823B9F38B
:10698000112319F48FEF90E00BC0212F33272150F2
:10699000304081E090E002C0880F991F2A95E2F70D
:1069A0009093220280932102A1E0B0E0EAE1F7E0B7
:1069B00040E050E06BE0CD01042E02C0880F991F2B
:1069C0000A94E2F72091210230912202822393233C
:1069D000892B11F01182128261504F5F5F4F389600
:1069E00067FFE9CF109227021092290280912302BB
:1069F0008E7F8093230285EA8093BC0080912302DE
:106A000080FD05C0CE010E9444198823B9F380910E
:106A1000210290912202892B29F0CE010E94441973
:106A2000882311F38091210290912202009711F0A6
:106A300082E090E0DF91CF911F9108950F931F9313
:106A4000CF93DF93982F8091DA02882321F48091ED
:106A5000BB01882319F081E090E092C09D30A0F442
:106A6000992319F486E090E08BC0C92FDD27FE0141
:106A700033E0EE0FFF1F3A95E1F7E65EF84F3597EA
:106A80008081359687FD03C082E090E079C0389719
:106A9000808180FD03C083E090E072C080ED97E0CC
:106AA0000E943B198C018091230280FD05C0C80122
:106AB0000E9444198823B9F3219721E030E0C901ED
:106AC00002C0880F991FCA95E2F790932002809325
:106AD0001F02D901EAE1F7E040E050E06BE0CD01B0
:106AE000042E02C0880F991F0A94E2F720911F021A
:106AF0003091200282239323892B11F0118212827C
:106B000061504F5F5F4F389667FFE9CF10922602C2
:106B100010921207109219071092290280912302F5
:106B20008E7F8093230285EA8093BC0080912302AC
:106B300080FD05C0C8010E9444198823B9F38091E3
:106B40001F0290912002892B29F0C8010E9444194C
:106B5000882311F380911207823019F084E090E0CD
:106B60000FC067E070E082E197E00E94902C909166
:106B70001907891719F085E090E002C080E090E0E5
:106B8000DF91CF911F910F910895CF93DF9380E014
:106B900022E83FEFCFEAD7E0EBE7F7E0DF0185300F
:106BA00020F411961C921E9202C031832083198218
:106BB000188222968F5F129632968A3180F3109255
:106BC0004703109246031092490310924803109213
:106BD0004B0310924A03DF91CF9108951F920F92B9
:106BE0000FB60F9211240F931F932F933F934F9340
:106BF0005F936F937F938F939F93AF93BF93CF9345
:106C0000DF93EF93FF938091B50682FDE1C0409141
:106C10008600509187008091300290913102481B8C
:106C2000590B809186009091870090933102809358
:106C30003002CA018D549440A0913202B0913302C7
:106C4000835F9A4178F48091320280937A07149797
:106C500014F01092400181E090E090933302809311
:106C600032022BC2AD30B1050CF027C2CA018B5FD6
:106C70009040845B914008F086C080913E019091E5
:106C80003F01481B590BE091B006EE2351F0FF275E
:106C9000EE0FFF1FE558F84F8081918184369105F2
:106CA000ECF4FD01EA0FFB1FE558F84F808191815C
:106CB000FA01E81BF90BCF01F7FF03C0909581950E
:106CC0009F4F06975CF48091DB02883C20F4809112
:106CD000DB02865F01C088EC8093DB02FD01EA0FD6
:106CE000FB1FE558F84F808191819C01220F331FD3
:106CF000280F391F240F351F37FF02C02D5F3F4F6C
:106D0000E901D595C795D595C795CA0101968C1708
:106D10009D0714F4219706C041505040C417D50771
:106D20000CF421968091DB02833CE0F08D010A0F88
:106D30001B1FF801E558F84F808191819E01281BA7
:106D4000390BC90163E070E00E94858DCB01880F8B
:106D5000991F860F971F0155184FD80111969C93C4
:106D60008E9307C0AA0FBB1FA155B84F11961C9256
:106D70001E92E0913202F0913302EE0FFF1FE558B0
:106D8000F84FD183C08320913202309133022F5FBC
:106D90003F4F3093330220933202809101018431BE
:106DA00008F08BC12530310511F45D9A01C05D9862
:106DB00080913202909133028630910511F45C9AF1
:106DC00001C05C98079711F45B9A77C15B9875C115
:106DD0004091860050918700809134029091350255
:106DE000481B590B80918600909187009093350243
:106DF00080933402CA018D54944060919E02835F57
:106E00009A4108F07AC060932F0280912F0284305B
:106E100008F453C090917A0780912F02981709F0D7
:106E20004CC050919F025B3008F43FC0109240016B
:106E300010929E0240E05F31C0F0E42FFF27EE0F7A
:106E4000FF1F9F0126593D4FDF01A558B84F8D9177
:106E50009C91D9018D939C93DF01A155B84F8D91E1
:106E60009C91EC57FD4F91838083E42FFF27EE0F19
:106E7000FF1F9F012558384FDF01AA5CBD4F8D9140
:106E80009C91D90111969C938E93DF01A05BBD4F1D
:106E90008D919C91E155F84F91838083842F8F5F72
:106EA000482F8D3040F280939E0280919F028F3F49
:106EB000B9F08F5F80939F0213C080919F02853647
:106EC00020F08AE080939F0202C010929F0280917E
:106ED00001018A3011F0843110F0289A01C02898FD
:106EE00081E080939E028091DA02882309F0E5C058
:106EF00080912F0280937A07E0C06D3008F0B5C012
:106F0000CA018B5F9040845B914008F090C08091F3
:106F10003E0190913F01481B590BE62FFF27EE0FD2
:106F2000FF1FEA5CFD4F80819181FA01E81BF90B9C
:106F3000CF0105960B9720F5E091B006EE2351F0B6
:106F4000FF27EE0FFF1FE558F84F808191818436AF
:106F50009105B4F480919F028A3120F08091DB0288
:106F6000865F05C08B3028F08091DB028E5F8093B6
:106F7000DB028091DB02893C18F088EC8093DB0215
:106F8000E62FFF27EE0FFF1FEA5CFD4F8081918106
:106F90009C01220F331F280F391F240F351F37FF85
:106FA00002C02D5F3F4FE901D595C795D595C7958F
:106FB000CA0101968C179D0714F4219706C0415011
:106FC0005040C417D5070CF421968091DB028E3B0C
:106FD000D8F0E62FFF27EE0FFF1FDF01AA5CBD4FA1
:106FE0008D919C919E01281B390BC90163E070E0D3
:106FF0000E94858DCB01880F991F860F971FE05B3C
:10700000FD4F9183808308C0E62FFF27EE0FFF1FFF
:10701000E05BFD4F1182108280919E02E82FFF27D6
:10702000EE0FFF1FEA5CFD4FD183C08309C0809142
:1070300001018A3011F0843110F0289A01C028989B
:1070400080910101843188F480919E02853011F491
:107050005D9A05C05D98863011F45C9A05C05C9815
:10706000873011F45B9A01C05B9880919E02843155
:1070700020F48F5F80939E0220C08431F1F48091D0
:1070800001018A3011F0843110F0289A01C028984B
:107090008EE180939E022CE0CFEAD7E0AAE6B2E030
:1070A000EBE7F7E08D919D91918380833296198271
:1070B00018822296215027FFF5CFFF91EF91DF91A3
:1070C000CF91BF91AF919F918F917F916F915F9180
:1070D0004F913F912F911F910F910F900FBE0F90E5
:1070E0001F901895EF92FF920F931F938091640663
:1070F0009927880F991F880F991F7C010027F7FC9B
:107100000095102F8091350390913603A09137039D
:10711000B0913803BC01CD01A80197010E94BA8D3E
:107120003093A8052093A70580912D0390912E03FD
:10713000A0912F03B0913003BC01CD01A8019701AC
:107140000E94BA8D3093AA052093A9058091380832
:107150009091390897FD0396959587959595879514
:107160009093AC058093AB058091480890914908B5
:1071700097FD039695958795959587959093AE0580
:107180008093AD0580914603909147032091FA01C9
:107190003091FB01821B930B9093B0058093AF0558
:1071A0008091D5029091D602A091D702B091D802D9
:1071B000BC01CD0125E030E040E050E00E94BA8DF6
:1071C0003093B2052093B1058091F4019091F501BF
:1071D0009093B4058093B30580918E0190918F01B7
:1071E0009093B8058093B70580911D0190911E0181
:1071F0009093BA058093B9058091DB02992790930B
:10720000BC058093BB058091F1079091F2079093A4
:10721000BE058093BD0580911B0799279093C005FB
:107220008093BF058091230799279093C20580938F
:10723000C10580912B0799279093C4058093C305BE
:107240008091330799279093C6058093C505809157
:10725000D6019091D7019093D0058093CF0580916E
:10726000D4089091D5089093D4058093D30580914C
:10727000D8089091D9089093D6058093D505809130
:10728000D1029091D202A091D302B091D402BC015C
:10729000CD0125E030E040E050E00E94BA8D30930F
:1072A000D8052093D7058091F3029091F402909332
:1072B000DE058093DD058091DA0899279093E20539
:1072C0008093E1058091A7039091A8039093E40532
:1072D0008093E3058091A5039091A6039093E60522
:1072E0008093E50580911B04882321F480911C0480
:1072F000882321F08091A605816003C08091A605B6
:107300008E7F8093A6051F910F91FF90EF900895B7
:107310001F93CF93DF93182FEB018091DA0288231C
:1073200009F5809101018C3010F4299801C0299A47
:1073300011501F3F81F0D093DD01C093DC0180919B
:10734000DC019091DD01892BD1F7CE018C0F9D1FBF
:107350000E945019EDCF809101018C3010F4299AD0
:1073600001C02998DF91CF911F910895CF93DF93AA
:10737000809101018D3011F40E94E71D10927A0076
:107380008091FE019091FF019093FD078093FC078F
:107390008091FC019091FD019093ED078093EC07A3
:1073A0008091FA019091FB0190933E0880933D08F3
:1073B0002091F6013091F701C901880F991F880FBC
:1073C000991F820F931F820F931F90933908809308
:1073D00038082091F8013091F901C901880F991FEF
:1073E000880F991F820F931F820F931F9093490854
:1073F000809348088FEC80937A00ACEDB2E0CDE446
:10740000D6E097E08991E82FFF27EE0FFF1FE558A0
:10741000F84F0190F081E02DE158FF4F1E161F0636
:107420001CF0E0E0F0E005C0EF3FF10514F0EFEFF5
:10743000F0E08C91282F3327E217F30714F48150E2
:1074400004C02E173F0714F48F5F8C939150119650
:1074500097FFD8CF809189069927AA27BB27BC011F
:10746000CD0124EC39E040E050E00E94468DDC0183
:10747000CB018093860190938701A0938801B093FC
:10748000890180918A069927AA27BB27BC01CD01D3
:107490000E94468DDC01CB01809382019093830191
:1074A000A0938401B0938501DF91CF910895A0E06E
:1074B000B0E0EDE5FAE30C94DB8D882EC0E0D0E07F
:1074C0007E016E0110921B04D0934103C0934003D0
:1074D000D0933F03C0933E03D0933B03C0933A0342
:1074E000D0934B03C0934A03D0934903C0934803FE
:1074F000D0934703C093460310926A01109269012A
:107500001092EF010E94B63984E690E00E945D1966
:107510000E94B6398091550680FF10C080911301FA
:1075200090911401875B934038F4809113019091FE
:1075300014018E5E924010F40E94651D0FE18AE0F6
:1075400090E00E945D198091FA019091FB01C80FB3
:10755000D91F8091FE019091FF01E80EF91E8091E4
:10756000FC019091FD01C80ED91E015007FFE7CF25
:107570009701205F3F4F3695279536952795309395
:107580004B0320934A03C60140969695879596959E
:10759000879590934903809348036096F5E0D695CC
:1075A000C795FA95E1F7D0934703C09346039093AC
:1075B0004503809344033093430320934203882080
:1075C00009F441C0809138089091390897FF03C0B1
:1075D000909581959F4F6CE070E00E94858D9B0196
:1075E000709341036093400380914808909149084B
:1075F00097FF03C0909581959F4F6CE070E00E94CB
:10760000858D70933F0360933E038091EA059091CE
:10761000EB0590933B0380933A03B90184E090E03B
:107620000E94842E60913E0370913F0386E090E0BB
:107630000E94842E60913A0370913B0388E090E0B1
:107640000E94842E65C084E090E00E947F2E90937B
:1076500041038093400386E090E00E947F2E909348
:107660003F0380933E0388E090E00E947F2E9C01C0
:1076700090933B0380933A038091400390914103A0
:107680008150984050F480913E0390913F03815087
:10769000984018F421503440D8F180E299E09F934B
:1076A0008F938CE295E19F938F93E0910204F09188
:1076B00003040995809138089091390897FF03C019
:1076C000909581959F4F6CE070E00E94858D70933E
:1076D000410360934003809148089091490897FFC7
:1076E00003C0909581959F4F6CE070E00E94858D5E
:1076F00070933F0360933E038091EA059091EB0500
:1077000090933B0380933A030F900F900F900F904C
:107710001092FD071092FC071092ED071092EC07F3
:1077200010923E0810923D0884E690E00E945D1998
:107730008091F6019091F7019C01220F331F220FD7
:10774000331F280F391F280F391F30933908209312
:1077500038088091F8019091F9018C01000F111FF8
:10776000000F111F080F191F080F191F1093490848
:107770000093480880916406C82EDD24EE24FF247F
:10778000442737FD4095542FC701B6010E94468D0E
:107790004B015C016093350370933603809337038C
:1077A000909338039801442737FD4095542FC70123
:1077B000B6010E94468DDC01CB0180932D0390938E
:1077C0002E03A0932F03B093300380921503909261
:1077D0001603A0921703B092180380930D039093A1
:1077E0000E03A0930F03B0931003109205031092A1
:1077F00006031092070310920803809115019091DF
:107800001601A0911701B09118019093ED05809396
:10781000EC051092EE011092ED011092F50210921B
:10782000F6021092F7021092F80200918E01109168
:107830008F011093F4020093F30284E690E090939A
:107840008B0180938A0182E390E09093DD01809325
:10785000DC01809189069927AA27BB27BC01CD01AD
:1078600024EC39E040E050E00E94468DDC01CB0181
:107870008856954CAF4FBF4F8093860190938701F8
:10788000A0938801B093890180918A069927AA273D
:10789000BB27BC01CD010E94468DDC01CB0188567F
:1078A000954CAF4FBF4F8093820190938301A0937B
:1078B0008401B09385011092470110924601C801DE
:1078C000AA2797FDA095BA2F20914201309143013C
:1078D0004091440150914501BC01CD010E94468D6B
:1078E000DC01CB018093440890934508A09346089F
:1078F000B09347081092F0021092EF020E94D76CEA
:107900008091A30284608093A3028FEF8093C408C8
:107910001092C50880E28093C608CCEDD2E0ADE4B9
:10792000B6E007E08D91E82FFF27EE0FFF1FE55827
:10793000F84F8081918181588993015007FFF2CFE0
:1079400084E68093DB028091DA018111579A80915D
:107950004A0390914B0380569940815C9B4228F0EA
:1079600080911B04816080931B0480914803909157
:10797000490380569940815C9B4228F080911B040A
:10798000826080931B0480914603909147038C5240
:1079900091408957954028F080911B048460809322
:1079A0001B0480914003909141038C529140835C71
:1079B000914028F080911B04886080931B04809183
:1079C0003E0390913F038C529140835C914028F09C
:1079D00080911B04806180931B0480913A039091F5
:1079E0003B03805092408355914028F080911B04C6
:1079F000806280931B0486E480937D010E949587BA
:107A0000ECE0CDB7DEB70C94F78DA3E1B0E0EBE08E
:107A1000FDE30C94D58D809146039091470320910E
:107A2000FA013091FB01821B930B90933E088093E7
:107A30003D08809104029091050297FD07969C01F4
:107A400013E0359527951A95E1F73093FD072093BC
:107A5000FC07809102029091030297FD0796B3E024
:107A600095958795BA95E1F79093ED078093EC078C
:107A70003093080820930708909300088093FF072D
:107A80008091380890913908AC01440F551F480F78
:107A9000591F2091F6013091F701C901880F991FF4
:107AA000880F991F820F931F820F931F480F591F32
:107AB00057FF02C04D5F5F4F5595479555954795C8
:107AC00050933908409338088091480890914908AC
:107AD000AC01440F551F480F591F2091F8013091F8
:107AE000F901C901880F991F880F991F820F931FF1
:107AF000820F931F480F591F57FF02C04D5F5F4F02
:107B00005595479555954795509349084093480892
:107B10002091F6013091F701C901880F991F880F54
:107B2000991F820F931F820F931F9C01442737FDDB
:107B30004095542F8091250390912603A09127030F
:107B4000B0912803820F931FA41FB51F80932503B4
:107B500090932603A0932703B09328032091F80164
:107B60003091F901C901880F991F880F991F820F61
:107B7000931F820F931F9C01442737FD4095542F7C
:107B80008091210390912203A0912303B0912403BB
:107B9000820F931FA41FB51F80932103909322038C
:107BA000A0932303B09324038091110890911208AD
:107BB0002091F6013091F701820F931F90931208E4
:107BC0008093110880914008909141082091F8011C
:107BD0003091F901820F931F9093410880934008E0
:107BE00080913C0390913D03019690933D038093D7
:107BF0003C038091EA059091EB0520913A03309186
:107C00003B03821B930B9C01442737FD4095542F67
:107C100080911D0390911E03A0911F03B09120033A
:107C2000820F931FA41FB51F80931D0390931E0303
:107C3000A0931F03B09320038FEC80937A001092DF
:107C40000F0120910D0330910E0340910F035091CD
:107C5000100329873A874B875C8729543B4641406C
:107C600050402CF028E43BE641E050E00DC089850F
:107C70009A85AB85BC85885B9449AE4FBF4F4CF469
:107C800028EB34E94EEF5FEF2D833E834F83588717
:107C900008C089859A85AB85BC858D839E83AF831B
:107CA000B887209115033091160340911703509126
:107CB00018032D873E874F87588B29543B464140F8
:107CC00050402CF028E43BE641E050E00DC08D85AB
:107CD0009E85AF85B889885B9449AE4FBF4F4CF401
:107CE00028EB34E94EEF5FEF29833A834B835C83C3
:107CF00008C08D859E85AF85B88989839A83AB83BB
:107D0000BC83A0913D08B0913E08BB8BAA8BFD01BE
:107D1000CF01AA2797FDA095BA2FA0900503B09098
:107D20000603C0900703D0900803A80EB91ECA1E10
:107D3000DB1EA0920503B0920603C0920703D09207
:107D40000803E0904408F09045080091460810911F
:107D50004708E80EF91E0A1F1B1FE0924408F09224
:107D600045080093460810934708F091BE02F98B2E
:107D7000FF2309F098C18091BD02882309F093C1C7
:107D80008091340886FF8FC18091EC079091ED07B8
:107D9000AA2797FDA095BA2FBC01CD0129813A8170
:107DA0004B815C810E94468D9B01AC0197FF04C012
:107DB0002150384F4F4F5F4FBBE055954795379552
:107DC0002795BA95D1F780916901682E7724882488
:107DD0009924CA01B901A40193010E94468DDC01D6
:107DE000CB018093560390935703A0935803B0930D
:107DF0005903B7FF04C08150904FAF4FBF4F1C01D4
:107E00002D01ACE05594479437942794AA95D1F767
:107E100020925603309257034092580350925903D0
:107E20008091FC079091FD07AA2797FDA095BA2F96
:107E3000BC01CD012D813E814F8158850E94468D28
:107E400097FF04C06150784F8F4F9F4FFBE095958F
:107E5000879577956795FA95D1F7A40193010E94CC
:107E6000468DDC01CB0180935A0390935B03A09372
:107E70005C03B0935D03B7FF04C08150904FAF4FD8
:107E8000BF4F9C01AD01ECE055954795379527957F
:107E9000EA95D1F720935A0330935B0340935C0338
:107EA00050935D0380915603909157039093E4079C
:107EB0008093E30780915A0390915B039093E807C6
:107EC0008093E707221933094409550920935A037F
:107ED00030935B0340935C0350935D03E20EF31E0B
:107EE000041F151FE0924408F092450800934608CD
:107EF00010934708809168018823B1F457FF04C0AC
:107F00002F5F3F4F4F4F5F4F5595479537952795BB
:107F1000A21AB30AC40AD50AA0920503B0920603B6
:107F2000C0920703D09208032A893B897901002770
:107F3000F7FC0095102F80915A0390915B03A0915C
:107F40005C03B0915D03E80EF91E0A1F1B1FC801F8
:107F5000B70129813A814B815C810E94468D9B014A
:107F6000AC0197FF04C02150384F4F4F5F4F6BE07B
:107F700055954795379527956A95D1F780916A0170
:107F8000A82EBB24CC24DD24CA01B901A601950189
:107F90000E94468DDC01CB0180934E0390934F03EA
:107FA000A0935003B0935103B7FF04C08150904F8A
:107FB000AF4FBF4F3C014D013CE0959487947794BF
:107FC00067943A95D1F760924E0370924F03809276
:107FD000500390925103C801B7012D813E814F811A
:107FE00058850E94468D97FF04C06150784F8F4F8F
:107FF0009F4F2BE095958795779567952A95D1F7B3
:10800000A60195010E94468DDC01CB0180935203AD
:1080100090935303A0935403B0935503B7FF04C048
:108020008150904FAF4FBF4FAC01BD018CE07595B3
:108030006795579547958A95D1F74093520350938A
:10804000530360935403709355032A893B8937FF88
:1080500003C0309521953F4F21343105E4F1D4011F
:10806000C30197FE07C0B095A095909581959F4F4D
:10807000AF4FBF4F81389105A105B10584F4DB01F5
:10808000CA0177FF07C0B095A095909581959F4F45
:10809000AF4FBF4F81389105A105B105E4F081E0F4
:1080A0008093F10218C01092E8071092E70710922F
:1080B000E4071092E30710925203109253031092B8
:1080C00054031092550310924E0310924F031092D6
:1080D0005003109251038091520390915303A09149
:1080E0005403B0915503BC01CD0124E630E040E0DB
:1080F00050E00E94BA8DE0904E03F0904F03E21AD8
:10810000F30AF092FB07E092FA0780914E039091F8
:108110004F03A0915003B0915103BC01CD0124E65F
:1081200030E040E050E00E94BA8DDA01C9012091B0
:108130005203309153038C01021B130B1093EF0772
:108140000093EE078091420190914301A091440178
:10815000B0914501BC01CD0128E631E040E050E09E
:108160000E94468D20914408309145084091460870
:1081700050914708261737074807590764F0261B10
:10818000370B480B590B2093440830934508409314
:108190004608509347082091440830914508409183
:1081A00046085091470857FF0CC0260F371F481F3D
:1081B000591F209344083093450840934608509334
:1081C00047086091EC077091ED076E0D7F1D9B01D4
:1081D000442737FD4095542F8091090390910A035D
:1081E000A0910B03B0910C03820F931FA41FB51F26
:1081F0008093090390930A03A0930B03B0930C039D
:108200008091C3029091C402681B790BCB01AA270D
:1082100097FDA095BA2F29853A854B855C85820FFD
:10822000931FA41FB51F80930D0390930E03A0937B
:108230000F03B0931003C0908201D0908301E090AF
:108240008401F0908501C816D906EA06FB06C4F43D
:1082500088EA91E6A0E0B0E08C199D09AE09BF095B
:1082600080930D0390930E03A0930F03B09310031C
:108270008093090390930A03A0930B03B0930C031C
:1082800022273327A9012C193D094E095F09809146
:108290000D0390910E03A0910F03B091100382176C
:1082A0009307A407B507B4F4D701C601885A9146CD
:1082B000A040B04080930D0390930E03A0930F0352
:1082C000B09310038093090390930A03A0930B03C8
:1082D000B0930C036091FC077091FD07600F711F54
:1082E0009B01442737FD4095542F809111039091B5
:1082F0001203A0911303B0911403820F931FA41FC4
:10830000B51F8093110390931203A0931303B093AE
:1083100014038091C1029091C202681B790BCB01BA
:10832000AA2797FDA095BA2F2D853E854F855889A0
:10833000820F931FA41FB51F8093150390931603FC
:10834000A0931703B0931803E0908601F090870183
:108350000091880110918901E816F9060A071B07A8
:10836000C4F488EA91E6A0E0B0E08E199F09A00B62
:10837000B10B8093150390931603A0931703B0934A
:1083800018038093110390931203A0931303B093E7
:10839000140322273327A9012E193F09400B510B43
:1083A0008091150390911603A0911703B0911803C3
:1083B00082179307A407B507B4F4D801C701885AF8
:1083C0009146A040B0408093150390931603A0936C
:1083D0001703B09318038093110390931203A09393
:1083E0001303B09314038091050390910603A091A9
:1083F0000703B09108038093190390931A03A09385
:108400001B03B0931C038091150390911603A09158
:108410001703B09118038093350390933603A0930C
:108420003703B093380380910D0390910E03A09110
:108430000F03B091100380932D0390932E03A0930C
:108440002F03B09330038091110390911203A091F8
:108450001303B09114038093310390933203A093DC
:108460003303B09334038091090390910A03A091E0
:108470000B03B0910C038093290390932A03A093DC
:108480002B03B0932C0380911B0190911C0197FD4D
:10849000079603E0959587950A95E1F79093FD0778
:1084A0008093FC078091190190911A0197FD07961E
:1084B00013E0959587951A95E1F79093ED078093D2
:1084C000EC078091FE019091FF010F9734F488E151
:1084D0009CEF9093FD078093FC078091FE019091A3
:1084E000FF01079734F480E398EF9093FD078093A2
:1084F000FC07209101012A30A9F48091FE0190919E
:10850000FF01835F934034F088EE93E09093FD0782
:108510008093FC078091FE019091FF018A5F934058
:10852000DCF014C08091FE019091FF01815D9740C5
:1085300034F088EE93E09093FD078093FC078091E0
:10854000FE019091FF01805E974034F080ED97E04E
:108550009093FD078093FC078091FC019091FD01B1
:108560000F9734F488E19CEF9093ED078093EC072C
:108570008091FC019091FD01079734F480E398EF1E
:108580009093ED078093EC072A30A9F48091FC01C9
:108590009091FD01835F934034F088EE93E09093D7
:1085A000ED078093EC078091FC019091FD018A5FBB
:1085B0009340DCF014C08091FC019091FD01815D3D
:1085C000974034F088EE93E09093ED078093EC07AA
:1085D0008091FC019091FD01805E974034F080ED28
:1085E00097E09093ED078093EC0760917401662308
:1085F00009F4AFC040911B0150911C0180915E03B2
:1086000090915F03481B590B50936503409364039B
:1086100020911B0130911C01280F391F37FF02C028
:108620002F5F3F4F3595279530935F0320935E036F
:10863000413851051CF080E890E005C040585F4F7C
:1086400034F480E89FEF9093650380936403409136
:10865000190150911A018091600390916103481BA8
:10866000590B509363034093620320911901309199
:108670001A01280F391F37FF02C02F5F3F4F359572
:1086800027953093610320936003413851051CF016
:1086900080E890E005C040585F4F34F480E89FEFD9
:1086A0009093630380936203462F55278091640360
:1086B00090916503849FB001859F700D949F700D0C
:1086C00011249B0177FF02C0215F3F4FF4E03595F5
:1086D0002795FA95E1F78091FC079091FD07820FAD
:1086E000931F9093FD078093FC0780916203909104
:1086F0006303849FD001859FB00D949FB00D11241A
:10870000AD019D01B7FF02C0215F3F4FE4E0359509
:108710002795EA95E1F78091EC079091ED07820F9C
:10872000931F9093ED078093EC0780911B0190912C
:108730001C01860F971F90931C0180931B01809151
:10874000190190911A01840F951F90931A0180933B
:1087500019010091FF07109100088091E3079091A3
:10876000E407101611065CF59C0197FF04C0222750
:108770003327281B390BC901AA2797FDA095BA2FCB
:1087800020916801332744275527BC01CD010E9461
:10879000468D9B01AC0197FF04C0215C3F4F4F4FBA
:1087A0005F4F76E055954795379527957A95D1F7A0
:1087B0008091FA079091FB07820F931F27C097FFC4
:1087C00003C0909581959F4FAA2797FDA095BA2F3A
:1087D00020916801332744275527BC01CD010E9411
:1087E000468D9B01AC0197FF04C0215C3F4F4F4F6A
:1087F0005F4F66E055954795379527956A95D1F770
:108800008091FA079091FB07821B930B9093FB07D3
:108810008093FA07E0900708F09008088091E70736
:108820009091E8071E141F045CF59C0197FF04C09B
:1088300022273327281B390BC901AA2797FDA095AA
:10884000BA2F20916801332744275527BC01CD0159
:108850000E94468D9B01AC0197FF04C0215C3F4FF5
:108860004F4F5F4F96E055954795379527959A95C9
:10887000D1F78091EE079091EF07820F931F27C0E9
:1088800097FF03C0909581959F4FAA2797FDA095CC
:10889000BA2F20916801332744275527BC01CD0109
:1088A0000E94468D9B01AC0197FF04C0215C3F4FA5
:1088B0004F4F5F4F86E055954795379527958A9599
:1088C000D1F78091EE079091EF07821B930B909365
:1088D000EF078093EE078091340887FF44C0B98981
:1088E000BB2309F040C08091BD028823E1F5E1E09F
:1088F000EE16E1E0FE064CF08091FC079091FD073A
:108900008E0D9F1D805091400DC0F0E0EF16FFEFDF
:10891000FF0664F48091FC079091FD078E0D9F1D6A
:1089200080509F4F9093FD078093FC0721E001301A
:1089300012074CF08091EC079091ED07800F911F8A
:10894000805091400CC03FEF0030130764F48091D9
:10895000EC079091ED07800F911F80509F4F9093EF
:10896000ED078093EC07E2E1CD5E0C94F18D8091F0
:10897000DA02882301F58091A3028C7F8093A30201
:10898000A0E2B4E0EAE1F7E09BE08091BB0188233C
:1089900009F48C938D91818312829150389697FFC0
:1089A000F4CF8091BB01882359F08091BB018150A5
:1089B0008093BB0105C08091A30281608093A302D4
:1089C00080912502882319F0109225020895809342
:1089D000270280932902809123028E7F80932302B5
:1089E00085EA8093BC000895CF93DF93ACEDB2E0AD
:1089F000CDE4D6E057E09991E92FFF27EE0FFF1F56
:108A0000E558F84F0190F081E02DE158FF4FEF3F1E
:108A1000F10521F01CF0EFEFF0E004C0F7FF02C019
:108A2000E0E0F0E0993111F4EC931BC04C91242F5D
:108A30003327E217F307A9F0CF01821B930B97FDB1
:108A400003969595879595958795242F280F2C93B8
:108A5000822F9927E817F90714F4215001C02F5FDE
:108A60002C935150119657FFC6CF80915706883FDF
:108A700038F0EFEFF0E0E81BF109E452FD4F8081A0
:108A800080937A0180917A01882329F0843618F046
:108A900084E680937A0180915906883F38F0EFEFA1
:108AA000F0E0E81BF109E452FD4F808180937801EA
:108AB00080917801882329F0843618F084E6809329
:108AC000780180916606883F38F0EFEFF0E0E81B10
:108AD000F109E452FD4F808180937301809173010D
:108AE0008B3010F48AE002C08F3F11F48093730141
:108AF00080919306883F38F0EFEFF0E0E81BF10932
:108B0000E452FD4F808180931308809113088630D2
:108B100010F485E002C08F3F11F480931308809118
:108B20009506883F38F0EFEFF0E0E81BF109E452DA
:108B3000FD4F808180933B0880913B08863010F484
:108B400085E002C08F3F11F480933B08809180063E
:108B5000873F19F4429905C006C0863F31F4439B14
:108B600002C08CE80BC086E409C0883F38F0EFEF04
:108B7000F0E0E81BF109E452FD4F8081809310087A
:108B800080918106873F19F4429905C006C0863F4F
:108B900031F4439B02C08CE80BC086E409C0883FD7
:108BA00038F0EFEFF0E0E81BF109E452FD4F80816F
:108BB0008093E90780918206883F38F0EFEFF0E07C
:108BC000E81BF109E452FD4F8081809319088091E0
:108BD0005806883F38F0EFEFF0E0E81BF109E45267
:108BE000FD4F80818093790180915B06883F38F04A
:108BF000EFEFF0E0E81BF109E452FD4F8081809334
:108C0000770180915D06883F38F0EFEFF0E0E81BD8
:108C1000F109E452FD4F80818093750180916506D2
:108C2000883F38F0EFEFF0E0E81BF109E452FD4F28
:108C300080818093760180916706883F38F0EFEF5E
:108C4000F0E0E81BF109E452FD4F8081809372014E
:108C500080916806883F38F0EFEFF0E0E81BF109FB
:108C6000E452FD4F80818093740180916906883FB2
:108C700038F0EFEFF0E0E81BF109E452FD4F80819E
:108C80008093710180916A06883F38F0EFEFF0E041
:108C9000E81BF109E452FD4F8081809370018091BF
:108CA0007006883F38F0EFEFF0E0E81BF109E4527E
:108CB000FD4F808180936E0180917106883F38F06E
:108CC000EFEFF0E0E81BF109E452FD4F8081809363
:108CD000B80280917206883F38F0EFEFF0E0E81BB1
:108CE000F109E452FD4F80818093B70280917306B1
:108CF000883F38F0EFEFF0E0E81BF109E452FD4F58
:108D000080818093B60280917406883F38F0EFEF3F
:108D1000F0E0E81BF109E452FD4F80818093B50239
:108D200080918E06883F38F0EFEFF0E0E81BF10904
:108D3000E452FD4F80818093B40280918F06883F7A
:108D400038F0EFEFF0E0E81BF109E452FD4F8081CD
:108D50008093B30280919006883F38F0EFEFF0E007
:108D6000E81BF109E452FD4F80818093B2028091AB
:108D70009106883F38F0EFEFF0E0E81BF109E4528C
:108D8000FD4F80818093B10280917506883F38F055
:108D9000EFEFF0E0E81BF109E452FD4F8081809392
:108DA0006D0180917906883F38F0EFEFF0E0E81B25
:108DB000F109E452FD4F808180936C01809183061C
:108DC000883F38F0EFEFF0E0E81BF109E452FD4F87
:108DD000808180936B0180918606883F38F0EFEFA9
:108DE000F0E0E81BF109E452FD4F808180936A01B5
:108DF00080918706883F38F0EFEFF0E0E81BF1093B
:108E0000E452FD4F80818093690180918806883FFC
:108E100038F0EFEFF0E0E81BF109E452FD4F8081FC
:108E2000809368018091AF06883F38F0EFEFF0E063
:108E3000E81BF109E452FD4F80818093F80790917F
:108E4000B103992321F08091F807981720F08091C1
:108E5000F807882311F49093F807809155068093C2
:108E600034088091B5068093180880918D06883F5C
:108E700038F0EFEFF0E0E81BF109E452FD4F80819C
:108E8000809367018091A806883F38F0EFEFF0E00B
:108E9000E81BF109E452FD4F808180934B088091DB
:108EA0006E01282F33272F5F3F4F8CE398E2B901E3
:108EB0000E94858D70937C0160937B018091630695
:108EC00080933C0880916206809301089091AA06E5
:108ED000933308F44AC081E08093B002983F58F081
:108EE000EFEFF0E0E91BF109E452FD4F808182339E
:108EF00010F41092B00280917D012091B00282178F
:108F000021F18330F8F43091A101222351F08CED4E
:108F100095E09093DD018093DC01332369F48EE2C8
:108F200009C088EC90E09093DD018093DC0133234D
:108F300019F487E18093A10185E08093C502209315
:108F40007D0103C0815080937D0180918B089091B9
:108F50008C0897FF0FC08091B002882359F0809150
:108F60001B04806880931B0405C01092B0028AE045
:108F700080937D0180918B0890918C0897FF1DC094
:108F80008091DA028823C9F08091B0028823A9F089
:108F900080910701909108018F5F9F4F71F488E9DC
:108FA0009AE39093DD018093DC0180E094EA909352
:108FB0000801809307011092B0028091B0028823CB
:108FC00069F08091A20281608093A20280916A017F
:108FD000823D48F4825E80936A0105C08091A202BE
:108FE0008E7F8093A202DF91CF910895A7E1B0E038
:108FF000ECEFF7E40C94D58D0E94053D8091B60608
:1090000082FF27C08091BF029091C0020097F1F0CB
:1090100002E088359007D4F49C0197FF02C02D5FD1
:109020003F4F359527953595279580916D06992762
:10903000289FA001299F500D389F500D1124CA016F
:1090400064E670E00E94858DCB0106C08DE290E061
:1090500003C080916D0699279093A1028093A0028E
:109060006091E5027091E6027A836983809101083C
:1090700099270A966817790714F49A83898380914F
:10908000DB02843608F06AC08091A20282FD66C0CD
:1090900080917A0390917B03009731F00197909330
:1090A0007B0380937A030BC01092DA029093A5029F
:1090B0008093A4028091A3028D7E8093A30280916D
:1090C00001018A3011F0843110F0289A01C02898EB
:1090D0008091A4029091A502895E9340E0F1809175
:1090E000DA088536C0F18091A0029091A1029A839E
:1090F00089838091A30280618093A30280914906B5
:10910000A82FBB27AA0FBB1FFD01E155F84F118205
:10911000108280914A06282F3327220F331FC9015E
:109120008155984FFC0111821082A558B84F1196B5
:109130001C921E922558384FD90111961C921E92EE
:1091400080914C06E82FFF27EE0FFF1FE558F84FE0
:109150001182108203C31092DA0200C38091DB02F5
:109160008D3808F4FBC28091A3028F7E8093A30206
:1091700090916E0682E3989FC001112490937B0327
:1091800080937A03E981FA81B9978CF08091DA02B1
:10919000882369F08091A4029091A502FFEF8F3F90
:1091A0009F0729F001969093A5028093A4028091D5
:1091B000A4029091A5028F3F910509F008F5109245
:1091C000FD021092FE021092FF0210920003109214
:1091D000F9021092FA021092FB021092FC02109215
:1091E000660310926703109268031092690310924D
:1091F000050310920603109207031092080305C09E
:109200008091A30282608093A30280914B06E82F95
:10921000FF27EE0FFF1FE558F84F808191818135C0
:1092200091050CF438C12091DA02222309F033C1F0
:1092300080914C06E82FFF27EE0FFF1FE558F84FEF
:10924000808191818C3491050CF402C180917C0362
:109250008F5F80937C03893C08F41DC188E1809373
:10926000A10120937C031092A5021092A4023091D8
:109270004906E32FFF27EE0FFF1FE558F84F8081C7
:10928000918187349105B4F480914A06E82FFF2735
:10929000EE0FFF1FE558F84F808191810190F0811A
:1092A000E02DF7FF03C0F095E195FF4FE734F1059E
:1092B0000CF478C041E020914A06A22FBB27AA0FE8
:1092C000BB1FA558B84F8D919C911197873491057C
:1092D00044F0E32FFF27EE0FFF1FE558F84F808182
:1092E00091818D919C918734910574F0809149060C
:1092F000E82FFF27EE0FFF1FE558F84F808191817F
:10930000873491050CF042E0E22FFF27EE0FFF1F9C
:10931000E558F84F808191818634910574F48091ED
:109320004906E82FFF27EE0FFF1FE558F84F808111
:109330009181873491050CF043E0E22FFF27EE0F77
:10934000FF1FE558F84F808191818A5B9F4F74F42D
:1093500080914906E82FFF27EE0FFF1FE558F84FD1
:1093600080819181873491050CF044E0E22FFF2742
:10937000EE0FFF1FE558F84F808191818A5B9F4F68
:1093800074F480914906E82FFF27EE0FFF1FE55880
:10939000F84F80819181863491050CF445E0842F4B
:1093A0000E94DE2E80914A06E82FFF27EE0FFF1F56
:1093B000E558F84F808191810190F081E02DF7FF11
:1093C00003C0F095E195FF4F7E97CCF4809149065C
:1093D000E82FFF27EE0FFF1FE558F84F808191819E
:1093E0008A5B9F4F64F481E0809336041092C6023A
:1093F00088EE93E09093DD018093DC014CC00E94E5
:10940000E72F0E94892E80E00E94800980916F06DC
:109410000E944B898091340880FF10C08091130115
:1094200090911401875B934038F4809113019091DF
:1094300014018E5E924010F40E94651D80E00E942F
:10944000573A81E08093C6028093DA01579A1AC096
:1094500080819181855B9F4FE4F480917C038F5FD5
:1094600080937C03893CB8F02093DA0220937C033C
:109470001092A5021092A40281E00E94573A81E066
:109480008093C6020E94E72F68E770E00E94883947
:1094900002C020937C0380914B06E82FFF27EE0F3C
:1094A000FF1FE558F84F808191818B5A9F4F0CF038
:1094B00053C12091AB06E22FFF27EF77F070EE0F3C
:1094C000FF1FE155F84F80819181069714F084E6E3
:1094D00006C0808191818B5F9F4F1CF48CE9809343
:1094E0007F038091DA02E0914C06882309F0ECC0FA
:1094F000FF27EE0FFF1FE558F84F80819181855BB4
:109500009F4F9CF48091B60683FD0BC0E22FFF278E
:10951000EE0FFF1FE558F84F80819181855B9F4FCB
:10952000DCF08091AB068823B9F08091B60683FF0A
:10953000C8C08091AB06E82FFF27EE0FFF1FE5584C
:10954000F84F80819181875F9F4F0CF4BAC0809162
:109550007F03843609F0B5C02091C602222329F08A
:109560008091A30288608093A30280917D038F5F26
:1095700080937D038E3F08F4F1C010927D038091AB
:109580001B04882309F092C0222309F48FC0809124
:10959000B603882309F08AC081E090E09093A50289
:1095A0008093A40281E08093DA0210926603109205
:1095B00067031092680310926903109205031092DA
:1095C00006031092070310920803109201031092F1
:1095D0000203109203031092040380916406E82EA4
:1095E000FF240027112780913808909139089C01A9
:1095F000442737FD4095542FC801B7010E94468D7E
:10960000DC01CB018093150390931603A0931703FD
:10961000B093180380914808909149089C01442711
:1096200037FD4095542FC801B7010E94468DDC01DB
:10963000CB0180930D0390930E03A0930F03B0937F
:1096400010038091350390913603A0913703B091B8
:1096500038038093110390931203A0931303B093E4
:10966000140380912D0390912E03A0912F03B091AC
:1096700030038093090390930A03A0930B03B093E4
:109680000C031092FD021092FE021092FF02109243
:1096900000031092F9021092FA021092FB0210924B
:1096A000FC0284E68093C50284E350C08CED95E013
:1096B0009093DD018093DC01222309F04FC081E00B
:1096C00045C010927D034AC0FF27EE0FFF1FE558EB
:1096D000F84F808191818C3491059CF08091B60681
:1096E00083FD0BC0E22FFF27EE0FFF1FE558F84F59
:1096F00080819181855B9F4FCCF08091AB06882360
:10970000A9F08091B60683FF24C08091AB06E82FB4
:10971000FF27EE0FFF1FE558F84F808191818E5C87
:109720009F4FBCF480917F038C3999F480917E0324
:109730008F5F80937E038B3F88F01092DA02109245
:109740007E031092A5021092A40286E28093A101EA
:1097500005C010927E0302C010927F0380914001E9
:10976000815080934001809140018F3F21F0809192
:10977000A30284FFA9C30E94F444B0905F068091C5
:109780008803909189039C01220F331F280F391FF2
:10979000C0904906AC2DBB27AA0FBB1FFD01E558A1
:1097A000F84F4B2D552780819181849FB001859F73
:1097B000700D949F700D1124260F371F37FF02C0C4
:1097C0002D5F3F4FB9017595679575956795A155C3
:1097D000B84F80916006082F11278D919C91809F32
:1097E000D001819FB00D909FB00D11246A0F7B1F97
:1097F000709389036093880380918A0390918B030F
:109800009C01220F331F280F391FD0904A06AD2D1F
:10981000BB27AA0FBB1FFD01E558F84F808191813E
:10982000849FF001859FF00D949FF00D11242E0F61
:109830003F1F37FF02C02D5F3F4FA9015595479548
:1098400055954795A155B84F8D919C91809F70017A
:10985000819FF00C909FF00C11244E0D5F1D5093D2
:109860008B0340938A038091B002882309F448C097
:10987000CB0177FD0396DC01B595A795B595A79526
:10988000CA0157FD0396FC01F595E795F595E79517
:1098900080919C01682F772767FD70956A9F9001E2
:1098A0006B9F300D7A9F300D11248091B803482FA3
:1098B000552747FD50954E9FC0014F9F900D5E9FCD
:1098C000900D1124280F391F37FF02C0295F3F4F29
:1098D00093E0359527959A95E1F73093EC02209324
:1098E000EB026E9F90016F9F300D7E9F300D112413
:1098F0004A9FC0014B9F900D5A9F900D11243FC06D
:109900008091A906E82FFF27E85BFE4F86818093B0
:109910009C0190819093B803A82FBB27A7FDB09519
:10992000A69F9001A79F300DB69F300D1124E92FFF
:10993000FF27E7FDF095E49FC001E59F900DF49FA0
:10994000900D1124280F391F37FF02C0295F3F4FA8
:1099500083E0359527958A95E1F73093EC022093C3
:10996000EB02A49F9001A59F300DB49F300D1124F0
:10997000E69FC001E79F900DF69F900D1124281BD4
:10998000390B37FF02C0295F3F4F03E0359527951C
:109990000A95E1F73093EA022093E90280914C06A0
:1099A000E82FFF27EE0FFF1FE558F84F80819181C8
:1099B000909581959F4F9093E8028093E7028530C0
:1099C000910514F0049705C00FEF8C3F900734F415
:1099D00004969093E8028093E70204C01092E80294
:1099E0001092E7028091A403882309F43EC0282F37
:1099F00033278091EB029091EC0297FD079613E0DC
:109A0000959587951A95E1F7289FA001299F500DFC
:109A1000389F500D1124CA0157FD0F96B4E095955B
:109A20008795BA95E1F79093EC028093EB028091D1
:109A3000E9029091EA0297FD0796A3E09595879534
:109A4000AA95E1F7289FB001299F700D389F700DEE
:109A50001124CB0177FD0F96F4E095958795FA9543
:109A6000E1F79093EA028093E9028090EB029090F4
:109A7000EC028091A7039091A803881A990A90920A
:109A8000EC028092EB020091E9021091EA028091CF
:109A9000A5039091A603081B190B1093EA020093EB
:109AA000E90280914B06E82FFF27EE0FFF1FE558D4
:109AB000F84FE080F1808FE790E0E80EF91EF09219
:109AC000E602E092E502809173019927AA2797FDAB
:109AD000A095BA2FBC01CD010E94BA8CDC01CB014C
:109AE00020E030E040E251E4BC01CD010E94288C2E
:109AF000DC01CB01BC01CD010E948C8CDC01CB01CF
:109B0000809342088091720180931A0880917101BC
:109B10009927AA2797FDA095BA2FBC01CD010E94D5
:109B2000BA8CDC01CB0120E030E040E251E4BC0122
:109B3000CD010E94288CDC01CB01BC01CD010E942B
:109B40008C8CDC01CB018093F307809170018093B2
:109B500009088091420480FF59C080914B088138E8
:109B600008F454C080913B04992787FD90952B2DD4
:109B70003327829FD001839FB00D929FB00D112497
:109B80008A0E9B1E9092EC028092EB0280913C0424
:109B9000992787FD9095829FF001839FF00D929FFA
:109BA000F00D11240E0F1F1F1093EA020093E9021B
:109BB00080913D04282F332727FD30958091E702BF
:109BC0009091E802820F931F9093E8028093E7023E
:109BD00080913F04282F332727FD309580915A0626
:109BE0009927289F8001299F100D389F100D11245F
:109BF000109347010093460180913E0499278E15EA
:109C00009F0524F49093E6028093E5028091E5029B
:109C10009091E60297FF04C01092E6021092E502CE
:109C20008091340882FF02C010921A084091EB0222
:109C30005091EC02CA0157FD03969C01359527957A
:109C40003595279537FF03C0309521953F4F80917B
:109C5000A8029091A90282179307B4F4CA0157FF92
:109C600003C0909581959F4F97FD03969595879595
:109C7000959587959093A9028093A80285369105C2
:109C800044F084E690E001C001979093A90280938C
:109C9000A8024091E9025091EA02CA0157FD0396D9
:109CA0009C01359527953595279537FF03C030954D
:109CB00021953F4F8091A6029091A70282179307AA
:109CC000B4F4CA0157FF03C0909581959F4F97FD4B
:109CD000039695958795959587959093A702809380
:109CE000A6028536910544F084E690E001C0019714
:109CF0009093A7028093A6028091A30284FF08C0DC
:109D00001092A9021092A8021092A7021092A60225
:109D1000ED2DFF27EE0FFF1FE558F84F4091840609
:109D2000242F3327808191812817390744F48091AB
:109D3000B30682FF04C081E08093BC0213C0ED2D06
:109D4000FF27EE0FFF1FE558F84F842F992720912A
:109D50008506821B9109208131812817390714F467
:109D60001092BC0240914A06E42FFF27EE0FFF1F1E
:109D7000E558F84F50918406852F992722273327DD
:109D8000281B390B808191818217930744F48091BD
:109D9000B30683FF04C081E08093BB0216C08091AC
:109DA000BB02882391F0E42FFF27EE0FFF1FE55839
:109DB000F84F809185069927851B91092081318173
:109DC0008217930714F41092BB02EC2DFF27EE0FBD
:109DD000FF1FE558F84F40918406242F33278081D8
:109DE00091812817390744F48091B30680FF04C09D
:109DF00081E08093B90217C08091B902882399F05D
:109E0000EC2DFF27EE0FFF1FE558F84F842F992701
:109E100020918506821B91092081318128173907FD
:109E200014F41092B90240914906E42FFF27EE0F77
:109E3000FF1FE558F84F50918406852F9927222758
:109E40003327281B390B808191818217930744F4B3
:109E50008091B30681FF04C081E08093BA0216C0EE
:109E60008091BA02882391F0E42FFF27EE0FFF1FA5
:109E7000E558F84F809185069927851B9109208127
:109E800031818217930714F41092BA028091BC02B8
:109E9000882319F48091BB02811181E08093BD0277
:109EA0008091B902882321F48091BA02882351F06D
:109EB00081E08093BE021092BD021092BC0210920B
:109EC000BB0202C08093BE028091BD02882321F4B0
:109ED0008091BE02882369F08091830699272981A9
:109EE0003A818217930714F49A83898381E08093DF
:109EF000F1028091A20299279C012470307082FFA8
:109F00002DC08091A7039091A803909581959F4FB4
:109F10009093EC028093EB028091A5039091A603AD
:109F2000909581959F4F9093EA028093E9028091EA
:109F30008001909181019093E6028093E5028091E7
:109F400034088B778B6680933408809118088C7B5B
:109F50008093180888EC809379011EC08091A30239
:109F600084FF1AC03093E8022093E7023093EC029A
:109F70002093EB023093EA022093E9029AE5909352
:109F8000420888E780931A089093F30780930908A2
:109F90001092BD021092BE0280910C0890910D08A3
:109FA000A0910E08B0910F0820913503309136032F
:109FB0004091370350913803820F931FA41FB51FA0
:109FC00080930C0890930D08A0930E08B0930F088F
:109FD0008091140890911508A0911608B091170867
:109FE000E0902D03F0902E0300912F031091300389
:109FF000EB82FC820D831E838E0D9F1DA01FB11F5F
:10A000008093140890931508A0931608B09317082E
:10A010008091030890910408A0910508B09106086A
:10A02000E0903103F0903203009133031091340338
:10A03000EF82F88609871A878E0D9F1DA01FB11F1A
:10A040008093030890930408A0930508B093060832
:10A050008091F4079091F507A091F607B091F7076A
:10A06000E0902903F0902A0300912B0310912C0318
:10A07000EB86FC860D871E878E0D9F1DA01FB11FCE
:10A080008093F4079093F507A093F607B093F70732
:10A09000F090BE02FF86FF2029F48091BD02882344
:10A0A00009F460C010922503109226031092270332
:10A0B000109228031092210310922203109223037E
:10A0C0001092240310920C0810920D0810920E08A2
:10A0D00010920F081092140810921508109216088A
:10A0E00010921708109203081092040810920508A5
:10A0F000109206081092F4071092F5071092F607D6
:10A100001092F7078091150390911603A091170301
:10A11000B09118038093110390931203A09313033B
:10A12000B093140380910D0390910E03A0910F033F
:10A13000B09110038093090390930A03A0930B033B
:10A14000B0930C031092EC011092EB011092C2023A
:10A150001092C1021092C4021092C3020F85002314
:10A1600009F0F8C18091BD02882309F0F3C1809104
:10A17000EA059091EB05815092402CF48091DA022F
:10A18000882309F4E7C19090C408A0906406209049
:10A190003808309039084090480850904908191400
:10A1A0000CF0E3C0BB24CC24DD24CA01B901A60114
:10A1B00095010E94BA8D79018A0180918D08909154
:10A1C0008E08281A390AC101AA2797FDA095BA2F2F
:10A1D000E81AF90A0A0B1B0B6B817C818D819E8129
:10A1E000A60195010E94BA8D59016A0180918F08DC
:10A1F00090919008481A590AC201AA2797FDA09584
:10A20000BA2FA81AB90ACA0ADB0A292C332427FC58
:10A210003094432C532CC801B701A20191010E9434
:10A22000468D97FF04C061507E4F8F4F9F4F3B017B
:10A230004C0109E095948794779467940A95D1F737
:10A24000C601B501A20191010E94468D97FF04C08D
:10A2500061507E4F8F4F9F4F5B016C0119E0D59489
:10A26000C794B794A7941A95D1F78091A8029091BA
:10A27000A902813491053CF48091A6029091A70235
:10A2800081349105D4F0D401C30197FE03C0019637
:10A29000A11DB11D3C014D0195948794779467945D
:10A2A000D601C501D7FE03C00196A11DB11D5C01F9
:10A2B0006D01D594C794B794A79480914C06E82F6C
:10A2C000FF27EE0FFF1FE558F84F80819181019025
:10A2D000F081E02DF7FF03C0F095E195FF4F7A97ED
:10A2E000A4F0C401B30123E030E040E050E00E945C
:10A2F000BA8D39014A01C601B50123E030E040E0E2
:10A3000050E00E94BA8D59016A018091C608282F39
:10A31000332727FD3095432F532F26153705480542
:10A32000590514F439014A01992787FD90959095B4
:10A3300081959F4FAA2797FDA095BA2F6816790699
:10A340008A069B0614F43C014D012A153B054C0579
:10A350005D0514F459016A01A816B906CA06DB06A0
:10A360000CF0D0C05C016D01CDC0EA2CFF240027A9
:10A370001127CA01B901A80197010E94BA8D3901BC
:10A380004A01C101AA2797FDA095BA2F681A790A38
:10A390008A0A9B0A6B817C818D819E81A80197012D
:10A3A0000E94BA8D59016A01C201AA2797FDA095A2
:10A3B000BA2FA81AB90ACA0ADB0AD401C30197FE48
:10A3C00003C00F96A11DB11D3C014D01F4E0959411
:10A3D000879477946794FA95D1F7D601C501D7FE93
:10A3E00003C00F96A11DB11D5C016D01E4E0D59481
:10A3F000C794B794A794EA95D1F78091A802909159
:10A40000A902813491053CF48091A6029091A702A3
:10A4100081349105A4F0C401B30123E030E040E0B1
:10A4200050E00E94BA8D39014A01C601B50123E00E
:10A4300030E040E050E00E94BA8D59016A018091FD
:10A440004C06E82FFF27EE0FFF1FE558F84F8081DD
:10A4500091810190F081E02DF7FF03C0F095E19527
:10A46000FF4F7A97A4F0C401B30123E030E040E04D
:10A4700050E00E94BA8D39014A01C601B50123E0BE
:10A4800030E040E050E00E94BA8D59016A0189E154
:10A4900080938C0121E262167104810491042CF0F6
:10A4A00070E2672E712C812C912C30EE63163FEFF9
:10A4B00073063FEF83063FEF930644F460EE662E8B
:10A4C0006FEF762E6FEF862E6FEF962E41E2A41679
:10A4D000B104C104D1042CF050E2A52EB12CC12C42
:10A4E000D12C50EEA5165FEFB5065FEFC5065FEF06
:10A4F000D50644F440EEA42E4FEFB42E4FEFC42EF9
:10A500004FEFD42E8091150390911603A09117035D
:10A51000B091180386199709A809B9098093150302
:10A5200090931603A0931703B093180380910D0323
:10A5300090910E03A0910F03B09110038A199B090B
:10A54000AC09BD0980930D0390930E03A0930F03F4
:10A55000B09310038091EB019091EC018F3F910536
:10A5600009F008F4C4C56F85662309F04EC58091D3
:10A57000BD02882309F049C58091F102882309F0C2
:10A5800044C570918C06788B772309F43EC5809181
:10A590000C0890910D08A0910E08B0910F08B7FF1C
:10A5A00004C081509F4FAF4FBF4FE92EFA2E0B2FA3
:10A5B000112707FD1A95E0920C08F0920D08009300
:10A5C0000E0810930F088091140890911508A0911F
:10A5D0001608B0911708B7FF04C081509F4FAF4FC6
:10A5E000BF4F892F9A2FAB2FBB27A7FDBA95898B19
:10A5F0009A8BAB8BBC8B8093140890931508A09317
:10A600001608B093170880916406A82EBB24CC24AA
:10A61000DD2420912503309126034091270350919A
:10A620002803C601B5010E94468D97FF04C0615002
:10A630007F4F8F4F9F4F672E782E892E992487FC4E
:10A640009A94609225037092260380922703909239
:10A65000280320912103309122034091230350913C
:10A660002403C601B5010E94468D97FF04C06150C6
:10A670007F4F8F4F9F4F272E382E492E552447FC52
:10A680005A94209221033092220340922303509245
:10A69000240380911D0390911E03A0911F03B0918C
:10A6A0002003B7FF04C081509F4FAF4FBF4F892F8A
:10A6B0009A2FAB2FBB27A7FDBA9580931D039093CC
:10A6C0001E03A0931F03B0932003D801C70186196E
:10A6D0009709A809B9098093720390937303A09313
:10A6E0007403B093750320918B06E22EFF2400279C
:10A6F0001127BC01CD01A80197010E94BA8D590113
:10A700006A01209380033093810340938203509326
:10A71000830389899A89AB89BC8982199309A40921
:10A72000B5098093760390937703A0937803B09351
:10A730007903BC01CD01A80197010E94BA8D209335
:10A740008403309385034093860350938703D60197
:10A75000C501D7FE04C081509F4FAF4FBF4F892F17
:10A760009A2FAB2FBB27A7FDBA959093C202809377
:10A77000C10257FF04C021503F4F4F4F5F4FBB27CF
:10A7800057FDBA95A52F942F832F9093C4028093E1
:10A79000C3028091A8029091A90281349105DCF452
:10A7A0008091A6029091A70281349105A4F4809132
:10A7B0004C06E82FFF27EE0FFF1FE558F84F80816A
:10A7C00091810190F081E02DF7FF03C0F095E195B4
:10A7D000FF4F7A97E4F08091C4088F3FC1F48091D5
:10A7E000C1029091C20297FD01969595879590932D
:10A7F000C2028093C1028091C3029091C40297FD6E
:10A800000196959587959093C4028093C302809199
:10A81000030890910408A0910508B0910608B7FFBD
:10A8200004C081509F4FAF4FBF4F892F9A2FAB2F3E
:10A83000BB27A7FDBA958093030890930408A093C3
:10A840000508B09306088091F4079091F507A09150
:10A85000F607B091F707B7FF04C081509F4FAF4F85
:10A86000BF4F892F9A2FAB2FBB27A7FDBA95809397
:10A87000F4079093F507A093F607B093F70780913C
:10A88000350390913603A0913703B09138032F819F
:10A89000388549855A85281B390B4A0B5B0B209359
:10A8A0006A0330936B0340936C0350936D03809164
:10A8B0002D0390912E03A0912F03B0913003EB84D0
:10A8C000FC840D851E85E81AF90A0A0B1B0BE09221
:10A8D0006E03F0926F030093700310937103209343
:10A8E0007203309373034093740350937503E092A3
:10A8F0007603F092770300937803109379038091A5
:10A90000110390911203A0911303B0911403821BC1
:10A91000930BA40BB50B8093110390931203A09398
:10A920001303B09314038091090390910A03A0913B
:10A930000B03B0910C038E199F09A00BB10B8093F0
:10A94000090390930A03A0930B03B0930C03888927
:10A950008823E1F02091EF023091F0022138310597
:10A960004CF08091460390914703019690934703E2
:10A970008093460320583F4F4CF4809146039091BA
:10A980004703019790934703809346031092F00288
:10A990001092EF0281E090E090938D0380938C03FE
:10A9A000E0907203F09073030091740310917503AB
:10A9B000D801C70117FF07C088279927DC018E1926
:10A9C0009F09A00BB10B81509240A040B04034F0E1
:10A9D00084E090E090938D0380938C0380919203A8
:10A9E00090919303A0919403B091950320910C084A
:10A9F00030910D0840910E0850910F08821B930B67
:10AA0000A40BB50B815E914BAF4FBF4F8F539C4949
:10AA1000A040B04028F08091C50889310CF4FFC0F7
:10AA200021E0E21620E1F20620E0020720E0120712
:10AA30000CF473C080918E03882309F46AC0D80196
:10AA4000C70117FF07C088279927DC018E199F09C6
:10AA5000A00BB10B9C01AD01B7FF04C021503E4FCC
:10AA60004F4F5F4FF9E05595479537952795FA95E4
:10AA7000D1F780918C0390918D03820F931F909357
:10AA80008D0380938C03D801C70117FF03C007967D
:10AA9000A11DB11DE3E0B595A79597958795EA951A
:10AAA000D1F78093800390938103A0938203B093A6
:10AAB000830389589341A040B04064F088E893E153
:10AAC000A0E0B0E08093800390938103A093820381
:10AAD000B0938303209180033091810340918203DE
:10AAE0005091830357FF04C021503F4F4F4F5F4F9A
:10AAF000232F342F452F552747FD5A958091C102AA
:10AB00009091C202820F931F9093C2028093C10260
:10AB100006C081E080938E0302C010928E0340E055
:10AB2000E41640EFF4064FEF04074FEF14070CF064
:10AB300073C080918F03882309F46AC0D801C701CC
:10AB400017FF07C088279927DC018E199F09A00BE2
:10AB5000B10B9C01AD01B7FF04C021503E4F4F4FD8
:10AB60005F4F69E055954795379527956A95D1F7D9
:10AB700080918C0390918D03820F931F90938D038E
:10AB800080938C03D801C70117FF03C00796A11D4E
:10AB9000B11D23E0B595A795979587952A95D1F78F
:10ABA0008093800390938103A0938203B0938303E7
:10ABB00088579C4EAF4FBF4F64F488E79CEEAFEFD1
:10ABC000BFEF8093800390938103A0938203B0939F
:10ABD000830320918003309181034091820350913F
:10ABE000830357FF04C021503F4F4F4F5F4F232F28
:10ABF000342F452F552747FD5A958091C1029091DA
:10AC0000C202820F931F9093C2028093C10211C0AF
:10AC100081E080938F030DC010928F030AC01092C1
:10AC20008D0310928C0384E690E090938B018093C7
:10AC30008A016889262F332780918C0390918D0398
:10AC40002817390724F430938D0320938C03109137
:10AC5000C508112379F0212F332727FD30958091E6
:10AC60008C0390918D032817390724F430938D03BA
:10AC700020938C034091720350917303609174038D
:10AC800070917503413851056105710574F080912B
:10AC90004A0390914B0320918C0330918D03820FD6
:10ACA000931F90934B0380934A0340585F4F6F4F1D
:10ACB0007F4F74F480914A0390914B0320918C0351
:10ACC00030918D03821B930B90934B0380934A0327
:10ACD00081E090E090938D0380938C03C090760385
:10ACE000D0907703E0907803F0907903D701C60104
:10ACF000F7FE07C088279927DC018C199D09AE094A
:10AD0000BF0981509240A040B04034F084E090E010
:10AD100090938D0380938C03809196039091970379
:10AD2000A0919803B09199032091140830911508CF
:10AD30004091160850911708821B930BA40BB50B7A
:10AD4000815E914BAF4FBF4F8F539C49A040B040A5
:10AD500018F019310CF4FFC001E0C01600E1D00674
:10AD600000E0E00600E0F0060CF473C08091900370
:10AD7000882309F46AC0D701C601F7FE07C08827F7
:10AD80009927DC018C199D09AE09BF099C01AD0111
:10AD9000B7FF04C021503E4F4F4F5F4F09E055951C
:10ADA0004795379527950A95D1F780918C03909117
:10ADB0008D03820F931F90938D0380938C03D70193
:10ADC000C601F7FE03C00796A11DB11D13E0B5959E
:10ADD000A795979587951A95D1F7809384039093BB
:10ADE0008503A0938603B093870389589341A040BD
:10ADF000B04064F088E893E1A0E0B0E08093840381
:10AE000090938503A0938603B093870320918403D6
:10AE100030918503409186035091870357FF04C00A
:10AE200021503F4F4F4F5F4F232F342F452F552732
:10AE300047FD5A958091C3029091C402820F931FDF
:10AE40009093C4028093C30206C081E08093900374
:10AE500002C01092900320E0C21620EFD2062FEF1E
:10AE6000E2062FEFF2060CF073C080919103882365
:10AE700009F46AC0D701C601F7FE07C088279927E1
:10AE8000DC018C199D09AE09BF099C01AD01B7FF1A
:10AE900004C021503E4F4F4F5F4FE9E05595479515
:10AEA00037952795EA95D1F780918C0390918D0382
:10AEB000820F931F90938D0380938C03D701C6015B
:10AEC000F7FE03C00796A11DB11D73E0B595A795C8
:10AED000979587957A95D1F780938403909385030E
:10AEE000A0938603B093870388579C4EAF4FBF4F04
:10AEF00064F488E79CEEAFEFBFEF809384039093F8
:10AF00008503A0938603B093870320918403309137
:10AF10008503409186035091870357FF04C0215059
:10AF20003F4F4F4F5F4F232F342F452F552747FD5E
:10AF30005A958091C3029091C402820F931F9093FF
:10AF4000C4028093C30211C081E0809391030DC0BD
:10AF5000109291030AC010928D0310928C0384E624
:10AF600090E090938B0180938A014889242F3327A6
:10AF700080918C0390918D032817390724F4309326
:10AF80008D0320938C038091C508882379F0282FA6
:10AF9000332727FD309580918C0390918D032817DE
:10AFA000390724F430938D0320938C03409176036A
:10AFB000509177036091780370917903413851057E
:10AFC0006105710574F080914803909149032091C7
:10AFD0008C0330918D03820F931F909349038093CC
:10AFE000480340585F4F6F4F7F4FCCF48091480328
:10AFF0009091490320918C0330918D03821B930B18
:10B0000090934903809348030AC01092C40210929F
:10B01000C3021092C2021092C1021092F1028091FA
:10B020001A08882341F41092C4021092C3021092AD
:10B03000C2021092C10280910C0890910D08A0915B
:10B040000E08B0910F088093920390939303A093FE
:10B050009403B09395038091140890911508A091E2
:10B060001608B09117088093960390939703A093C6
:10B070009803B0939903109225031092260310921F
:10B08000270310922803109221031092220310929A
:10B0900023031092240310921D0310921E0310929A
:10B0A0001F031092200310920C0810920D081092AA
:10B0B0000E0810920F0810921408109215081092A2
:10B0C00016081092170810920308109204081092A4
:10B0D0000508109206081092F4071092F5071092D6
:10B0E000F6071092F7071092EC011092EB01E09036
:10B0F000E702F090E802C701F7FE04C0882799270D
:10B100008E199F0904973CF08091340884FD03C098
:10B1100082E38093C50210916106A12EBB24CC244A
:10B12000DD24B701882777FD8095982F9701F7FEDA
:10B1300004C0222733272E193F09442737FD4095A5
:10B14000542F0E94468D9B01AC01C601B5010E949F
:10B15000468D97FF04C061507E4F8F4F9F4F59E03F
:10B1600095958795779567955A95D1F79B01812F8E
:10B1700099278E9DD0018F9DB00D9E9DB00D1124FD
:10B18000CD01B7FD03969595879595958795280FE1
:10B19000391F8091C7029091C802280F391F442798
:10B1A00037FD4095542F20936603309367034093F7
:10B1B0006803509369038091050390910603A09161
:10B1C0000703B0910803821B930BA40BB50B80936C
:10B1D000050390930603A0930703B09308038155DA
:10B1E000934CA040B04064F080E593ECA0E0B0E068
:10B1F0008093050390930603A0930703B09308037D
:10B200008091050390910603A0910703B091080374
:10B21000805B9C43AF4FBF4F64F480EB9CE3AFEF88
:10B22000BFEF8093050390930603A0930703B093A9
:10B23000080300918E0110918F0117FDFCC08091D1
:10B24000340883FFF8C080918D01815080938D0177
:10B25000882309F0F4C08DE080938D01809135033F
:10B2600090913603A0913703B0913803B7FF04C023
:10B2700081509E4FAF4FBF4F39E0B595A795979539
:10B2800087953A95D1F77C0197FF04C0F094E1943B
:10B29000F108F39480912D0390912E03A0912F0338
:10B2A000B0913003B7FF04C081509E4FAF4FBF4FE6
:10B2B00029E0B595A795979587952A95D1F79C0193
:10B2C00097FF03C0309521953F4FE216F3060CF42B
:10B2D0007901B701F7FE02C0695F7F4F2B01A3E040
:10B2E00055944794AA95E1F722E030E0420E531EB0
:10B2F00060904408709045088090460890904708F8
:10B300002091420130914301409144015091450107
:10B31000C401B3010E94BA8D59016A013093F2074A
:10B320002093F107021B130BC801845E9D4F68E652
:10B3300071E00E94858D9C01245B304080918A01E0
:10B3400090918B01009731F0019790938B0180933E
:10B350008A011BC049E1E416F104BCF48091EF02BC
:10B360009091F002820F931F9093F0028093EF026E
:10B370008091C502882349F081508093C5028823BB
:10B3800021F4B092F402A092F30280918A0190918C
:10B390008B01892BF9F480918C019927289FB001AA
:10B3A000299F700D389F700D1124CB01B2010E94AE
:10B3B000858DCB01AA2797FDA095BA2F680E791E1F
:10B3C0008A1E9B1E6092440870924508809246082F
:10B3D000909247088091C502882369F58091F30215
:10B3E0009091F4022091F1073091F207821B930BA8
:10B3F000845E9D4F68E671E00E94858D9C01245B10
:10B4000030408091760186959927289FD001299F09
:10B41000B00D389FB00D11249D01B7FF02C0215F10
:10B420003F4FF4E035952795FA95E1F73093C80240
:10B430002093C70204C01092C8021092C7028091E4
:10B44000F102882381F01092F9021092FA02109210
:10B45000FB021092FC021092FD021092FE0210926A
:10B46000FF0210920003F090BE02FF20F1F48091E1
:10B470001A08282F332744275527809135039091A8
:10B480003603A0913703B0913803BC01CD010E946F
:10B49000468DDC01CB01BC01CD0128EF3AE240E052
:10B4A00050E00E94BA8D390102C066247724E090F2
:10B4B000BD02EE20F1F480911A08282F332744278B
:10B4C000552780912D0390912E03A0912F03B091C9
:10B4D0003003BC01CD010E94468DDC01CB01BC01D3
:10B4E000CD0128EF3AE240E050E00E94BA8D2901F8
:10B4F00002C0442455248091EE079091EF07893CC7
:10B5000091051CF088EC90E005C088539F4F34F4FF
:10B5100088E39FEF9093EF078093EE078091FA07FF
:10B520009091FB07893C91051CF088EC90E005C0E8
:10B5300088539F4F34F488E39FEF9093FB078093E9
:10B54000FA078091FC079091FD07AA2797FDA09527
:10B55000BA2F20914208A22EBB24CC24DD24BC01AA
:10B56000CD01A60195010E94468D9B01AC01809101
:10B57000EE079091EF07AA2797FDA095BA2FE7E075
:10B58000880F991FAA1FBB1FEA95D1F7280F391FF3
:10B590004A1F5B1F57FF04C0215C3F4F4F4F5F4F57
:10B5A00076E055954795379527957A95D1F783019C
:10B5B000020F131F1093FD070093FC078091EC0707
:10B5C0009091ED07AA2797FDA095BA2FBC01CD0158
:10B5D000A60195010E94468D9B01AC018091FA075E
:10B5E0009091FB07AA2797FDA095BA2F67E0880FD7
:10B5F000991FAA1FBB1F6A95D1F7280F391F4A1F31
:10B600005B1F57FF04C0215C3F4F4F4F5F4FF6E079
:10B610005595479537952795FA95D1F74201820EB2
:10B62000931E9092ED078092EC0780913D089091D7
:10B630003E08880F991FAA2797FDA095BA2F209141
:10B64000F307332744275527BC01CD010E94468DBF
:10B650005B016C0197FF08C02FE330E040E050E051
:10B66000A20EB31EC41ED51EE6E0D594C794B794AF
:10B67000A794EA95D1F780910908282F332744270A
:10B6800055278091190390911A03A0911B03B09143
:10B690001C03BC01CD010E94468DDC01CB01BC0125
:10B6A000CD0120EF35E540E050E00E94BA8DB501B4
:10B6B000620F731F70933E0860933D080150104164
:10B6C00034F080E090E19093FD078093FC07809137
:10B6D000FC079091FD078050904F34F480E090EF8C
:10B6E0009093FD078093FC0751E0851650E1950685
:10B6F00034F080E090E19093ED078093EC07809127
:10B70000EC079091ED078050904F34F480E090EF7B
:10B710009093ED078093EC076150704134F080E026
:10B7200090E190933E0880933D0880913D08909170
:10B730003E088050904F34F480E090EF90933E08A4
:10B7400080933D0880910001482F552780911D016D
:10B7500090911E014817590794F420911D013091D2
:10B760001E0109811A81049FC001059F900D149F3D
:10B77000900D1124B9010E94718D7A83698329810A
:10B780003A81220F331F220F331F3A8329834091BE
:10B79000340840FD02C00C94D663EE2011F00C94E6
:10B7A000D663FF2011F00C94D66300E010E048014E
:10B7B0008091BF029091C0029093D2058093D105F1
:10B7C00020914C0330914D032115310509F03FC004
:10B7D00080911301909114018959934058F087B5D5
:10B7E000803F20F48091EF01815011C081E080936F
:10B7F000A3034EC0809113019091140184369105EA
:10B8000008F587B58031D0F08091EF018F5F80938C
:10B81000EF019FE08902900111248091F405821BC1
:10B8200087BD8CE291E09093DD018093DC018EE591
:10B8300091E090934D0380934C032AC081E0809364
:10B84000A20326C0F092A203F092A30321C080912C
:10B85000D5029091D602A091D702B091D80264E0AF
:10B86000880F991FAA1FBB1F6A95D1F78093F0011B
:10B870009093F101A093F201B093F3011093EE01C4
:10B880000093ED012150304030934D0320934C0341
:10B890002091790141FF3DC0223338F5809190011C
:10B8A0008150809390018F3F09F053C08091F20244
:10B8B000882339F08091A101882319F488E28093CC
:10B8C000A1011092F2028091D5029091D602A0912E
:10B8D000D702B091D8028093D1029093D202A09364
:10B8E000D302B093D40281E011C0273490F180914B
:10B8F000F202882339F48091A101882319F487E2A8
:10B900008093A10181E08093F20288EC8093900102
:10B9100020C08091460190914701820F911D209196
:10B920005A063327829FA001839F500D929F500D8E
:10B930001124CA01AA2797FDA095BA2F8093D1029E
:10B940009093D202A093D302B093D40281E080936B
:10B95000F2028091350390913603A0913703B091A4
:10B960003803E0904201F0904301009144011091AE
:10B970004501BC01CD01A80197010E94BA8D590172
:10B980006A0180912D0390912E03A0912F03B09115
:10B990003003BC01CD01A80197010E94BA8DB90105
:10B9A000C5010E945B815C01CC971CF05CE3A52E75
:10B9B000B12CC5010E94ED705C0180E280934101D1
:10B9C0001092D0021092CF028091F202882309F4E3
:10B9D0005FC58091A30299279C012071307084FD7E
:10B9E00057C58091A20282608093A20270911808CC
:10B9F000872F992741E0C42ED12CC822D92280FD5F
:10BA000004C08091340881FD10C0C980DA80309371
:10BA10009B0320939A033093D0022093CF0280910E
:10BA2000A302806C8093A302ABC28091A30281FF2A
:10BA30007AC20091800110918101C8010F96209077
:10BA4000E5023090E602821593050CF058C0809113
:10BA5000A203882309F053C08091A30287FF15C079
:10BA60008091A3028F778093A3028091D502909159
:10BA7000D602A091D702B091D8028093D1029093C0
:10BA8000D202A093D302B093D4028091A302806427
:10BA90008093A302E090F807EE20F1F08091D102AC
:10BAA0009091D202A091D302B091D402BC01CD01F9
:10BAB00024E630E040E050E00E94BA8D8E2D9927B8
:10BAC000AA27BB2782179307A407B5072CF4D092A7
:10BAD000D002C092CF0210C0C101801B910B0F9702
:10BAE00097FF03C0909581959F4F9093D0028093CC
:10BAF000CF028BE2809341011092C90216C1C801A6
:10BB00000F9728163906C4F52091A3032223A1F527
:10BB10008091A30286FF15C08091A3028F7B809342
:10BB2000A3028091D5029091D602A091D702B09144
:10BB3000D8028093D1029093D202A093D302B09303
:10BB4000D4028091A30280688093A302C101801B6C
:10BB5000910B0F9697FF03C0909581959F4F9095FD
:10BB600081959F4F9093D0028093CF028DE2809376
:10BB700041012093C902D9C08DE3809341016091B6
:10BB8000CA02662371F12091CB023091CC02409120
:10BB9000CD025091CE028091D1029091D202A0911B
:10BBA000D302B091D40282179307A407B507CCF44F
:10BBB0008091A30280648093A302862F992790939B
:10BBC000D0028093CF028AE08093C9028EE58093F1
:10BBD00041018091A30287FFA8C08091A3028F77C3
:10BBE00033C0662309F443C02091CB023091CC02CC
:10BBF0004091CD025091CE028091D1029091D2021B
:10BC0000A091D302B091D402281739074A075B07E5
:10BC100074F58091A30280688093A302862F9927F0
:10BC2000909581959F4F9093D0028093CF0286EF9D
:10BC30008093C90286E7809341018091A30286FF29
:10BC400074C08091A3028F7B8093A3028091D50260
:10BC50009091D602A091D702B091D8028093D102E0
:10BC60009093D202A093D302B093D4025EC080918D
:10BC7000A302807C09F459C08091C902882379F518
:10BC8000E090D502F090D6020091D7021091D80230
:10BC9000D801C70180589040A040B0402091D10207
:10BCA0003091D2024091D3025091D402821793076F
:10BCB000A407B5075CF4D801C70180589F4FAF4F68
:10BCC000BF4F281739074A075B075CF08093D10202
:10BCD0009093D202A093D302B093D40202C01092E8
:10BCE000C9028091A3028F738093A30210929B03D9
:10BCF00010929A0371FF06C084EF91E09093DD01EA
:10BD00008093DC018091D902882379F48091D50257
:10BD10009091D602A091D702B091D802C397A10505
:10BD2000B1051CF081E08093D90260919A03709173
:10BD30009B038091CF029091D002680F791F70937E
:10BD40009B0360939A03CB0177FF04C08827992750
:10BD5000861B970B855F91400CF4CEC04091C902C1
:10BD6000442389F18091CB029091CC022091D102A1
:10BD70003091D202821B930B0996439748F480912D
:10BD8000CB029091CC02A091CD02B091CE0212C014
:10BD9000242F332727FD3095432F532F8091D10235
:10BDA0009091D202A091D302B091D402820F931F3E
:10BDB000A41FB51F8093D1029093D202A093D30207
:10BDC000B093D40224C080915A062091D1023091C0
:10BDD000D2024091D3025091D4021616170644F4B1
:10BDE00063E00E94658D280F311D411D511D07C064
:10BDF00063E00E94658D281B310941095109209398
:10BE0000D1023093D2024093D3025093D4021092C5
:10BE10009B0310929A03E090D502F090D602009115
:10BE2000D7021091D802D801C70180509440A04099
:10BE3000B0402091D1023091D2024091D302509172
:10BE4000D40282179307A407B5075CF4D801C70191
:10BE500080509C4FAF4FBF4F281739074A075B07E9
:10BE600044F08093D1029093D202A093D302B09376
:10BE7000D4028091180881FF06C084E690E0909378
:10BE8000DD018093DC0180915E068823A9F5809115
:10BE9000CA02882389F54091BF025091C00257FF22
:10BEA00002C04D5F5F4F55954795559547958091D9
:10BEB0001D0190911E01209100013327489FF00140
:10BEC000499FF00D589FF00D1124CF01B9010E9438
:10BED000858D7093810160938001663471051CF437
:10BEE00086E490E005C06739710534F086E990E09A
:10BEF000909381018093800180914C0390914D0338
:10BF0000892BD1F18091D5029091D602A091D702D0
:10BF1000B091D8028093D1029093D202A093D30221
:10BF2000B093D40229C08091D5029091D602A091FD
:10BF3000D702B091D80280599140A040B040809380
:10BF4000D1029093D202A093D302B093D4028091F5
:10BF50005E06882311F0992702C088E790E090934D
:10BF6000810180938001E980FA80F092C002E09222
:10BF7000BF028EE280934101C090BF02D090C00208
:10BF8000E090D502F090D6020091D7021091D8022D
:10BF90002091D1023091D2024091D3025091D4022B
:10BFA0002E153F054007510724F08091180880FDA9
:10BFB000BBC280914C0390914D03892B39F0C09006
:10BFC000BF02D090C00200E010E0D7C0D801C70186
:10BFD000821B930BA40BB50B80936A0390936B03A6
:10BFE000A0936C03B0936D03823000E890070FEFCD
:10BFF000A0070FEFB0072CF481E090E8AFEFBFEFA0
:10C0000009C08F5F9F47A040B04064F08FEF9FE76B
:10C01000A0E0B0E080936A0390936B03A0936C035D
:10C02000B0936D0300916A0310916B0380917801C6
:10C03000282F33274427552780916A0390916B035B
:10C04000A0916C03B0916D03BC01CD010E94468D9F
:10C0500097FF04C0615E7F4F8F4F9F4F25E09595FE
:10C060008795779567952A95D1F760936A037093C2
:10C070006B0380936C0390936D0365302EEF720712
:10C080002FEF82072FEF92072CF484E09EEFAFEFA3
:10C09000BFEF09C0605074408040904064F080E081
:10C0A00094E0A0E0B0E080936A0390936B03A093C8
:10C0B0006C03B0936D0380906A0390906B032091A2
:10C0C000ED013091EE0137FF02C0295F3F4F83E061
:10C0D000359527958A95E1F74FEF223834071CF400
:10C0E00021E83FEF05C02038310514F020E830E0AA
:10C0F000C901AA2797FDA095BA2F20917A0133276D
:10C1000044275527BC01CD010E94468D97FF04C0EE
:10C110006D5F7F4F8F4F9F4FB2E0959587957795D5
:10C120006795BA95D1F79B015FEF613075071CF4F5
:10C1300020E03FEF06C06F3F710519F014F020E0DA
:10C1400031E08091A302807C49F0C90137FD03965C
:10C150009C0135952795359527950DC08091180838
:10C1600080FF09C0C90137FD07969C01F3E03595B2
:10C170002795FA95E1F7820E931E209177012223ED
:10C1800009F454C06091F5027091F6028091F702B3
:10C190009091F80297FF04C061587F4F8F4F9F4FD7
:10C1A000E7E09595879577956795EA95D1F73327D9
:10C1B000442755270E94468D97FF04C0615E7F4F3C
:10C1C0008F4F9F4F55E095958795779567955A9531
:10C1D000D1F760936A0370936B0380936C03909321
:10C1E0006D036138AFEF7A07AFEF8A07AFEF9A07B9
:10C1F0002CF480E89FEFAFEFBFEF0AC06F3F7105EF
:10C200008105910569F064F080E091E0A0E0B0E084
:10C2100080936A0390936B03A0936C03B0936D03B8
:10C2200080916A0390916B03880E991E809175012D
:10C23000282F33278091C808992787FD9095289F3C
:10C24000F001299FF00D389FF00D11249F01F7FF99
:10C2500002C021583F4F220F232F221F330BFFEF25
:10C2600021383F071CF420E83FEF06C02F3F31057F
:10C2700019F014F020E031E0820E931EC401AA27C9
:10C2800097FDA095BA2FE090BF02F090C0029701F1
:10C29000442737FD4095542FBC01CD010E94468DA7
:10C2A00097FF04C061507E4F8F4F9F4F29E09595B7
:10C2B0008795779567952A95D1F7C61AD70A809101
:10C2C000CF029091D002892B09F060C01E141F0488
:10C2D0000CF05CC0980117FF03C0309521953F4FCB
:10C2E0002D33310540F48091ED029091EE028C15D2
:10C2F0009D0574F526C02C53304085E03695279572
:10C300008A95E1F72031310510F02FE030E04091BF
:10C31000ED025091EE0210161106E4F480E190E077
:10C32000821B930B489F9001499F300D589F300D01
:10C330001124B4E036952795BA95E1F72C153D0503
:10C3400020F580917E0190917F01C816D906F4F006
:10C350006C011CC0205F3F4F80917E0190917F0156
:10C36000829F8001839F100D929F100D11249801D0
:10C37000A4E036952795AA95E1F74C155D0514F0D4
:10C380006A0104C0C216D30608F06901C601AA27D3
:10C3900097FDA095BA2FFDE0880F991FAA1FBB1F1C
:10C3A000FA95D1F79501442737FD4095542FBC01EC
:10C3B000CD010E94BA8D20936E0330936F0340939A
:10C3C000700350937103C0906E03D0906F038091FF
:10C3D0009C0390919D039C01220F331F280F391F4E
:10C3E0002C0D3D1D37FF02C02D5F3F4FA901559514
:10C3F00047955595479550939D0340939C03809195
:10C400005606282F3327220F331F220F331F2417DE
:10C4100035076CF480913C08282F3327220F331FF7
:10C42000220F331F205530404217530724F030931A
:10C430009D0320939C038091180880FF14C0809175
:10C440009C0390919D0329813A818217930724F0E0
:10C4500030939D0320939C0340919C0350919D0336
:10C460005A83498361C029813A812E193F0937FFD8
:10C4700002C02D5F3F4F35952795359527956091E3
:10C480009C0370919D03620F731F7A8369834CC074
:10C4900080915E06882301F56091BF027091C00211
:10C4A00077FF02C06D5F7F4F7595679575956795AE
:10C4B00040911D0150911E0180910001282F3327CA
:10C4C000649FC001659F900D749F900D1124B90168
:10C4D0000E94858DCB0101C09927909381018093A3
:10C4E00080018091800190918101873491051CF435
:10C4F00086E490E005C08639910534F086E990E045
:10C50000909381018093800189819A8190939D030A
:10C5100080939C038091A302806C8093A3028091FE
:10C52000A2028D7F8093A2028091A30299279C0191
:10C530002270307081FF2BC180919E0390919F03E8
:10C54000A091A003B091A1030097A105B10521F02E
:10C550008091D9028130B1F4E981FA81CF01AA2713
:10C5600097FDA095BA2F1EE0880F991FAA1FBB1F29
:10C570001A95D1F780939E0390939F03A093A003F5
:10C58000B093A1038091D902813019F482E08093A5
:10C59000D902E980FA80C701AA2797FDA095BA2F92
:10C5A0009501442737FD4095542FBC01CD010E94D1
:10C5B000468DDC01CB0180936E0390936F03A093B3
:10C5C0007003B0937103B7FF04C08150904EAF4F1A
:10C5D000BF4F7C018D01ADE015950795F794E79469
:10C5E000AA95D1F7E0926E03F0926F030093700367
:10C5F000109371036091A4027091A5022FE0603A3C
:10C60000720750F580919E0390919F03A091A00323
:10C61000B091A1039C01AD01FAE05695479537957D
:10C620002795FA95D1F7821B930BA40BB50BA801A4
:10C630009701E4E0220F331F441F551FEA95D1F7FD
:10C64000820F931FA41FB51F80939E0390939F0397
:10C65000A093A003B093A10360547F4118F580918B
:10C660009E0390919F03A091A003B091A1039C0110
:10C67000AD016CE056954795379527956A95D1F7AA
:10C68000821B930BA40BB50BA8019701F2E0220FBC
:10C69000331F441F551FFA95D1F7820F931FA41F14
:10C6A000B51F38C08091ED019091EE018091ED01B0
:10C6B0009091EE0197FF03C0909581959F4F84362E
:10C6C000910584F58091D5029091D6022091D102F6
:10C6D0003091D202821B930B81509F4F8F5F91400C
:10C6E00008F580919E0390919F03A091A003B091C3
:10C6F000A1039C01AD01EEE056954795379527952E
:10C70000EA95D1F7821B930BA40BB50B8E0D9F1DE1
:10C71000A01FB11F80939E0390939F03A093A0033B
:10C72000B093A10380919E0390919F03A091A003D9
:10C73000B091A1037EE0B695A795979587957A95D8
:10C74000D1F79093C0028093BF0240915C064423CE
:10C7500099F055279C01BA010E94858DC901861B5D
:10C76000970B9093EE028093ED02260F371F3093C4
:10C770007F0120937E011FC01092EE021092ED0205
:10C780008FEF93E090937F0180937E0114C010920D
:10C79000D90210929E0310929F031092A003109250
:10C7A000A1033093C0022093BF0205C08091A30271
:10C7B000806C8093A3028091B20381FF37C089818E
:10C7C0009A8197FD039695958795959587952091E4
:10C7D000A0023091A1022817390760F48091BF02AE
:10C7E0009091C002892B31F0220F331F220F331F8B
:10C7F0003A8329838091D5029091D602A091D702E5
:10C80000B091D8028093D1029093D202A093D30228
:10C81000B093D40288E99AE39093DD018093DC0120
:10C8200080E09EE090930801809307012091010829
:10C83000822F9927880F991F880F991F88966981E1
:10C840007A818617970714F09A83898370913C0840
:10C850007D8B872F9927880F991F880F991F8055E7
:10C860009040A981BA818A179B0714F49A8389831F
:10C8700080912402882341F48091DA088F3F21F4CB
:10C880008091B6038823E9F08091A4029091A502DB
:10C890000297C097B0F4E981FA811E161F068CF446
:10C8A00081E090E09093A5028093A402E22EFF2401
:10C8B000EE0CFF1CEE0CFF1C8701085D1F4F1A8356
:10C8C000098329813A813093B6052093B50580917B
:10C8D000660390916703A0916803B091690312E029
:10C8E000880F991FAA1FBB1F1A95D1F700913D0809
:10C8F00010913E08081B190B213A31058CF0C90133
:10C9000037FD019695958795801791070CF48C015A
:10C91000909581959F4F081719076CF48C010BC0F7
:10C920000135110514F000E510E03FEF003B13075F
:10C9300014F400EB1FEF4D89242F3327220F331FF0
:10C94000220F331FC90169817A81861B970B8017DB
:10C9500091070CF48C0189819A81821B930B081733
:10C9600019070CF48C018091FC079091FD076091F0
:10C97000EB027091EC02861B970B90930B0880934F
:10C980000A08D0901A082091FD023091FE024091D1
:10C99000FF0250910003DD2041F0661A770AC301BF
:10C9A000AA2797FDA095BA2F04C0AA2797FDA095A6
:10C9B000BA2F280F391F4A1F5B1F2093FD023093A7
:10C9C000FE024093FF02509300038091FD0290917C
:10C9D000FE02A091FF02B091000381509A4FA04047
:10C9E000B04064F080E09AEFA0E0B0E08093FD02F8
:10C9F0009093FE02A093FF02B09300038091FD028A
:10CA00009091FE02A091FF02B091000380509640E9
:10CA1000AF4FBF4F64F480E096E0AFEFBFEF80937D
:10CA2000FD029093FE02A093FF02B0930003C0901A
:10CA30006B0620910A0830910B0878E0E72EEC1481
:10CA400098F08C2D9927829FA001839F500D929F73
:10CA5000500D1124CA0157FD07967C0163E0F5943F
:10CA6000E7946A95E1F712C08C2D86959927829FED
:10CA7000B001839F700D929F700D1124CB0177FD43
:10CA800003967C01F594E794F594E794A0907B01DC
:10CA9000B0907C019501442737FD4095542F80913B
:10CAA000FD029091FE02A091FF02B0910003BC0133
:10CAB000CD010E94BA8DE20EF31E90906701692DA0
:10CAC000772788279927980117FF04C02227332743
:10CAD000201B310B37FF02C02F5F3F4F3595279545
:10CAE000A981BA812A0F3B1F442737FD4095542F57
:10CAF0000E94468D97FF04C0615C7F4F8F4F9F4F10
:10CB000026E095958795779567952A95D1F79B01AE
:10CB10006E157F050CF47B01309521953F4FE21691
:10CB2000F3060CF479018091EC079091ED07609188
:10CB3000E9027091EA02861B970B9093EB078093B2
:10CB4000EA072091F9023091FA024091FB025091DC
:10CB5000FC02DD2041F0461A570AC201AA2797FDC0
:10CB6000A095BA2F04C0AA2797FDA095BA2F280F29
:10CB7000391F4A1F5B1F2093F9023093FA0240933A
:10CB8000FB025093FC028091F9029091FA02A0916D
:10CB9000FB02B091FC0281509A4FA040B04064F07B
:10CBA00080E09AEFA0E0B0E08093F9029093FA025F
:10CBB000A093FB02B093FC028091F9029091FA02DB
:10CBC000A091FB02B091FC0280509640AF4FBF4F46
:10CBD00064F480E096E0AFEFBFEF8093F9029093AA
:10CBE000FA02A093FB02B093FC022091EA07309175
:10CBF000EB0748E04C1598F08C2D9927829FB001E7
:10CC0000839F700D929F700D1124CB0177FD0796C5
:10CC10006C01B3E0D594C794BA95E1F712C0C694FD
:10CC20008C2D9927829FD001839FB00D929FB00DCC
:10CC30001124CD01B7FD03966C01D594C794D5940A
:10CC4000C7949501442737FD4095542F8091F902F0
:10CC50009091FA02A091FB02B091FC02BC01CD01BF
:10CC60000E94BA8DC20ED31E692D77278827992777
:10CC7000980117FF04C022273327201B310B37FFF1
:10CC800002C02F5F3F4F35952795E981FA812E0F1E
:10CC90003F1F442737FD4095542F0E94468D97FF34
:10CCA00004C0615C7F4F8F4F9F4FE6E0959587955D
:10CCB00077956795EA95D1F79B016C157D050CF486
:10CCC0006B01309521953F4FC216D3060CF46901D4
:10CCD00080910108282E33245090AC066AE1862EFC
:10CCE00067E0962E51EDA52E56E0B52E4BE0442E72
:10CCF0003BE1632E38E0732ED5012C9112160CF017
:10CD000029C1203429F4E981FA81FF8BEE8B1FC001
:10CD100049815A81CA01AA2797FDA095BA2F3327C6
:10CD200027FD3095432F532FBC01CD010E94468D26
:10CD300097FF04C0615C7F4F8F4F9F4F26E0959512
:10CD40008795779567952A95D1F77F8B6E8BF5013F
:10CD50002181203439F42E893F892E0D3F1D3F8BD0
:10CD60002E8B2AC0203C39F44E895F894E195F0909
:10CD70005F8B4E8B21C0C701AA2797FDA095BA2FC4
:10CD8000332727FD3095432F532FBC01CD010E943F
:10CD9000468D97FF04C0615C7F4F8F4F9F4FB6E079
:10CDA0009595879577956795BA95D1F7AE89BF899F
:10CDB000A60FB71FBF8BAE8BF5012281203439F44B
:10CDC0002E893F892C0D3D1D3F8B2E8B2AC0203C88
:10CDD00039F44E895F894C195D095F8B4E8B21C0F8
:10CDE000C601AA2797FDA095BA2F332727FD3095B6
:10CDF000432F532FBC01CD010E94468D97FF04C0E5
:10CE0000615C7F4F8F4F9F4FA6E0959587957795F3
:10CE10006795AA95D1F7AE89BF89A60FB71FBF8BBB
:10CE2000AE8BF5012381203439F42E893F89200F00
:10CE3000311F3F8B2E8B2AC0203C39F44E895F89ED
:10CE4000401B510B5F8B4E8B21C0C801AA2797FD59
:10CE5000A095BA2F332727FD3095432F532FBC01C0
:10CE6000CD010E94468D97FF04C0615C7F4F8F4FBC
:10CE70009F4FF6E09595879577956795FA95D1F749
:10CE8000AE89BF89A60FB71FBF8BAE8BF301808120
:10CE900091812E893F898217930764F4B901680F45
:10CEA000791F77FF02C06F5F7F4F759567957F8B06
:10CEB0006E8B1DC0552049F44E895F89440F551F64
:10CEC000481B590B5F8B4E8B12C051E0551578F4FF
:10CED000252D33276E897F89861B970BB9010E9408
:10CEE000858DAE89BF89A60FB71FBF8BAE8BC101E1
:10CEF000880F991F880F991FEE89FF898E179F074A
:10CF000064F4FD898F2F9927880F991F880F991F27
:10CF10002E893F892817390714F09F8B8E8B8E89B5
:10CF20009F8997FD03969595879595958795F4012B
:10CF30008183880F991F880F991F2E893F89281B8D
:10CF4000390BC901880F8283EE89FF89D301ED93E4
:10CF5000FC9303C0F401118212824A9422E030E073
:10CF6000620E731E44E050E0A40EB51E68E070E04F
:10CF7000860E971E47FEC0CEE2E1C95E0C94F18D8D
:10CF800084B1806A84B93D9A82E58CBD1DBC459A06
:10CF900081E080934E088AEA80935F0883E880935B
:10CFA00060088AE08093610810926308109262081A
:10CFB00010926508109264081092C70810928308B6
:10CFC000089530914E08332309F085C00DB407FE53
:10CFD00082C084E08093DB01459A2EB58091B9032D
:10CFE00099278130910589F0823091051CF4892BB5
:10CFF00021F03EC00297B9F03BC0309382082093E5
:10D00000BA032138A9F581E008C0253549F480919B
:10D01000BA03820F8093BA0382E08093B90328C0D9
:10D020003093B90325C080918208E82FFF27EC5583
:10D03000F74F20838F5F809382089091BA038032EC
:10D04000A0F0291769F480E2A4EAB8E0E4E8F8E087
:10D050000D9001928A95E1F781E08093830802C0E8
:10D06000309383081092B90303C0920F9093BA03D0
:10D0700020915E08223208F028C045980000000088
:10D0800000000000000000000000000000000000A0
:10D090000000000000000000000000000000000090
:10D0A000000000000000000000000000E0915708B0
:10D0B000F0915808E20FF11D80818EBD80918008AB
:10D0C0009081890F8093800803C081E080934E088F
:10D0D0002F5F20935E080895EF92FF920F931F93A6
:10D0E000809164069927880F991F880F991F7C01EA
:10D0F0000027F7FC0095102F80913503909136039F
:10D10000A0913703B0913803BC01CD01A80197016C
:10D110000E94BA8D309363082093620880912D039A
:10D1200090912E03A0912F03B0913003BC01CD014B
:10D13000A80197010E94BA8D309365082093640876
:10D140002091440830914508409146085091470885
:10D15000DA01C90163E0880F991FAA1FBB1F6A95F6
:10D16000D1F7820F931FA41FB51F820F931FA41F17
:10D17000B51F2091420130914301409144015091EB
:10D180004501BC01CD010E94BA8D30936B082093FC
:10D190006A0880914603909147032091FA013091EB
:10D1A000FB01821B930B9093710880937008E091B0
:10D1B0003C03F0913D038091110890911208BF014A
:10D1C0000E94858D9B01220F331F220F331F260FD4
:10D1D000371F260F371F37FF02C02D5F3F4F359592
:10D1E0002795359527953093670820936608809199
:10D1F000400890914108BF010E94858D9B01220F3C
:10D20000331F220F331F260F371F260F371F37FFFD
:10D2100002C02D5F3F4F3595279535952795309363
:10D2200069082093680810923D0310923C03109205
:10D230001208109211081092410810924008809133
:10D24000610899278D30910509F48CC08E309105C5
:10D250005CF48B30910509F4B4C08C3091050CF06E
:10D2600035C10A9761F0E7C18F30910509F4B3C168
:10D270008F3091050CF480C14097A9F1DCC18091F9
:10D28000B802809374088091B702809375088091EA
:10D29000B602809376088091B502809377088091DA
:10D2A000B402809378088091B302809379088091CA
:10D2B000B20280937A088091B10280937B088091BA
:10D2C000A30280937C088091A302837F8093A302B2
:10D2D0000E94E72F80937D088091AD0680937E08A1
:10D2E0008091A202A6C18091D4089091D508909314
:10D2F0007508809374088091D8089091D90890930C
:10D3000077088093760880911D0190911E0180938B
:10D310007808809100018093790880914101809381
:10D320007A089091BB0390937B08E92FFF27A3E035
:10D33000EE0FFF1FAA95E1F7E65EF84F8681809316
:10D340007C08838180937D08878180937E08858116
:10D3500080937F08892F8F5F6CE00E94658D90938A
:10D36000BB0369C1809198068093740880919906E7
:10D370008093750880919A068093760880919B0629
:10D380008093770880919C06809378088091A0060E
:10D39000809379088091A10680937A088091A206F3
:10D3A00080937B088091A50680937C088091A306DA
:10D3B00080937D088091A40680937E088091A606C4
:10D3C00038C1F89480914B06E82FFF27EE0FFF1F1E
:10D3D000E558F84F0190F081E02DE038F1051CF0A0
:10D3E000EFE7F0E006C02FEFE138F20714F4E1E8D0
:10D3F000FFEFE093740880914C06E82FFF27EE0FB3
:10D40000FF1FE558F84F0190F081E02DE038F1055D
:10D410001CF0EFE7F0E006C07FEFE138F70714F407
:10D42000E1E8FFEFE093750880914A06E82FFF27B7
:10D43000EE0FFF1FE558F84F0190F081E02DE03826
:10D44000F1051CF0EFE7F0E006C08FEFE138F807D8
:10D4500014F4E1E8FFEFE093760880914906E82FA5
:10D46000FF27EE0FFF1FE558F84F0190F081E02DE8
:10D47000E038F1051CF0EFE7F0E006C02FEFE138EF
:10D48000F20714F4E1E8FFEF7894E09377088091D5
:10D49000DC02809378088091DD0280937908809186
:10D4A000DE0280937A088091DF0280937B0880916E
:10D4B000E00280937C088091E10280937D08809156
:10D4C000E20280937E088091E302B3C0809136042B
:10D4D000863018F01092360485E0809374088091AD
:10D4E000A706809375088091D5029091D602A091ED
:10D4F000D702B091D802BC01CD0125E030E040E078
:10D5000050E00E94BA8D309377082093760880917E
:10D51000D1029091D202A091D302B091D402BC0169
:10D52000CD0125E030E040E050E00E94BA8D30931C
:10D5300079082093780880919D0680937A088091DD
:10D540009E0680937B0880919F0680937C08809143
:10D55000DB0280937D0880917B0790917C0780930C
:10D560007E088091B5059091B60597FD0396959537
:10D570008795959587955DC01092740888E580938E
:10D5800075088DE08093760883E380937708809117
:10D5900001018093780880911B0480937908809121
:10D5A0001C0480937A0810921B04807180931C04E1
:10D5B00080911D0480937B088091340880937C08BF
:10D5C0008091180880937D088091A90680937E0839
:10D5D0008091B6062EC080917D068093740880915C
:10D5E000B4068093750880916D01809376088091D0
:10D5F00076068093770880917706809378088091EB
:10D6000078068093790880916C0180937A088091E4
:10D610007A0680937B0880917B0680937C088091BA
:10D620007C0680937D088091DA0880937E08809143
:10D63000DF0580937F0880918308882309F469C1FE
:10D640006091840880919D01681719F08AEF80939A
:10D650009B0160939D0181E080938D01409185083D
:10D6600050918608CA0181509E4F8F5F9340B0F45D
:10D670002091870830918808C90181509E4F8F5FA3
:10D68000934060F48091550685FF08C05093A8032D
:10D690004093A7033093A6032093A50380918B08A2
:10D6A00090918C0821E08936920724F490938F01A1
:10D6B00080938E0120919508309196088091DC012D
:10D6C0009091DD018217930740F48091B001882387
:10D6D00021F43093DD012093DC01862F99278936D0
:10D6E000910509F4A5C08A36910544F48736910561
:10D6F00071F08836910509F462C013C18A3691052C
:10D7000009F400C18B36910509F4E2C00AC1809189
:10D7100097088093C408809198088093C6088091E8
:10D7200099088093C50880919A0880938C01809114
:10D730009B088093C80880919C0880939C018091ED
:10D740009D088093B80380919E088093A4038091E4
:10D75000B0028823F9F020919F083091A00837FD8E
:10D7600019C03093F4022093F30290917F0699231D
:10D7700089F08FE0989FC0011124281B390BC90143
:10D7800088599E4F68E671E00E94858D9093F4025F
:10D790008093F3022091AF033091B0038091A108F0
:10D7A0009091A208280F391F37FF02C02F5F3F4F0B
:10D7B000359527953093B0032093AF03B2C0809185
:10D7C0009708809359088091980880935A0880910F
:10D7D000990880935B0880919A0880935C088091F7
:10D7E0009B0880935D088091A50590919C08892BEA
:10D7F0008093A5059091A605937080919D088C70EB
:10D80000982B9093A60580919E088093B6038091F3
:10D810009F08809391018091A0088093C708809110
:10D82000A1088093B2038091A2088093B10379C0CC
:10D830008091970880934F088091980880935008B2
:10D84000809199088093510880919A08809352089A
:10D8500080919B0890919C08909354088093530862
:10D8600080919D0890919E0890935608809355084A
:10D8700080919F08992787FD90959093AE0780939C
:10D88000AD078091A0088093CA028091A108909171
:10D89000A2089C01442737FD4095542FDA01C901A5
:10D8A00063E0880F991FAA1FBB1F6A95D1F7820FEB
:10D8B000931FA41FB51F820F931FA41FB51F809332
:10D8C000CB029093CC02A093CD02B093CE0229C09C
:10D8D000809197088093B503809198088093B40352
:10D8E000809199088093B30390919A089923C9F085
:10D8F0008091A101882319F08151833090F4909395
:10D90000A1010FC080916F06863059F40E94847285
:10D9100008C01092A8031092A7031092A6031092B9
:10D92000A5031F910F91FF90EF90089580914E08ED
:10D93000882309F43BC045988FE598E090935808F8
:10D94000809357089091B703E92FFF27EE56FE4FBB
:10D950009F5F9093B703808180936108993010F0A6
:10D960001092B70310924E080E946C6881E0809379
:10D970005E08000000000000000000000000000041
:10D980000000000000000000000000000000000097
:10D990000000000000000000000000000000000087
:10D9A000000080915F08809380088EBD089587B144
:10D9B0008C6087B9429843981092BD0380E88093A9
:10D9C0009F011092BC0380939E0108958091C20331
:10D9D00081508093C2038F3F09F019C189E0809381
:10D9E000C2038091A302992780739070892B21F440
:10D9F00080911C0480FF1DC080919606882351F001
:10DA00008091C503882319F484E08093BD0381E0ED
:10DA10008093C503809197068823B9F08091C6034F
:10DA2000882319F484E08093BC0381E08093C603CB
:10DA30000CC01092C5031092C60380919206809389
:10DA4000C303809194068093C4038091C503882307
:10DA500009F045C08091B306282F332724FF07C063
:10DA60008091DA02882319F425FD52C053C09091A9
:10DA70009306983F48F0809113088D3D28F08091DF
:10DA8000C30388236CF00AC0983F78F08091130894
:10DA9000853059F48091C30387FF02C0429801C0CA
:10DAA000429A81E080939F0136C08091BD038150EE
:10DAB0008093BD038F3F79F58091130886958093FD
:10DAC000BD0380919F01813011F480E801C08695EB
:10DAD00080939F0180919F019091C30317C0809113
:10DAE000BD0381508093BD038F3FA9F489E08093EB
:10DAF000BD0380919F01813011F480E801C08695BB
:10DB000080939F0180919F0190919606892311F047
:10DB1000429A01C042988091C603882309F043C00D
:10DB20009091B30697FF07C08091DA02882319F419
:10DB300096FD52C053C090919506983F48F0809151
:10DB40003B088D3D28F08091C40388236CF00AC007
:10DB5000983F78F080913B08853059F48091C40358
:10DB600087FF02C0439801C0439A81E080939E01E1
:10DB700036C08091BC0381508093BC038F3F79F500
:10DB800080913B0886958093BC0380919E018130F3
:10DB900011F480E801C0869580939E0180919E01DA
:10DBA0009091C40317C08091BC0381508093BC0343
:10DBB0008F3FA9F489E08093BC0380919E0181305E
:10DBC00011F480E801C0869580939E0180919E01AA
:10DBD00090919706892311F0439A01C04398429B84
:10DBE00004C08091A202886003C08091A202877F56
:10DBF0008093A202439B06C08091A2028061809321
:10DC0000A20208958091A2028F7E8093A2020895BD
:10DC10000F931F93CF93DF93482FEB018091DB028B
:10DC2000E42FFF27843BD8F08F010E0F1F1FF80150
:10DC3000E558F84F808191819B01281B390BC90160
:10DC400063E070E00E94858DCB01880F991F860FDD
:10DC5000971F0155184FF8019183808306C0EE0F7E
:10DC6000FF1FE155F84F11821082E42FFF27EE0FBE
:10DC7000FF1FE558F84FD183C083DF91CF911F91EB
:10DC80000F9108954FB724E130E0F8948091C900D6
:10DC90008F778093C9008091C9008F7B8093C900E2
:10DCA0008091C9008F7D8093C9005A9A52985B9ADF
:10DCB000539A832F99278093CD002093CC00809195
:10DCC000C80082608093C80080E18093C900809181
:10DCD000CA008F778093CA008091CA008F7B80939F
:10DCE000CA008091CA008F7D8093CA008091CA00CB
:10DCF0008F7E8093CA008091CA00877F8093CA007C
:10DD00008091C9008B7F8093C9008091CA00846094
:10DD10008093CA008091CA0082608093CA0080917B
:10DD2000C80087FF03C08091CE00F9CF8091C90061
:10DD300080688093C9004FBF0895EF92FF920F93C0
:10DD40001F93CF93DF93482F00E010E08091A00154
:10DD5000813061F41092A00184E48093C903109291
:10DD6000CB031092CA031092CC03E6C18091C90381
:10DD7000882319F421E030E001C098019091CA0392
:10DD8000992371F4232B11F081E010C084E4809377
:10DD9000C9039093CB039093CA039093CC03B5C16E
:10DDA000913069F4232B09F0A6C182E08093CA0365
:10DDB0008091CB038F5F8093CB0383E0A4C192302B
:10DDC000D1F4232B09F097C183E08093C9034093DA
:10DDD000CC039091CB03923039F41092CD0347FFDE
:10DDE00003C081E08093CD0383E08093CA039F5FEB
:10DDF0009093CB038AC1933009F07DC1232B09F0A6
:10DE00007AC19093C90382E08093CA038091CB03C7
:10DE10008F5F8093CB032091CC03822F9927782F9B
:10DE20006627842F9927682B792B80916F06813084
:10DE300051F47370CB018050924063E070E00E9417
:10DE4000858DEB0119C0823069F47770CB01805069
:10DE5000944066E070E00E94858DEB012695269542
:10DE600026950CC0EB01D370C856D140CE01D7FD2A
:10DE70000196EC01D595C79526952695022F112779
:10DE80000F7010700F5F1F4F0D30110508F02CC17F
:10DE90000230110519F404E010E005C0043011054A
:10DEA00011F402E010E0D801A00FB11FFD01E55808
:10DEB000F84F808191819E01281B390BC90137FFE2
:10DEC00003C0909581959F4F069704F5E091B006A9
:10DED000EE2351F0FF27EE0FFF1FE558F84F80812A
:10DEE00091818436910594F48091DB02883C30F472
:10DEF0008091DB02865F8093DB0208C088EC809310
:10DF0000DB0280916F008F7D80936F00A558B84F22
:10DF10008D919C91BC01660F771F680F791F6C0F64
:10DF20007D1F77FF02C06D5F7F4F7B01F594E79403
:10DF3000F594E794CE0101968E159F0524F408947C
:10DF4000E108F10808C0CE010197E816F9061CF4B3
:10DF50000894E11CF11C0630110509F0ABC0C53670
:10DF6000D1050CF482C09091C803E92FFF27E75335
:10DF7000F74FE081ED3729F48091C70380958093B6
:10DF8000C703993009F06DC08091C703882319F445
:10DF9000E33821F066C0ED3709F063C08091CA080C
:10DFA0008D3739F48091CB08833899F463E87FEF9B
:10DFB0000DC0833871F48091CB08833819F460E088
:10DFC00070E004C08D3729F46DE770E085E00E94B1
:10DFD000086E8091CC088D3739F48091CF08833852
:10DFE00099F46DE770E00DC0833871F48091CF082B
:10DFF000833819F460E070E004C08D3729F463E8D9
:10E000007FEF86E00E94086E8091D0088D3739F44A
:10E010008091D108833899F463E87FEF0DC083388D
:10E0200071F48091D108833819F460E070E004C085
:10E030008D3729F46DE770E089E00E94086E8091C9
:10E04000CE08992787FD9095BC018AE00E94086E52
:10E050008091CD08992787FD9095BC018CE00E94A6
:10E06000086E1092C8031092C703CA30D1055CF441
:10E070008091C8038F5F8093C803E82FFF27E75381
:10E08000F74F83E880838091C8038A3011F410929F
:10E09000C8033FEFCC39D3076CF48091C803E82F55
:10E0A000FF27E753F74F8DE780838091C703809563
:10E0B0008093C7030530110518F4B701802F11C0F4
:10E0C0000730110519F4BE0187E00BC005301105BA
:10E0D00019F4BE0188E005C008301105B1F4BE0195
:10E0E0008BE00E94086E11C00231110570F081E0D2
:10E0F0008093A0010AC081E08093A0011092CB031D
:10E100001092CD0384E48093C9038091CB038031C6
:10E1100098F08091CD03882331F48091A001882369
:10E1200011F4809340011092CB031092CD03109212
:10E13000CA0384E48093C903E6E0CDB7DEB70C944C
:10E14000FD8DCF93FC0197FF05C0CFEFF095E195D2
:10E15000FF4F01C0C1E028E631E0CF01B9010E94C4
:10E16000858DFC018B35910554F08B5590408A3597
:10E17000910538F484EB90E08E1B9F0BFC0141E08D
:10E180000DC0CF01855B90408A35910518F4E45BA2
:10E19000F04003C02E1B3F0BF9014FEFEE0FFF1FA6
:10E1A000E85CF64F259134918C2F992787FD909547
:10E1B000289FB001299F700D389F700D1124842F66
:10E1C000992787FD9095689FA001699F500D789FC2
:10E1D000500D1124CA01CF9108952AE530E0281B83
:10E1E000390BC9010E94A1700895089508950895FA
:10E1F0000895089580E090E008951092D508109257
:10E20000D4081092D9081092D8081092D70810920A
:10E21000D6081092DA088AE090E00E943B199093A9
:10E22000CF038093CE030895CF93DF938091CE03E5
:10E230009091CF030E944419882309F4AFC08091C4
:10E24000CE039091CF030A969093CF038093CE0391
:10E25000E0E0F0E09F0190E05FEFAAE1B7E04BE083
:10E26000ED018B8187FF0BC09F5F8D81E80FF11D52
:10E270008981280F311D8E81851708F4582F415050
:10E28000189647FFEDCF5093DA08232B41F52091E4
:10E29000D4033091D5034091D6035091D703BB27C7
:10E2A000A52F942F832F9093D3038093D203AA2773
:10E2B000BB27281B390B4A0B5B0BCF01AA27BB27B7
:10E2C000280F391F4A1F5B1F2093D4033093D503B7
:10E2D0004093D6035093D703E5E0F0E013C02091BC
:10E2E000D2033091D3032E173F0718F4E21BF30B30
:10E2F00002C0E0E0F0E0892F9927880F991FE80F0E
:10E30000F91F3596F093D508E093D408EF3FF10557
:10E3100078F480911D0190911E018E9F90018F9F36
:10E32000300D9E9F300D1124C90164E670E013C0CA
:10E33000CF01969587959695879520911D013091EF
:10E340001E01289FA001299F500D389F500D1124B8
:10E35000CA0169E170E00E94718D7093D7086093E3
:10E36000D6082091D0033091D1032E0F3F1F309358
:10E37000D1032093D0035EE02131350778F08091FE
:10E38000D8089091D90801969093D9088093D8081D
:10E3900020513E403093D1032093D003DF91CF91A1
:10E3A00008953091DD03E32FFF2783E0EE0FFF1F79
:10E3B0008A95E1F7E65EF84F2781422F552747FD02
:10E3C00050958091DE039927841795072CF42093AC
:10E3D000DE033093E0030AC0222341F08091DF0383
:10E3E00099274817590714F42093DF03832F8F5F71
:10E3F0008093DD038D30D0F01092DD038091DF0338
:10E400008F3F19F08093D90302C01092D9038091F5
:10E41000DE038093DA038091E0038093D8038FEFCB
:10E420008093DF031092DE031092E003089595E1DC
:10E43000899F802D11240E94908787E69CE09F93FE
:10E440008F9382E697E89F938F93E0910204F09177
:10E45000030409950F900F900F900F900895CF939C
:10E46000C0E08091A30285FF02C0C0E125C0909169
:10E47000B6039923B1F08091DA02882349F4E92F99
:10E48000FF27EE0FFF1FE151F64F8491882349F4D7
:10E49000E92FFF27EE0FFF1FE251F64FC491CC2367
:10E4A00059F480E190E00E946B2E80FD03C0109231
:10E4B000A10102C0C091A1018091E1038C1771F408
:10E4C0008091E2039091E3030E944419882319F498
:10E4D00080E090E017C088E893E102C080ED97E00B
:10E4E0000E943B199093E3038093E203CC2331F025
:10E4F0008091A101C81711F41092A101C093E1030A
:10E500008C2F9927CF91089540E050E030E0809122
:10E51000A20899278A38910589F08B38910524F44F
:10E520008938910541F013C08D38910569F08E3816
:10E53000910539F00CC043E359E008C04BE05AE0C4
:10E5400005C04BED58E002C047E059E03CE2909135
:10E55000970820E080919808281770F4931760F4CA
:10E56000DA01A90FB11DE22FFF27EC57F74F85897C
:10E570008C939F5F2F5FEECF089520E335E7809166
:10E5800041018B3211F08D32F9F480915A06282F17
:10E5900033278091CF029091D002829FA001839F68
:10E5A000500D929F500D1124CA0163E070E00E944B
:10E5B000858DCB019B01205D3A48C196C19708F03B
:10E5C0003FC02EEF34E73CC0803229F58091A30292
:10E5D00081FF36C02091DB033091DC03205D3A4897
:10E5E00055E72133350748F085E72439380718F413
:10E5F00020E335E702C02456304045E72033340796
:10E60000F8F454E72D3C350718F020E335E718C03F
:10E610002C593F4F15C08E3549F49091CA028AE0BB
:10E62000989F90011124205D3A480AC0863741F432
:10E630009091CA028AE0989FC0011124281B390BCF
:10E64000C9010895EF92FF920F931F9399278A387B
:10E65000910509F4A6C08B38910524F489389105F9
:10E6600051F040C28D38910509F486C18E3891056C
:10E6700009F4E8C037C28091D5029091D602A091EA
:10E68000D702B091D802BC01CD0124E630E040E0D1
:10E6900050E00E94BA8DDA01C9018C509E4F9093D0
:10E6A0003909809338090E94BD7290933F09809385
:10E6B0003E099093410980934009909343098093C8
:10E6C0004209209138093091390980913C09909193
:10E6D0003D092817390724F430933D0920933C095C
:10E6E00080913A0990913B098217930724F4309363
:10E6F0003B0920933A091092350983E399E09093FE
:10E70000F2038093F1038091410180935909809134
:10E71000A20280FF02C083E401C080E280935A0914
:10E720002091B603222309F181E1289FF0011124F1
:10E73000A8E4B9E0E45DF54F9FE084918D9391509A
:10E74000319697FFFACF822F6AE00E94658D805D37
:10E7500080934409822F0E94658D892F805D80936C
:10E7600045098AE380934609BAC18091A30285FFD7
:10E770000CC0A4E4B9E0EBE3FCE094E184918D9358
:10E780009150319697FFFACFAAC1A4E4B9E0E1E530
:10E79000FCE094E184918D939150319697FFFACFEC
:10E7A0009EC18091D5029091D602A091D702B091DE
:10E7B000D802BC01CD0124E630E040E050E00E94E8
:10E7C000BA8DDA01C9018C509E4F9093210A809333
:10E7D000200A0E94BD729093230A8093220A88E740
:10E7E0008093240A809150088093250A0E942F72FA
:10E7F00080930D0A80914F0881FF02C084E407C016
:10E8000080915108833011F480E201C081E280934D
:10E81000260A8BE09AE09093F2038093F1038091B3
:10E8200091018093320A8091260A8093340A809164
:10E8300055089091560897FD019695958795809378
:10E84000270A4DC10E94D1718091D5029091D602C4
:10E85000A091D702B091D802BC01CD0124E630E0EE
:10E8600040E050E00E94BA8DDA01C9018C509E4F01
:10E870009093F6088093F50880911D0190911E01F8
:10E880009093F0088093EF0880911D0190911E01F4
:10E890009093F2088093F1088091F1079091F2072C
:10E8A00097FD0196959587958093E1088093E808F8
:10E8B000209155083091560837FF02C02F5F3F4F17
:10E8C000359527952093E608809153089091540838
:10E8D00064E170E00E94718D6093E7082093ED0879
:10E8E0006093EE080E94BD729093FE088093FD082D
:10E8F00088E78093FF0880911D0190911E019093FD
:10E90000FA088093F9088091D9038C5E8093F3080C
:10E910008091DA038C5E8093F4088091D8089091FE
:10E92000D9086AE070E00E94718D7093FC086093D2
:10E93000FB081092DD088091D4089091D50890933F
:10E94000F8088093F7088BED98E09093F20380939A
:10E95000F1032091AA013091AB01C9016CE370E091
:10E960000E94718D60930209C9016CE370E00E94FE
:10E97000718D80930309B3C00E94D17180915308B7
:10E980009091540864E670E00E94718D70931D09A7
:10E9900060931C098091F1079091F20797FD019611
:10E9A0009595879580930D0980915508909156080B
:10E9B00097FD0196959587958093120980910001A6
:10E9C000482F55279A012B5F3F4F80911D01909151
:10E9D0001E012817390784F480911D0190911E01B2
:10E9E000841B950B9C01220F331F280F391F822F88
:10E9F00082518093190902C010921909E090D50242
:10EA0000F090D6020091D7021091D802C801B70148
:10EA100024E630E040E050E00E94BA8D30931B09BC
:10EA200020931A0937FF04C010921B0910921A098B
:10EA3000C801B70124E630E040E050E00E94BA8D02
:10EA4000DA01C9018C509E4F90931F0980931E09D3
:10EA500080911D0190911E019093140980931309D8
:10EA600080911D0190911E019093160980931509C4
:10EA70000E94BD72909321098093200988E78093BA
:10EA8000220980911D0190911E0190932609809387
:10EA900025098091D9038C5E809317098091DA0350
:10EAA0008C5E809318098091D8089091D9086AE00B
:10EAB00070E00E94718D709328096093270910926D
:10EAC00009098091D4089091D508909324098093E6
:10EAD000230987E099E09093F2038093F1032CE2FD
:10EAE00030E002C020E030E0C9011F910F91FF909B
:10EAF000EF900895EF92FF920F931F93CF93DF93C0
:10EB00008091DB039091DC039C0153E0220F331FC3
:10EB10005A95E1F7281B390B8091ED019091EE0198
:10EB2000280F391F37FF02C0295F3F4F43E035955B
:10EB300027954A95E1F73093DC032093DB0390910E
:10EB4000E503992309F01DC38091E403282F33279F
:10EB5000442755278F5F8093E403F9012131310564
:10EB600008F00CC3E058FF4F0C940C8E8091A30268
:10EB700085FF2AC080E00E94908780911D019091BE
:10EB80001E016AE070E00E94858D9F938F938091B3
:10EB90001D0190911E016AE070E00E94858D7F93B7
:10EBA0006F938DE79CE09F938F9383E897E89F9303
:10EBB0008F93E0910204F091030409952DB73EB7BD
:10EBC000285F3F4F2DBF28C080E00E949087809132
:10EBD0001D0190911E016AE070E00E94858D9F9357
:10EBE0008F9380911D0190911E016AE070E00E9458
:10EBF000858D7F936F938AE89CE09F938F9382E645
:10EC000097E89F938F93E0910204F0910304099594
:10EC10008DB79EB708968DBF8091340880FF39C0AC
:10EC20008091F2028823E9F08AE00E949087809127
:10EC3000410199279F938F938091D5029091D6029D
:10EC4000A091D702B091D802BC01CD0124E630E0FA
:10EC500040E050E00E94BA8D3F932F9387E99CE0FB
:10EC600094C68AE00E9490878091D5029091D60246
:10EC7000A091D702B091D802BC01CD0124E630E0CA
:10EC800040E050E00E94BA8D3F932F9383EA9CE0CE
:10EC9000A4C78AE00E9490878EEA9CE00C94817F52
:10ECA0008091A30285FF2AC085E10E949087809110
:10ECB000AA019091AB016CE370E00E94718D9F936B
:10ECC0008F938091AA019091AB016CE370E00E9458
:10ECD000718D7F936F9388EB9CE09F938F9383E874
:10ECE00097E89F938F93E0910204F09103040995B4
:10ECF0002DB73EB7285F3F4F2DBF28C085E10E944A
:10ED000090878091AA019091AB016CE370E00E9422
:10ED1000718D9F938F938091AA019091AB016CE3C9
:10ED200070E00E94718D7F936F9385EC9CE09F93C0
:10ED30008F9382E697E89F938F93E0910204F0917E
:10ED4000030409958DB79EB708968DBF8FE10E9489
:10ED5000908780E690E09F938F938091F107909148
:10ED6000F2079F938F9382ED9CE09F938F93C2E66F
:10ED7000D7E8DF93CF93E0910204F0910304099563
:10ED80008091A2022DB73EB7285F3F4F2DBF80FF75
:10ED900006C089E20E9490878DED9CE074C389E2F1
:10EDA0000E9490878FED9CE00C94777F8091A30266
:10EDB00085FF1BC08AE20E9490878091D8089091BD
:10EDC000D9089F938F9381EE9CE09F938F9383E864
:10EDD00097E89F938F93E0910204F09103040995C3
:10EDE0008DB79EB706968DBF1BC08AE20E949087A2
:10EDF0008091D8089091D9089F938F9389EE9CE0D9
:10EE00009F938F9382E697E89F938F93E0910204FC
:10EE1000F091030409952DB73EB72A5F3F4F2DBFF0
:10EE200086E30E9490878091D4089091D5086AE08B
:10EE300070E00E94718D9F938F938091D408909180
:10EE4000D5086AE070E00E94718D7F936F9381EF27
:10EE50009CE09F938F9382E697E89F938F93E09136
:10EE60000204F091030409958DB79EB70896C3C6B6
:10EE700089E00E9490878DEF9CE09F938F9302E63C
:10EE800017E81F930F93E0910204F0910304099592
:10EE90008EE10E9490870F900F900F900F908FEF50
:10EEA0009CE09F938F931F930F93E0910204F09146
:10EEB0000304099583E30E9490870F900F900F90B1
:10EEC0000F9081E09DE09F938F931F930F93E091AC
:10EED0000204F091030409958FE30E9490870F903C
:10EEE0000F900F900F9083E09DE09F938F931F935F
:10EEF0000F93E0910204F091030409958EE70E94BC
:10EF000090870F900F900F900F9089E19DE09F9355
:10EF10008F931F930F93FBC780919B01882309F464
:10EF200062C08DE50E9490878FE29DE09F938F9352
:10EF3000C2E6D7E8DF93CF93E0910204F091030497
:10EF4000099584E50E9490870F900F900F900F9085
:10EF50008091500899279F938F9381E39DE09F9321
:10EF60008F93DF93CF93E0910204F091030409950E
:10EF70008EE50E9490872DB73EB72A5F3F4F2DBF89
:10EF800080915308909154086AE070E00E94718D5E
:10EF90007F936F938AE39DE09F938F93DF93CF934B
:10EFA000E0910204F091030409958DB79EB706968F
:10EFB0008DBF80915108833081F480914F0881FF8B
:10EFC00006C08BE50E94908784E49DE090C78BE5A6
:10EFD0000E94908787E49DE08AC78BE50E94908716
:10EFE0008AE49DE027C784E0D3C380919B018823F6
:10EFF00009F47AC08091E70392E6E92E97E8F92EAA
:10F00000882309F44BC089E60E9490878091B5035C
:10F0100099279F938F938DE49DE09F938F93FF9209
:10F02000EF92E0910204F0910304099585E70E94B4
:10F0300090872DB73EB72A5F3F4F2DBF809191013A
:10F0400099279F938F9300E610E01F930F93809171
:10F050005508909156089F938F9388E59DE09F9364
:10F060008F93FF92EF92E0910204F09103040995CF
:10F0700082E70E9490878DB79EB70A968DBF8091D8
:10F08000B30399279F938F931F930F938091B4039A
:10F0900099279F938F9384E69DE06DC689E60E9431
:10F0A00090878091910199279F938F9380E690E0BC
:10F0B0009F938F9380915508909156089F938F93BB
:10F0C0008091520899279F938F9384E79DE09F93A7
:10F0D0008F93FF92EF92E0910204F091030409955F
:10F0E0008DB79EB70C9687C585E052C39091B60345
:10F0F0009923D1F08091EE03882381F09F3170F441
:10F1000087E00E94177283E90E9490878091B6037E
:10F1100099279F938F938DE89DE0A4C383E90E9474
:10F12000908788E99DE0B3C38091A30202E6E02EB8
:10F1300007E8F02E85FF06C084E90E9490878EE9DB
:10F140009DE0DAC383E90E94908781EB9DE0D4C300
:10F150008091500A863059F48091E703882319F092
:10F160001092E70391C681E08093E7038DC6883053
:10F1700009F08AC60E94958781E07BC69093E403DC
:10F18000F0C6913009F0DEC38091E403282F3327C5
:10F19000442755278F5F8093E403F901213131051E
:10F1A00008F0DAC6EF56FF4F0C940C8E8091A30244
:10F1B00085FF43C080E00E9490878091D80890919D
:10F1C000D9089F938F9380911D0190911E016AE051
:10F1D00070E00E94858D9F938F9380911D01909187
:10F1E0001E016AE070E00E94858D7F936F9380918D
:10F1F000AA019091AB016CE370E00E94718D9F9326
:10F200008F938091AA019091AB016CE370E00E9412
:10F21000718D7F936F9387EC9DE09F938F9383E82D
:10F2200097E89F938F93E0910204F091030409956E
:10F230002DB73EB7225F3F4FABC580E00E9490875D
:10F240008091D8089091D9089F938F9380911D0148
:10F2500090911E016AE070E00E94858D9F938F93CC
:10F2600080911D0190911E016AE070E00E94858DE1
:10F270007F936F938091AA019091AB016CE370E052
:10F280000E94718D9F938F938091AA019091AB0101
:10F290006CE370E00E94718D7F936F9382EE9DE02E
:10F2A000C2C285E10E94908780E690E09F938F9391
:10F2B00080918E0190918F019F938F938DEF9DE0B0
:10F2C0009F938F93C2E6D7E8DF93CF93E091020438
:10F2D000F09103040995809134082DB73EB7285F5B
:10F2E0003F4F2DBF80FF51C08091F202882339F13A
:10F2F0008FE10E9490878091D5029091D602A091D3
:10F30000D702B091D802BC01CD0124E630E040E044
:10F3100050E00E94BA8D3F932F9387E09EE09F9329
:10F320008F9382E797E89F938F93E0910204F09187
:10F33000030409958DB79EB706968DBF38C08FE13F
:10F340000E9490878091D5029091D602A091D70219
:10F35000B091D802BC01CD0124E630E040E050E09D
:10F360000E94BA8D3F932F9380E19EE09F938F93ED
:10F37000DF93CF93E0910204F091030409952DB738
:10F380003EB72A5F3F4F2DBF12C08FE10E9490878A
:10F3900089E19EE09F938F93DF93CF93E0910204E6
:10F3A000F091030409950F900F900F900F9089E250
:10F3B0000E9490878091410199279F938F9383E2C8
:10F3C0009EE09F938F93DF93CF930DC480919B0119
:10F3D0008823F9F08BE20E94908780919101992710
:10F3E0009F938F9380915308909154086AE070E046
:10F3F0000E94718D7F936F9380E690E09F938F932F
:10F4000080915508909156089F938F9386E29EE0D5
:10F4100058C182E0BDC18FE30E9490878091D608D9
:10F420009091D7089F938F938091D4089091D5089D
:10F430006AE070E00E94718D9F938F938091D40851
:10F440009091D5086AE070E00E94718D7F936F9370
:10F450008DE39EE09F938F93C2E6D7E8DF93CF932F
:10F46000E0910204F091030409958091A2022DB766
:10F470003EB7265F3F4F2DBF80FF0AC082E50E9446
:10F48000908781E59EE09F938F9382E797E83DC543
:10F4900082E50E94908784E59EE029C580919B01CA
:10F4A00012E6E12E17E8F12E882309F449C084E51D
:10F4B0000E9490878091500899279F938F93809105
:10F4C000520899279F938F9387E59EE09F938F9390
:10F4D000E701FF92EF92E0910204F0910304099595
:10F4E0008DB79EB708968DBF80915108833051F437
:10F4F00084E60E9490878AE69EE09F938F93FF9216
:10F50000EF920BC084E60E94908780E79EE09F9375
:10F510008F9383E897E89F938F93E0910204F09193
:10F52000030409950F900F900F900F9080914F0852
:10F5300081FF17C584E60E94908786E79EE0D7C4C6
:10F5400084E50E9490878CE79EE0D6C18091E60317
:10F55000C2E6EC2EC7E8FC2E882309F450C089E6E9
:10F560000E949087809137076AE00E94658D892FFD
:10F5700099279F938F93809137070E94658D9927D4
:10F580009F938F9380912F070E94658D892F9927D4
:10F590009F938F9380912F070E94658D99279F934A
:10F5A0008F93809127070E94658D892F99279F93BC
:10F5B0008F93809127070E94658D99279F938F9342
:10F5C00080911F070E94658D892F99279F938F93A4
:10F5D00080911F070E94658D99279F938F9382E9E1
:10F5E0009EE09F938F93FF92EF92E0910204F0913F
:10F5F000030409952DB73EB72C5E3F4FC9C389E67A
:10F600000E94908780E690E09F938F9380913907C6
:10F61000992787FD90959F938F9380913107992724
:10F6200087FD90959F938F9380912907992787FD58
:10F6300090959F938F9380912107992787FD9095AF
:10F640009F938F938FEA9EE09F938F93FF92EF9209
:10F65000E0910204F091030409958DB79EB70E96D0
:10F66000CAC28091E60390914706882309F48DC0B1
:10F67000943009F48CC09630A1F58EE70E949087F3
:10F68000809147076AE00E94658D892F99279F9393
:10F690008F93809147070E94658D99279F938F9341
:10F6A00080913F070E94658D892F99279F938F93A3
:10F6B00080913F070E94658D99279F938F9382ECDD
:10F6C0009EE09F938F9382E697E89F938F93E091BC
:10F6D0000204F091030409952DB73EB7245F3F4F14
:10F6E00057C3973008F43DC48EE70E9490878091FD
:10F6F00057076AE00E94658D892F99279F938F9302
:10F70000809157070E94658D99279F938F938091D1
:10F710004F070E94658D892F99279F938F93809122
:10F720004F070E94658D99279F938F93809147077C
:10F730000E94658D892F99279F938F93809147070A
:10F740000E94658D99279F938F9380913F070E9418
:10F75000658D892F99279F938F9380913F070E94F2
:10F76000658D99279F938F9381ED9EE09F938F9353
:10F7700082E697E89F938F93E0910204F09103044F
:10F7800009958DB79EB7449636C2943021F486E031
:10F790000E941772E6C39630F1F48EE70E949087BC
:10F7A00080E690E09F938F9380914907992787FD8A
:10F7B00090959F938F9380914107992787FD90950E
:10F7C0009F938F938EEE9EE09F938F9382E697E8B0
:10F7D0009F938F93D4C2973008F4C3C38EE70E94DF
:10F7E000908780E690E09F938F93809159079927A7
:10F7F00087FD90959F938F9380915107992787FD5F
:10F8000090959F938F9380914907992787FD9095B5
:10F810009F938F9380914107992787FD90959F93A0
:10F820008F9381E09FE09F938F9382E697E89F9369
:10F830008F930ECF9091B603992309F44AC080911B
:10F84000EE038823F9F09F31E8F487E00E941772F5
:10F8500083E90E9490878091B60399279F938F93A5
:10F8600084E19FE09F938F9382E797E89F938F9324
:10F87000E0910204F091030409952DB73EB72A5F89
:10F880003F4F86C283E90E9490878FE19FE09F935C
:10F890008F9302E617E81F930F93E0910204F09113
:10F8A000030409951F921F929091B60381E1989FDE
:10F8B000C0011124845D954F9F938F931F930F93E5
:10F8C000E0910204F091030409958DB79EB70A9662
:10F8D00092C18091A302B2E6EB2EB7E8FB2E85FF22
:10F8E00006C084E90E94908785E29FE005C083E915
:10F8F0000E94908788E39FE09F938F93FF92EF92FF
:10F9000006C38091500A863079F48091E6038823FB
:10F9100019F01092E60303C081E08093E60385E0CE
:10F920000E94177286E09DC2883021F40E9495875C
:10F9300082E09FC2813009F0A7C20E949587109291
:10F94000E503A0C2923009F0A2C28091E403282FFF
:10F950003327442755278F5F8093E403F901213132
:10F96000310508F0F9C2EE55FF4F0C940C8E80E083
:10F970000E94908787EB96E09F938F930E94E72FDA
:10F9800099279F938F938EE49FE09F938F9382E7B5
:10F9900097E89F938F93E0910204F09103040995F7
:10F9A0002DB73EB7285F3F4FF3C185E10E94908796
:10F9B00085EC96E09F938F93809100016AE00E940E
:10F9C000658D892F99279F938F93809100010E94C5
:10F9D000658D99279F938F938DE59FE09F938F93DC
:10F9E00082E697E89F938F93E0910204F0910304DD
:10F9F00009956BCF8AE20E9490878EE69FE09F93E5
:10FA00008F93C2E6D7E8DF93CF93E0910204F091A1
:10FA100003040995809134080F900F900F900F9078
:10FA200080FF41C0809155069091790181FD0BC006
:10FA3000892F99279F938F9383E79FE09F938F93BD
:10FA4000DF93CF9315CFE0910204F0910304933339
:10FA500018F08DE79FE002C084E89FE09F938F93AA
:10FA6000DF93CF9309950F900F900F900F90809197
:10FA70001808E0910204F09103049091790180FF4D
:10FA80000BC0892F99279F938F938BE89FE09F93BB
:10FA90008F93DF93CF93ABC0892F99279F938F9339
:10FAA00081E99FE0CBC087E99FE021C28FE30E94FC
:10FAB000908780EA9FE09F938F93C2E6D7E8DF9319
:10FAC000CF93E0910204F091030409950F900F90F9
:10FAD0000F900F908091AA06882319F484EA9FE082
:10FAE00006C28091B002E0910204F09103048823E1
:10FAF00019F08DEA9FE002C084EB9FE09F938F9303
:10FB0000DF93CF9309950F900F900F900F908091F6
:10FB1000B50686FF26C28BEB9FE0E9C184E50E9413
:10FB2000908782EC9FE09F938F93C2E6D7E8DF93A4
:10FB3000CF93E0910204F091030409958091340879
:10FB40000F900F900F900F9085FD03C087EC9FE002
:10FB500011C080919806883F10F4E82F07C0EFEF9E
:10FB6000F0E0E81BF109E452FD4FE081E23358F484
:10FB700080ED9FE09F938F93DF93CF93E0910204FA
:10FB8000F091030416C0E43B18F087ED9FE0F2CF3C
:10FB90008091B506E0910204F091030485FF03C053
:10FBA0008EED9FE002C085EE9FE09F938F93DF93E1
:10FBB000CF9309950F900F900F900F908091AE0604
:10FBC000882309F4CEC18EE50E9490878091AE060D
:10FBD00099279F938F938CEE9FE09F938F9382E65C
:10FBE00097E89F938F93E0910204F09103040995A5
:10FBF0008DB79EB706968DBFB4C189E60E949087E7
:10FC000087EF9FE09F938F93C2E6D7E8DF93CF9370
:10FC1000E0910204F091030409950F900F900F906A
:10FC20000F908091AD06E0910204F09103048823C7
:10FC300051F099279F938F9381E090E19F938F9349
:10FC4000DF93CF9319CE85E090E19F938F93DF935D
:10FC5000CF9361C18091E803A2E6EA2EA7E8FA2ECD
:10FC6000882309F053C08EE70E94908780916D0130
:10FC700099279F938F9380914A06E82FFF27EE0FD5
:10FC8000FF1FE558F84F808191819F938F9380915A
:10FC90004906E82FFF27EE0FFF1FE558F84F808138
:10FCA00091819F938F938BE090E19F938F93FF922D
:10FCB000EF92E0910204F0910304099583E90E9418
:10FCC00090878DB79EB70A968DBF80914C06E82F1E
:10FCD000FF27EE0FFF1FE558F84F808191819F931A
:10FCE0008F9380914B06E82FFF27EE0FFF1FE558FB
:10FCF000F84F8081918181589F4F9F938F938FE11F
:10FD000090E19F938F93FF92EF9245CE8EE70E94F2
:10FD100090878091DE0299279F938F938091DD02D7
:10FD200099279F938F938091DC0299279F938F93BC
:10FD30008EE290E19F938F93FF92EF92E091020405
:10FD4000F0910304099583E90E9490878DB79EB7CF
:10FD50000A968DBF8091E10299279F938F9380919E
:10FD6000E00299279F938F938091DF0299279F93B9
:10FD70008F9382E490E19F938F93FF92EF92E091B3
:10FD80000204F091030409952DB73EB7265F3F4F5B
:10FD90002DBFE7C08091EE03882309F4E2C08EE70F
:10FDA0000E9490878091340886FD11C086E590E11D
:10FDB0009F938F9383E897E89F938F93E09102043A
:10FDC000F091030409950F900F900F900F90809180
:10FDD000B30699278F709070892B89F085E690E1A2
:10FDE0009F938F9383E897E89F938F93E09102040A
:10FDF000F091030409950F900F900F900F90809150
:10FE0000340882FF11C08FE690E19F938F9383E8BF
:10FE100097E89F938F93E0910204F0910304099572
:10FE20000F900F900F900F908091340883FD99C030
:10FE300084E790E19F938F9383E897E866C00091F1
:10FE4000500A063089F48091E803882319F0109253
:10FE5000E80303C081E08093E80386E00E94177204
:10FE600087E00E94177210C0083031F40E94958715
:10FE700083E08093E50306C0013031F40E9495874A
:10FE80000093E5031092E4031092500A6AC0933085
:10FE900009F065C08091E403282F33278F5F80939A
:10FEA000E4032130310581F0223031051CF4232B8D
:10FEB00029F037C022303105F9F033C08AE20E94C0
:10FEC000908782E890E11DC080E190E00E946B2E57
:10FED000C2E7D7E880FF06C081E30E94908789E8E7
:10FEE00090E105C081E30E94908787E990E19F93AC
:10FEF0008F93DF93CF930BC085E50E94908785EAAF
:10FF000090E19F938F9382E697E89F938F93E09180
:10FF10000204F091030409950F900F900F900F9039
:10FF200020C08091500A863061F480E190E00E9408
:10FF30006B2E91E09827692F80E190E00E94732E4C
:10FF400009C0813039F40E94958782E08093E503EF
:10FF50001092E4031092500A1092E40302C010922F
:10FF6000E503E6E0CDB7DEB70C94FD8D4FB728E191
:10FF700030E0F8948091C9008F778093C900809118
:10FF8000C9008F7B8093C9008091C9008F7D8093C9
:10FF9000C9005A9A52985B9A539A832F9927809353
:10FFA000CD002093CC008091C80082608093C8006F
:10FFB00080E18093C9008091CA008F778093CA0046
:10FFC0008091CA008F7B8093CA008091CA00809183
:10FFD000CA008F7E8093CA008091CA008860809397
:10FFE000CA008091C9008B7F8093C9008091CA00AC
:10FFF00084608093CA008091CA0082608093CA00A6
:020000021000EC
:100000008091C80087FF03C08091CE00F9CF809116
:10001000C90080688093C90080914E0A84608093F3
:100020004E0A4FBF08959091C903992341F48F3030
:1000300031F49093EA0380E58093C9030895E09139
:10004000EA03EF5FE093EA03E83121F481E0809373
:10005000E9030895E93120F089E18093EA030895E6
:10006000FF27E95CF54F80830895A0E0B0E0EBE363
:10007000F0E80C94DD8D91E0D92E82E0A82EBD2C05
:10008000E12C01E0F02E80914E0A82FDB5C08091F6
:100090006F008F7D80936F00E091B006EE2351F0EA
:1000A000FF27EE0FFF1FE558F84F808191818436BE
:1000B00091055CF48091DB02883C20F48091DB02A6
:1000C0008C5E01C088EC8093DB028091380A682F37
:1000D00077278091EB0381508093EB038F3F31F4BE
:1000E0001CE7C12E82E08093EB0302C0C4E2CC2E59
:1000F00040E04C1508F07EC0EA2DFF27E95CF54F83
:1001000080818D2111F06E297F298D2D9927880FEF
:10011000991FD82E882319F4B1E0DB2EAD0CEE0C1C
:10012000FF1C20E0E21628E0F20609F061C0A1E021
:10013000EA2EF12CCB018050944065E070E00E94E3
:10014000858DAB2DBB27FD01EA0FFB1FE558F84F4E
:10015000808191819C01220F331F280F391F260FA8
:10016000371F37FF02C02D5F3F4FE901D595C79577
:10017000D595C795CB0101968C179D0714F421974F
:1001800006C061507040C617D7070CF421968091C5
:10019000DB02833CD8F08D010A0F1B1FF801E558E4
:1001A000F84F80819181FE01E81BF90BCF0163E0DC
:1001B00070E00E94858DCB01880F991F860F971FD5
:1001C0000155184FF8019183808307C0AA0FBB1F08
:1001D000A155B84F11961C921E92EB2DFF27EE0FE2
:1001E000FF1FE558F84FD183C08360E070E0B394FF
:1001F0004F5F7FCF109240011092E903EAE0CDB744
:10020000DEB70C94F98D0895089500242227332732
:10021000442751E0BB27EE27FF27A0E1660F771F99
:10022000881F991F001C221F331F441F660F771F52
:10023000881F991F001C221F331F441F2AF4050E1C
:100240002B1F3E1F4F1F04C0051A2B0B3E0B4F0BDD
:10025000550FBB1FEE1F587F556047FD5250AA95A2
:10026000E9F6E695B7955795E695B7955795852F95
:100270009B2F08952227332741E0552768E0880FF8
:10028000991F221F331F880F991F221F331F1AF433
:10029000240F351F02C0241B350B440F551F487F08
:1002A000456037FD42506A9551F7569547955695EA
:1002B0004795842F0895AA2797FF04C080959095AD
:1002C0008A1F9A1F77FF04C0609570956A1F7A1F76
:1002D000669F9001779FA001679F300D411D5A1FB7
:1002E000300D411D5A1F889FF001999F2E0F3F1F0F
:1002F000401D511D899F300D411D5A1F300D411D5C
:100300005A1FCA01B901112480CF4FB720E430E051
:10031000F8948091C9008F778093C9008091C900BB
:100320008F7B8093C9008091C9008F7D8093C90025
:100330005A9A52985B9A539A832F99278093CD00AB
:100340002093CC008091C80082608093C80088E12F
:100350008093C9008091CA008F778093CA008091F2
:10036000CA008F7B8093CA008091CA008F7D8093E2
:10037000CA008091CA008F7E8093CA008091CA0013
:10038000877F8093CA008091C9008B7F8093C900CA
:100390008091CA0084608093CA008091CA00826004
:1003A0008093CA008091C80087FF03C08091CE006F
:1003B000F9CF8091C90080688093C9004FBF08952C
:1003C0000F931F93CF93DF93482F4F5F893108F02E
:1003D0008BC080917A07841720F44F5F40937A078F
:1003E0004150CB0183539B4268E170E00E94858DB0
:1003F000A42FBB27FD01EA0FFB1FE558F84F8081B2
:1004000091819B01281B390BC90137FF03C09095CF
:1004100081959F4F069794F48091DB02883C30F4DD
:100420008091DB02865F8093DB0208C088EC8093BA
:10043000DB0280916F008F7D80936F00FD01EA0FDA
:10044000FB1FE558F84F808191819C01220F331FDB
:10045000280F391F260F371F37FF02C02D5F3F4F70
:10046000E901D595C795D595C795CB0101968C1710
:100470009D0714F4219706C061507040C617D70736
:100480000CF421968091DB02843BD8F08D010A0F99
:100490001B1FF801E558F84F80819181FE01E81B90
:1004A000F90BCF0163E070E00E94858DCB01880FCE
:1004B000991F860F971F0155184FF801918380836C
:1004C00007C0AA0FBB1FA155B84F11961C921E92D0
:1004D000E42FFF27EE0FFF1FE558F84FD183C083AD
:1004E000443011F410924001DF91CF911F910F9190
:1004F0000895CF93DF932091510A822F9927807F0F
:100500009070409709F06CC02F3109F046C080917F
:10051000520A8093F5032091540A2093F7038091A7
:10052000550A8093F603822F992790937C07809336
:100530007B07222309F054C080914906282F3327D6
:10054000220F331FF901E155F84F1182108280917B
:100550004A06A82FBB27AA0FBB1FFD01E155F84F84
:100560001182108280914C06E82FFF27EE0FFF1FAB
:10057000CF018155984FEC01198218822558384FC8
:10058000E90119821882A558B84F11961C921E9243
:10059000E558F84F1182108223C0C22FCF70CA30A5
:1005A000F8F48091520A80937D0A8091530A8093D7
:1005B0007C0A8091540A80937F0A8091550A809327
:1005C0007E0A60917C0A70917D0A8C2F0E94E081E6
:1005D00060917E0A70917F0A8C2F8F5F0E94E0816C
:1005E000DF91CF910895CF93C82F8F3F49F4809129
:1005F000F8038F3F29F41092FA031092F90332C0E6
:100600002091FA03222339F4CF3111F485E001C09F
:1006100084E08093FB038091FB039091F9038217A0
:10062000A0F4892F80958093F9038F3F19F48EEF02
:100630008093F9038091F903C81711F40E9479821D
:100640001092FA031092F9030BC0E22FFF27EF5A22
:10065000F54FC0832F5F2093FA039C0F9093F9030B
:10066000C093F803CF9108959091F403933240F42E
:10067000E92FFF27E75AF54F80839F5F9093F4039C
:100680000895833218F48D5F8093F403089590E207
:10069000ECE5FAE08FE19193815087FFFCCF08955C
:1006A000CF93CFB723E031E0F8948091C9008F77E2
:1006B0008093C9008091C9008F7B8093C90080918D
:1006C000C9008F7D8093C9005A9A52985B9A539AB9
:1006D000832F99278093CD002093CC008091C80070
:1006E00082608093C80088E18093C9008091CA002D
:1006F0008F778093CA008091CA008F7B8093CA0055
:100700008091CA0080628093CA008091CA00806193
:100710008093CA008091CA0088608093CA0080914B
:10072000C90084608093C9008091CA00846080936E
:10073000CA008091CA0082608093CA008091C8007C
:1007400087FF03C08091CE00F9CF8091C9008068F7
:100750008093C9008091C90080648093C9000E9481
:100760004783CFBFCF910895282F99278F7090701E
:10077000892B31F420958091F303822B8093F3032E
:1007800008958091A401882309F44BC08091A302AD
:1007900085FD04C08091A801882381F082E98093BF
:1007A000590A83E280935A0A8091A801882309F4A8
:1007B00085E580935B0A1092A80102C08093590AD4
:1007C0008091A5018F3071F48091F3030E94FA703B
:1007D000882341F081E98093590A80935A0A81E382
:1007E00080935B0A1092A4018091C80085FFFCCF22
:1007F0008091C9008F7E8093C9008091C9008E7F4F
:100800008093C9008091590A882311F48EEF01C0AA
:100810008EE78093CE008091F3038093A501109220
:10082000F30308951F920F920FB60F9211248F9326
:100830009F93EF93FF939091A401992309F040C0F7
:100840008091FC03882361F48091590A882311F474
:1008500083E003C0813999F481E08093FC030FC0E9
:10086000833099F48091590A882349F09093590A6A
:100870008091C9008E7F8093C9008EEF1EC0809149
:10088000C90081608093C9000EC0833261F48091F9
:10089000C9008E7F8093C9008FEF8093CE0081E0E6
:1008A0008093A40114C08091FC03E82FFF27E75A2E
:1008B000F54F8F5F8093FC0380818093CE0007C04B
:1008C0001092FC038091C90080618093C900FF9160
:1008D000EF919F918F910F900FBE0F901F901895E1
:1008E000EF92FF920F931F93CF93DF937C018B01C5
:1008F000EA01452B39F0F80181918F01F701099543
:100900002197C9F7E6E0CDB7DEB70C94FD8DEF92E5
:10091000FF920F931F93CF93DF937C018B01EA012A
:10092000452B41F0F8010F5F1F4F8491F7010995A6
:100930002197C1F7E6E0CDB7DEB70C94FD8D0F939C
:100940001F93CF938C01C62F161634F480E2F80162
:100950000995C1501C16D4F3CF911F910F910895A2
:100960000F931F93CF938C01C62F161634F480E398
:10097000F8010995C1501C16D4F3CF911F910F9126
:100980000895A5E3B0E0E7ECF4E80C94D58D2E963D
:10099000EEADFFAD2E978824992454018091ED038C
:1009A000882321F42C961FAE1EAE2C975EE4452EB4
:1009B000512C4C0E5D1E6F01B60105C0153239F089
:1009C0000894C11CD11CF60114911123B9F7A6019A
:1009D000461B570B31F02C968EAD9FAD2C970E9485
:1009E0008784112309F46AC20894C11CD11CFF2416
:1009F000FDA6FCA64FEFE42EF9A6F6010894C11C53
:100A0000D11C1491153721F0812F80628837B1F401
:100A1000F0FE0AC0F20124E030E0420E531E808056
:100A20009180A280B3800AC0F20142E050E0440EFF
:100A3000551E808191814C01AA24BB24103221F4DF
:100A400089A58823D1F61DC0133219F458E0F52A80
:100A5000D4CF1A3211F01D3291F41A3259F4F20146
:100A600082E090E0480E591EE081ECA7EE232CF6C0
:100A7000E195ECA790E1F92AAFEDFA22BECF1B3247
:100A800011F419A7BACF1E32C1F5F6010894C11CA2
:100A9000D11C14911A3279F4F20122E030E0420EB6
:100AA000531E408151813FEF4F3F530714F44FEFE6
:100AB0005FEFE42EA2CF40E050E0812F80538A30D8
:100AC000A0F4CA0133E0880F991F3A95E1F7840F2B
:100AD000951F480F591F410F511D40535040F601BB
:100AE0000894C11CD11C1491E8CF8FEF4F3F5807D9
:100AF00014F44FEF5FEFE42E85CF103329F4F4FCAC
:100B00007CCF90E2F92A79CF812F81538930D8F4B4
:100B100040E050E0CA0123E0880F991F2A95E1F7D1
:100B2000840F951F480F591F410F511D40535040CE
:100B3000F6010894C11CD11C1491812F80538A3076
:100B400048F34CA75FCF183619F4A4E0FA2A55CF22
:100B50001C3619F4B1E0FB2A50CF133661F43E0184
:100B60000894611C711CF20122E030E0420E531E19
:100B7000808189833CC1143421F0143611F0193678
:100B800051F5143411F431E0F32AF0FE0AC0F201F9
:100B900044E050E0440E551E80809180A280B380D6
:100BA0000CC0F20182E090E0480E591E80819181D4
:100BB0004C01AA2497FCA094BA2CB7FE0AC0B094AA
:100BC000A09490948094811C911CA11CB11C8DE276
:100BD00089A70AE06FC01F3411F01F3631F41F34AB
:100BE00011F491E0F92A08E064C0103779F4F201B9
:100BF000A2E0B0E04A0E5B1E808191814C01AA24E4
:100C0000BB2400E1B0E4FB2A18E753C01337C1F559
:100C1000F20122E030E0420E531E608071806114C8
:100C2000710489F43E010894611C711C88E2898377
:100C30008EE6F301818385E78B838CE68C838D833D
:100C400089E28E831F82E7FC13C08E2D992787FDD2
:100C50009095AC0160E070E0C3010E94A28B009708
:100C600029F0382E3618E3140CF0C3C03E2CC1C056
:100C7000F30101900020E9F731973E2E3618B9C0F4
:100C8000153511F0153731F4153511F4F1E0FF2A5F
:100C90000AE00FC0183519F0183709F0A0C000E1BC
:100CA000F3FE07C081149104A104B10411F020E403
:100CB000F22A19A6EDA6E7FC02C03FEDF32289E275
:100CC000682E712C6C0E7D1E81149104A104B10458
:100CD00021F44DA5442309F47BC0802F9927AA272E
:100CE000BB278EA79FA7A8ABB9AB202E332490E0DB
:100CF000891690E0990691E0A90690E0B90648F0BF
:100D0000C501B4012EA53FA548A959A90E94988DF7
:100D100017C0AFEF8A169104A104B10449F040F066
:100D2000C401B1010E94718D9B014427552708C061
:100D3000882D602F0E94658D282F33274427552743
:100D40002AAB3BAB4CAB5DAB0A3059F48AA9880F98
:100D5000880F880F9AA9990F890F382D381B832F78
:100D600010C0003139F48AA98295807F482D481B34
:100D7000842F07C08AA9880F880F880F582D581B09
:100D8000852F90E02EA53FA548A959A98216930664
:100D9000A406B50608F091E08AA89BA8ACA8BDA857
:100DA0008A3010F4805D04C0895A183509F48F7DAB
:100DB000D3018E933D01992309F099CF083041F476
:100DC000F3FE06C0803321F080E3FD0182933F01F2
:100DD000CE010196382E3618F8E23F0E0BC01123D3
:100DE00009F46CC03E010894611C711C1983B1E0C8
:100DF0003B2E19A6032D2DA4231827FC222489A5F8
:100E0000882311F00F5F02C0F6FC0E5F020DEF2C7D
:100E1000FF24C70180739070892B49F48CA5801B37
:100E2000682F2C968EAD9FAD2C970E949F8489A52C
:100E3000882331F041E050E0BE01675D7F4F0AC07A
:100E4000E6FE0EC080E38AA71BA742E050E0BE0189
:100E5000665D7F4F2C968EAD9FAD2C970E9470845F
:100E6000C70180739070809749F48CA5801B682F10
:100E70002C968EAD9FAD2C970E94B084622D2C963F
:100E80008EAD9FAD2C970E94B084832D992787FD4E
:100E90009095AC01B3012C968EAD9FAD2C970E941E
:100EA0007084E4FE89CD2CA5201B2CA7622F2C96E4
:100EB0008EAD9FAD2C970E949F847ECDE2E1CB5CEE
:100EC0000C94F18D982F8091580A883A50F48091B3
:100ED000580AE82FFF27E15AF64F93838F5F8093DC
:100EE000580A0895982F8091580A883A58F48091AA
:100EF000580AE82FFF27E15AF64F906893838F5FD7
:100F00008093580A0895982F8091EE03882321F04A
:100F1000892F0E9472870895892F0E946287089501
:100F2000883A10F48093580A089580E090E2E2E64F
:100F3000F9E091938F5F883AE0F308954FB721E885
:100F400030E0F8948091C9008F778093C900809138
:100F5000C9008F7B8093C9008091C9008F7D8093E9
:100F6000C9005A9A52985B9A539A832F9927809373
:100F7000CD002093CC008091C80082608093C8008F
:100F800088E18093C9008091CA008F778093CA005E
:100F90008091CA008F7B8093CA008091CA008F7DA8
:100FA0008093CA008091CA008F7E8093CA0080918E
:100FB000CA00877F8093CA008091C90084608093B3
:100FC000C9008091CA0084608093CA008091CA00E1
:100FD00082608093CA008091C90081608093C900BB
:100FE0008091C80087FF03C08091CE00F9CF809127
:100FF000C90080688093C9004FBF3CE73093DB088D
:101000002DE7209306098EE88093DC081092F808FB
:101010001092F7081092E10880EE8093DE0830937A
:10102000330920935E0910923F0910923E091092F5
:10103000410910924009109243091092420984EF2D
:1010400091E090933D0980933C0990933B098093F4
:101050003A0990933909809338091092350989E843
:101060008093340910925C0910925D0980E98093A5
:10107000360930930B0A2093360A10920D0A8AE83B
:1010800080930C0A1092130A1092120A1092110AFD
:101090001092150A1092160A1092170A1092180A46
:1010A00010921A0A10921B0A10921C0A10921D0A22
:1010B0001092210A1092200A10921F0A10921E0A02
:1010C00080EA80930E0A3093070920933209109228
:1010D00009098DE8809308091092310980ED809309
:1010E0000A098BE780935F0980E88093600910927A
:1010F00061098091E10890E2E2E6F9E091938F5F67
:10110000883AE0F38DE780930A0A0895CF93C82FB9
:101110008091FD03803879F48C2F0E942273809394
:10112000F0038091F003882331F1C093570A809136
:10113000F0038F5F16C08F37F1F48091500A882337
:1011400029F48C2F80958F708093500A0E942F7203
:10115000809361098FE599E09093F2038093F10306
:101160008DEA8093F0038091C9008F7E8093C9003F
:1011700082E08093EF03C093FD03CF9108953091F7
:10118000EF03332331F08091EF0381508093EF031D
:1011900008958091F003882381F14091F0039091AC
:1011A000FE03413091F4292F3093FE038091C90052
:1011B00080618093C9008091EE03882319F03093F9
:1011C000EE0310C04093EE030DC0E091F103F091E7
:1011D000F2038191F093F203E093F103282F980F2B
:1011E0009093FE038091C80085FFFCCF2093CE0032
:1011F0008091F00381508093F00308952FB740E071
:10120000F894E0E0F0E081E2809357009491E2E00E
:10121000F0E0809357003491E4E0F0E080935700D1
:1012200084912FBF9E3199F4363941F4893011F4FD
:1012300041E00DC08A3059F442E009C0373939F431
:10124000863011F443E003C0853009F444E0842F74
:10125000992708959FB7F8948091C900877F80935C
:10126000C9008091C9008F7E8093C9008091C90018
:101270008F778093C9008091C9008F7B8093C900CC
:101280008091C9008F7D8093C90052985A9A5398D3
:101290005B9A9FBF08951F93CF93DF93182F809180
:1012A000ED03882309F4A7C08091A301181709F45E
:1012B000A2C08091EC03882321F40E94FE888093D1
:1012C000EC0382ED91E090933F0180933E0188E52D
:1012D00091E19F938F93CCE2D5E1DF93CF93E0919F
:1012E0000204F091030409950F900F900F900F9056
:1012F000812F9927AA27BB27FC01099778F5ED5480
:10130000FF4F20910204309103040C940C8E84E56D
:1013100091E102C08BE491E19F938F93DF93CF9390
:10132000F901099527C086E491E1F6CF8EE391E1BA
:10133000F3CF86E391E19F938F93DF93CF93F901EE
:10134000099588ED91E090933F0180933E0112C092
:1013500081E391E1E1CF85E691E1DECF8BE691E19A
:101360009F938F93DF93CF93E0910204F091030456
:10137000099510E00F900F900F900F908091EC0363
:10138000843011F0823011F50E942A89812F81501A
:10139000833018F40E94426E2CC0143019F40E945D
:1013A000508327C0153019F40E94858122C018305F
:1013B00019F40E9403811DC0163019F40E949E8703
:1013C00018C01730B1F40E94B67F13C0112389F002
:1013D00081E891E19F938F938CE295E19F938F93A6
:1013E000E0910204F091030409950F900F900F9083
:1013F0000F901093A301DF91CF911F9108950F9348
:101400001F9381E08093ED034091A201E1EEF0E1B2
:1014100020E030E05FE4849199272F5F3F4F829F67
:10142000B001839F700D929F700D1124462751507B
:10143000319657FFF0CF4093A201E9EBF0E120E0B5
:1014400030E057E2849199272F5F3F4F829FB00190
:10145000839F700D929F700D112446275150319635
:1014600057FFF0CF4093A2018091EC03882321F431
:101470000E94FE888093EC038091A201833459F08E
:1014800088E190E029E20FB6F894A8958093600077
:101490000FBE2093600081EC94E890930304809346
:1014A00002040E9439098EE690E09F938F9388E5AD
:1014B00090E09F938F931F921F92809101016AE0A9
:1014C0000E94658D892F99279F938F9380910101A9
:1014D0000E94658D99279F938F938CE991E19F934B
:1014E0008F930CE215E11F930F93E0910204F091AA
:1014F0000304099581EE90E19F938F931F930F93BF
:10150000E0910204F0910304099589EB90E19F9327
:101510008F931F930F93E0910204F09103040995B8
:101520000E94390983EC8093810080916F00806272
:1015300080936F008DB79EB746968DBF1F910F9118
:1015400008958091AE068D3338F080914F0887FD65
:1015500003C08CE38093AE0680915E06882331F051
:101560008055853618F08FE780935E060895809148
:10157000ED03882309F477C08091FF0381508093A5
:10158000FF03882309F053C089E18093FF03809112
:10159000AE068E3338F080914F0887FD03C08DE38F
:1015A0008093AE068091DB02823820F58091A40200
:1015B0009091A502885E934020F08091DA088436ED
:1015C00020F4109201041092000480910004909184
:1015D0000104009739F1019790930104809300046E
:1015E000419728F180914F0884FF21C08091A20289
:1015F00084601BC08091DB02853BC8F09091AE06F1
:1016000084E1989FC00111244096209100043091FC
:1016100001042817390730F42F5F3F4F309301043E
:10162000209300048091A2028B7F8093A20290916C
:10163000A301963019F40E94BF880FC08091A601C3
:10164000882321F081508093A601089586E9809334
:10165000A601943011F40E94C1838091A2018334C9
:1016600011F01092ED0308951F920F920FB60F9292
:1016700011242F933F934F935F936F937F938F9397
:101680009F93AF93BF93EF93FF932091CE008091F0
:10169000B2018823B1F02093C6008091B20182305C
:1016A000B9F52F3FA9F58FEF94E3ACE0B0E0C29716
:1016B000A109B109B7FFFBCF809145048093CE000B
:1016C00027C09091A301892F8150833020F4822F6D
:1016D0000E949D6E1DC0943021F4822F0E94B4831D
:1016E00017C0953021F4822F0E94F38211C09830E8
:1016F00021F4822F0E9404810BC0963021F4822FA6
:101700000E94868805C0973019F4822F0E941380AA
:10171000FF91EF91BF91AF919F918F917F916F91C9
:101720005F914F913F912F910F900FBE0F901F909F
:101730001895FB01DC0102C005900D92415050400C
:10174000D8F70895FC014150504030F00190061642
:10175000D1F73197CF010895882799270895A0E000
:10176000B0E0E5EBFBE80C94DD8D6C017B01EA0158
:10177000590121978FEFCF3FD80789F08601089450
:10178000C11CD11CC7010894E11CF11CF50109958D
:10179000F80180832197FFEFCF3FDF0779F7EAE079
:1017A000CDB7DEB70C94F98DCF92DF92EF92FF9216
:1017B0000F931F937C016B01FB010995082FC70153
:1017C0000196F6010995182FC8011F910F91FF90FE
:1017D000EF90DF90CF900895A0E0B0E0E2EFFBE85B
:1017E0000C94DF8D8C017B01EA01690121978FEF59
:1017F000CF3FD80771F0F70121917F01C8010F5F3A
:101800001F4F622FF60109952197FFEFCF3FDF07AA
:1018100091F7E8E0CDB7DEB70C94FB8DCF92DF9265
:10182000EF92FF920F931F936C018B017A01FA01E3
:101830000995812F9927682FC6010196F70109950F
:101840001F910F91FF90EF90DF90CF900895505827
:10185000BB27AA270ED0E0C0D1D030F0D6D020F0E0
:1018600031F49F3F11F41EF4C6C00EF4E095E7FB7F
:10187000BCC0E92FE2D080F3BA1762077307840770
:10188000950718F071F49EF5FAC00EF4E0950B2E52
:10189000BA2FA02D0B01B90190010C01CA01A001C2
:1018A0001124FF27591B99F0593F50F4503E68F11D
:1018B0001A16F040A22F232F342F4427585FF3CF5E
:1018C000469537952795A795F0405395C9F77EF42F
:1018D0001F16BA0B620B730B840BBAF09150A1F078
:1018E000FF0FBB1F661F771F881FC2F70EC0BA0FFE
:1018F000621F731F841F48F4879577956795B79586
:10190000F7959E3F08F0B3CF9395880F08F099277D
:10191000EE0F97958795089598D088F09F5790F08F
:10192000B92F9927B751A0F0D1F0660F771F881F04
:10193000991F1AF0BA95C9F712C0B13081F09FD043
:10194000B1E008959CC0672F782F8827B85F39F0E1
:10195000B93FCCF3869577956795B395D9F73EF463
:1019600090958095709561957F4F8F4F9F4F08950B
:10197000E89409C097FB3EF4909580957095619529
:101980007F4F8F4F9F4F9923A9F0F92F96E9BB27DF
:101990009395F695879577956795B795F111F8CF5B
:1019A000FAF4BB0F11F460FF1BC06F5F7F4F8F4FC6
:1019B0009F4F16C0882311F096E911C0772321F0BC
:1019C0009EE8872F762F05C0662371F096E8862F54
:1019D00070E060E02AF09A95660F771F881FDAF7AB
:1019E000880F9695879597F9089597F99F6780E8EE
:1019F00070E060E008959FEF80EC089500240A9461
:101A00001616170618060906089500240A941216D9
:101A10001306140605060895092E0394000C11F40C
:101A2000882352F0BB0F40F4BF2B11F460FF04C0B9
:101A30006F5F7F4F8F4F9F4F089557FD9058440F12
:101A4000551F59F05F3F71F04795880F97FB991F1D
:101A500061F09F3F79F087950895121613061406DA
:101A6000551FF2CF4695F1DF08C016161706180667
:101A7000991FF1CF86957105610508940895E89442
:101A8000BB2766277727CB0197F90895629FD0017E
:101A9000739FF001829FE00DF11D649FE00DF11D29
:101AA000929FF00D839FF00D749FF00D659FF00DD8
:101AB0009927729FB00DE11DF91F639FB00DE11DC5
:101AC000F91FBD01CF0111240895991B79E004C0CD
:101AD000991F961708F0961B881F7A95C9F780956D
:101AE0000895AA1BBB1B51E107C0AA1FBB1FA61765
:101AF000B70710F0A61BB70B881F991F5A95A9F7B7
:101B000080959095BC01CD01089597FB092E07267D
:101B10000AD077FD04D0E5DF06D000201AF47095D6
:101B200061957F4F0895F6F7909581959F4F0895A1
:101B3000A1E21A2EAA1BBB1BFD010DC0AA1FBB1FD1
:101B4000EE1FFF1FA217B307E407F50720F0A21B43
:101B5000B30BE40BF50B661F771F881F991F1A94B0
:101B600069F760957095809590959B01AC01BD01DA
:101B7000CF01089597FB092E05260ED057FD04D0FE
:101B8000D7DF0AD0001C38F4509540953095219548
:101B90003F4F4F4F5F4F0895F6F7909580957095A2
:101BA00061957F4F8F4F9F4F08952F923F924F9295
:101BB0005F926F927F928F929F92AF92BF92CF92DD
:101BC000DF92EF92FF920F931F93CF93DF93CDB7E6
:101BD000DEB7CA1BDB0B0FB6F894DEBF0FBECDBF5E
:101BE00009942A88398848885F846E847D848C842F
:101BF0009B84AA84B984C884DF80EE80FD800C8138
:101C00001B81AA81B981CE0FD11D0FB6F894DEBF1A
